:020000040800F2
:1000000000040020A51F0008F71F0008F71F0008C4
:10001000F71F0008F71F0008F71F00080000000086
:10002000000000000000000000000000F71F0008B2
:10003000F71F000800000000F71F000865200208F5
:10004000F1210208F3210208F5210208F921020832
:10005000192202081B2202081D220208412202085E
:100060006522020889220208AD220208D122020874
:10007000D3220208D5220208D7220208D922020878
:10008000DB220208DD220208DF220208F71F000837
:10009000F71F0008F71F0008F71F0008E1220208F9
:1000A0002D2302082F2302083123020833230208DC
:1000B000352302083923020865230208D5230208E4
:1000C000D7230208D9230208DB230208DD23020814
:1000D000E1230208512502087924020815260208A6
:1000E000D92602089D2702089F270208A127020897
:1000F000A52702080D2802080F2802081128020867
:1001000013280208152802081728020819280208CF
:100110001D280208F1280208F3280208F528020821
:10012000012A0208032A0208052A0208072A0208EF
:1001300000000000000000000000000000000000BF
:1001400000000000000000000000000000000000AF
:10015000000000000000000000000000000000009F
:10016000000000000000000000000000000000008F
:10017000000000000000000000000000000000007F
:10018000000000000000000000000000000000006F
:10019000000000000000000000000000000000005F
:1001A000000000000000000000000000000000004F
:1001B000000000000000000000000000000000003F
:1001C000000000000000000000000000000000002F
:1001D000000000000000000000000000000000001F
:0401E0005FF8E0F1F3
:1001E800032A70B404460D4626D941EA000313F0E9
:1001F800030F13D020782B78984208BF294606D0E1
:100208001EE014F8010F11F8013F984218D1012A95
:1002180002F1FF32F5D1002070BC70470B4604464E
:1002280051F8045B50F8046BAE4204D1043A04461A
:10023800032A0B46F2D81D461046002ADAD1EBE70E
:10024800C01AE9E7032A2DE9F00109D82AB10023E9
:10025800CC5CC45401339342FAD1BDE8F001704735
:100268000B468218014603E02478013301F8014B5C
:1002780011F0030F1C46F7D113F003055DD06E4251
:10028800C5F1040CED009B594FEACC0C08E004348E
:10029800A7593B4607FA0CF748EA070741F8047BD9
:1002A800571A23FA05F8032FF1DC03E014F8013B91
:1002B80001F8013B8A42F9D8CFE753F8404C41F89E
:1002C800404C53F83C4C41F83C4C53F8384C41F8FE
:1002D800384C53F8344C41F8344C53F8304C41F80E
:1002E800304C53F82C4C41F82C4C53F8284C41F81E
:1002F800284C53F8244C41F8244C53F8204C41F82E
:10030800204C53F81C4C41F81C4C53F8184C41F83D
:10031800184C53F8144C41F8144C53F8104C41F84D
:10032800104C53F80C4C41F80C4C53F8084C41F85D
:10033800084C53F8044C41F8044C561A1D460C4618
:10034800403340313F2EB8DC2B460FE053F8101CE9
:1003580044F8101C53F80C1C44F80C1C53F8081CE7
:1003680044F8081C53F8041C44F8041C161B2146C6
:100378001D46103410330F2EE8DC2B4602E02468AB
:1003880041F8044B551A1C46032D03F10403F6DC0F
:1003980090E700BF032AC9B270B408D82AB103464F
:1003A800121803F8011B9342FBD170BC70478218E6
:1003B800044601E004F8011B14F0030FFAD14FF0D2
:1003C800013303FB01F31FE044F8403C44F83C3C94
:1003D80044F8383C44F8343C44F8303C44F82C3C6D
:1003E80044F8283C44F8243C44F8203C44F81C3C9D
:1003F80044F8183C44F8143C44F8103C44F80C3CCD
:1004080044F8083C44F8043C161B254640343F2E6B
:10041800DADC2C4607E044F8103C44F80C3C44F87D
:10042800083C44F8043C161B254610340F2EF2DC19
:1004380001E045F8043B541B032CFADC01E005F805
:10044800011B9542FBD3B0E710F0030F38B5044603
:1004580012D10368A3F1013222EA030313F0803FAB
:100468000AD1031D184653F8042BA2F1013525EAD9
:10047800020212F0803FF5D003782BB1431C1846D6
:1004880013F8012B002AFAD100F076F9204638BD7E
:10049800C9B2F0B4002950D010F0030F10D003787F
:1004A800002B79D0994246D0431C05E013F8012B64
:1004B800002A3FD091423ED013F0030F1846F5D1E1
:1004C800036841EA01270646A3F1013247EA0747D4
:1004D80022EA030212F0803F1DD187EA0303A3F149
:1004E800013222EA030313F0803F14D1043002E002
:1004F80012F0803F0FD1064650F8043BA3F10135B6
:1005080087EA030225EA0303A2F1013413F0803FCE
:1005180024EA0202ECD033783046002B3CD09942D2
:1005280009D0731C01E0914205D0184613F8012B3D
:10053800002AF8D11046F0BC704710F0030F0CD019
:100548000378002BF7D0431C03E013F8012B002A93
:10055800F1D013F0030F1846F7D102680346A2F151
:10056800013121EA020212F0803F0AD10430034629
:1005780050F8042BA2F1013121EA020212F0803F67
:10058800F5D01A781846002AD5D00133184613F842
:10059800012B002AFAD1CEE71846CCE780EA0102FF
:1005A80012F0030F3AD110F0030220F0030021F0FB
:1005B800030150F804CB08BF51F8043B0DD082F07A
:1005C80003024FEAC2026FF07F4323FA02F251F8A6
:1005D800043B4CEA020C43EA020300BFACF10132CF
:1005E8009C4501BF22EA0C0212F0803F50F804CB70
:1005F80051F8043BF2D04FEA0C604FEA1C2C01285A
:1006080028BFB0EB036F08BF1B0AF4D003F0FF0349
:100618004FEA1060A0EB0300704700BF10F0030F13
:100628000AD010F8012B11F8013B012A28BF9A4281
:10063800F4D0A2EB030070474DF8045D4DF8044D6B
:100648004FF0010242EA022242EA024201F0030CA0
:1006580021F0030150F8044B51F8045BBCF1020F80
:1006680026D04BD824F07F4CBCEB152FA4EB02030B
:1006780023EA04030DD113EAC21308BF51F8045B3F
:100688000AD18CEA040CBCEB056F0CD150F8044B72
:10069800E8E74FEA15255CE033F07F4352D10D7847
:1006A8004FEA146C55E04FEA146C05F0FF0550E072
:1006B8004FEA044CA4EB02034FEA1C4C23EA040360
:1006C800BCEB154F17D113EAC21308BF51F8045BEE
:1006D80007D18CEA040CBCEB054F08D150F8044B49
:1006E800E6E71B042ED10D884FEA144C31E04FEA9F
:1006F80005454FEA144C4FEA15452AE004F0FF0C73
:10070800BCEB156FA4EB020323EA04030DD113EA33
:10071800C21308BF51F8045B0AD18CEA040CBCEB85
:10072800052F0AD150F8044BE8E74FEA156510E0A9
:1007380014F0FF0F06D051F8045B4FEA142C25F093
:100748007F4506E04FF000005DF8044B5DF8045B60
:1007580070470CF0FF0205F0FF00012828BF904207
:1007680004BF4FEA1C2C2D0AF3D0A2EB00005DF861
:10077800044B5DF8045B704780EA0102844612F07E
:10078800030F4FD111F0030F32D14DF8044D11F082
:10079800040F51F8043B0BD0A3F101329A4312F035
:1007A800803F04BF4CF8043B51F8043B16D100BF0E
:1007B80051F8044BA3F101329A4312F0803FA4F19F
:1007C80001320BD14CF8043BA24312F0803F04BF26
:1007D80051F8043B4CF8044BEAD023460CF8013B93
:1007E80013F0FF0F4FEA3323F8D15DF8044B70473D
:1007F80011F0010F06D011F8012B0CF8012B002A7B
:1008080008BF704711F0020FBFD031F8022B12F069
:10081800FF0F16BF2CF8022B8CF8002012F47F4F24
:10082800B3D1704711F8012B0CF8012B002AF9D12C
:10083800704700BF20F0030110F00300C0F1000072
:1008480051F8043B00F1040C4FEACC0C6FF00002A5
:100858001CBF22FA0CF213434FF0010C4CEA0C2C8B
:100868004CEA0C4CA3EB0C0222EA030212EACC126B
:1008780004BF51F8043B0430F4D013F0FF0F1FBF3E
:10088800013013F47F4F013013F47F0F18BF01308C
:10089800704700BFF0B4002A46D041EA000313F0C5
:1008A80003032CD1032A07460E4643D904680D6872
:1008B800AC423FD1043A37D0A4F1013525EA04040B
:1008C80014F0803F18BF18462CD1041D0D1D0EE0F2
:1008D80054F8043B55F8041BA3F101308B4220EA7D
:1008E800030027D1043A1FD010F0803F1ED1032AFD
:1008F80027462E46ECD820462946002A1DD00478E3
:10090800013A0D78AC420CD172B18CB1002302E0EF
:1009180093420BD064B1013310F8014FCD5CAC4267
:10092800F6D0601BF0BC70471046FBE70020F9E7E3
:100938002046F7E738463146E1E724782D78F0E796
:1009480041EA000313F0030F0B4670B414BF0024F0
:100958000124032A94BF002404F001040546D4B9F5
:10096800BAB10E782B46013A03F8016B56B1AC1CAC
:100978007AB111F8015F2346013A04F8015C0134A9
:10098800002DF5D12AB19A18002103F8011B9342D2
:10099800FBD170BC7047194653F8044BA4F10136DB
:1009A80026EA040616F0803FDAD1043A45F8044BEB
:1009B800032A1946EFD8D3E701232DE9F0071D468E
:1009C80000264FF0FF37AC1900EB070C8C420DD214
:1009D8001CF805C010F80480E0452ED201252646F3
:1009E800E31BAC198C4200EB070CF1D34FF0010963
:1009F80000264D464FF0FF3C1360AC1900EB0C0885
:100A0800A1420ED918F8058010F804A0C2451AD9D9
:100A180001252646CCEB0409AC19A14200EB0C08D1
:100A2800F0D80CF101000137B8423CBF994638466E
:100A3800C2F80090BDE8F00770470BD00123374695
:100A48001D46F618BFE709D04FF00109B4464D46D8
:100A58004E44D2E79D4205D00135B4E74D4505D057
:100A68000135CAE72B4626460125ACE7A9462646A6
:100A78000125C2E72DE9F04FADF5826D81B014462E
:100A8800074610460DF580628B460C3219461D4606
:100A9800FFF792FF03AE04A901F57E72331F0090A1
:100AA80043F8045F9342FBD14DB1681E0023E25C1A
:100AB800C11A013303AEAB4246F82210F7D1DDF874
:100AC8000C142046009A6118FFF78AFB002877D19A
:100AD8000099814605F1FF380646C1F101020192ED
:100AE8005A46AB4609EB0B0501F1FF3AB81800214D
:100AF800AA1A00F0E5F900284FD1002D00F0C080B7
:100B08007B1903A913F8013C51F82330002B4CD171
:100B1800009B9E4228BF334698450FD903EB090135
:100B2800E05C7A18795C884205D038E012F8011F39
:100B3800E05C884233D101339845F7D8009A964251
:100B480080F0A48007EB090214F80A10534612F843
:100B58000A20914204BF0AEB0901791807D095E0F1
:100B680014F802C011F8010D844503D113465A1E2A
:100B7800B342F5D101369E4200F28D80DDF80C6457
:100B88002A46B144C6EB0B0609EB0B05B818002141
:100B9800AA1A00F095F90028AFD0002071E0019A58
:100BA8000026914499442A46EEE7002EFAD0DDF853
:100BB8000C2493423CBFC2EB0B0306469944F2E770
:100BC800009E4FF000080099AB1BB34238BF334674
:100BD800C1F101026E1E019201F1FF3A5A4689469F
:100BE800AB460133CDF80C3408EB0B05B8180021DF
:100BF800AA1A00F065F90028CFD1002D40D07B1942
:100C080003A913F8013C51F82330002B30D1B1452A
:100C180013D208EB090314F80910FA18FB5C99427F
:100C280018BF4B4627D14B4604E012F8011FE05C81
:100C3800884220D10133B342F7D3BAF1FF3F53467C
:100C48002CD007EB080C14F80A101CF80A20914263
:100C58000CD10AEB0802BA1804E0E05C12F8011D96
:100C6800884203D1013BF8D260460AE0DDF80C3433
:100C780098442A46B8E701992A4688449844B3E735
:100C8800284605B00DF5806DBDE8F08F009B013654
:100C98009E427FF673AF07EB0900F2E707EB080CFB
:100CA8006046EEE72DE9F04F8346037885B00C46A1
:100CB800002B00F0F9800A78A2B106460131012024
:100CC80002E011F8012B8AB1934214BF002000F012
:100CD800010016F8013F0D46002BF2D12B782BB1FD
:100CE8004FF0000B584605B0BDE8F08F0028F9D149
:100CF8000BF101002178FFF7CBFB2D1BA5F10102B9
:100D0800534243EB0203002808BF43F001030746A0
:100D180083B90BEB0508404594BFC0EB08084FF0BA
:100D280001081F2D08D9414622462B46FFF7A2FE8F
:100D38008346D7E78346D5E7294603AA2046FFF727
:100D48003BFE03996118814620464A46FFF748FA58
:100D580000284FD109F1FF33C9F10102064601927B
:100D680082464246C84699460AEB050BB818002148
:100D7800C2EB0B0200F0A4F80028B1D1BBF1000FC0
:100D8800B0D046452CBF334643469D420FD903EBAE
:100D98000A01E05C7A18795C884205D075E012F89F
:100DA800011FE05C884270D101339D42F7D1B04504
:100DB8007DD907EB0A0214F809104B4612F80920EE
:100DC800914202BF09EB0A01AC46791806D06EE0E1
:100DD800A55C11F8010D854203D113465A1EB34292
:100DE800F6D1654601369E4267D8039E5A46B244FC
:100DF800AE1BB9E7C9F10101C9EB0503424600265C
:100E080009F1FF3A88464B4538BF4B4601330393F7
:100E180006EB050BB8180021C2EB0B0200F050F8E6
:100E280000287FF45DAFBBF1000F3FF45BAF4D4589
:100E380012D906EB090314F80910FA18FB5C994259
:100E480008BF4B4605D026E012F8011FE05C884237
:100E580022D101339D42F7D1BAF1FF3F534628D042
:100E680007EB060C14F80A101CF80A20914217D157
:100E78000AEB0602BA1804E0E05C12F8011D884289
:100E88000ED1013BF8D2E3462CE7019A00269244A2
:100E98005A469A4468E74B4646445A46F618B7E716
:100EA800039B5A46F618B3E70D46012016E743465A
:100EB80098E707EB060CE34614E707EB0A0B11E784
:100EC80010F0030F034670B4C9B211D0002A22D023
:100ED80003788B421DD0013A013005E0DAB110F8F1
:100EE800014B013A8C4218D010F0030F0346F5D19C
:100EF800032A14D87AB1187888420ED0541E5D1C83
:100F080003E015F8016B8E4203D0013C2846F8D265
:100F1800002070BC70471046FBE71846F9E741EA25
:100F2800012646EA0646184653F8044B86EA0404A6
:100F3800A4F1013525EA040414F0803F03D1043AF2
:100F48001846032AEFD80346D4E700BF0000000084
:100F5800C1F30A5C0246ACF57E7C2DE9F84FACF192
:100F68000704132C0B4606460F468946804627DCA5
:100F7800002C52DB4FF6FF7CC0F20F0C4CFA04FA3F
:100F88000AEA0105054317D037A3D3E9002300F087
:100F980075F80022002300F0B3FC002856D0002F7B
:100FA80005DD4FF4801353FA04F407EB040929EA2A
:100FB8000A0900264B46324610461946BDE8F88F06
:100FC800332C07DDB4F5806FF6D100F057F80246F0
:100FD8000B46F1E74FF0FF3BACF11B0C2BFA0CFB77
:100FE8001BEA000FE8D020A3D3E9002300F046F85D
:100FF8000022002300F084FC40B3002F0ADD142CEB
:1010080006D00126C4F13404A64016EB080601D325
:1010180007F1010926EA0B0619E013A3D3E9002317
:1010280000F02CF80022002300F06AFC78B1002FB1
:1010380013DB46EA07054FF000094D45C3F6F07982
:101048000CBF2E46002608BFA94600E0B9464B460D
:10105800324610461946BDE8F88F00264FF0004981
:10106800F5E700BFAFF300809C7500883CE4377E4D
:1010780081F0004102E000BF83F0004330B54FEA41
:1010880041044FEA430594EA050F08BF90EA020FAE
:101098001FBF54EA000C55EA020C7FEA645C7FEA41
:1010A800655C00F0E2804FEA5454D4EB5555B8BF64
:1010B8006D420CDD2C4480EA020281EA030382EAD5
:1010C800000083EA010180EA020281EA0303362D67
:1010D80088BF30BD11F0004F4FEA01314FF4801C3A
:1010E8004CEA113102D0404261EB410113F0004F4C
:1010F8004FEA03334CEA133302D0524263EB430303
:1011080094EA050F00F0A780A4F10104D5F1200EA0
:101118000DDB02FA0EFC22FA05F2801841F10001FB
:1011280003FA0EF2801843FA05F359410EE0A5F1CF
:1011380020050EF1200E012A03FA0EFC28BF4CF000
:10114800020C43FA05F3C01851EBE37101F00045B6
:1011580007D54FF0000EDCF1000C7EEB00006EEBC3
:101168000101B1F5801F1BD3B1F5001F0CD349084D
:101178005FEA30004FEA3C0C04F101044FEA4452A4
:1011880012F5800F80F09A80BCF1004F08BF5FEA2B
:10119800500C50F1000041EB045141EA050130BD0B
:1011A8005FEA4C0C404141EB010111F4801FA4F1AE
:1011B8000104E9D191F0000F04BF01460020B1FA03
:1011C80081F308BF2033A3F10B03B3F120020CDA3B
:1011D8000C3208DD02F1140CC2F10C0201FA0CF019
:1011E80021FA02F10CE002F11402D8BFC2F1200C7E
:1011F80001FA02F120FA0CFCDCBF41EA0C01904034
:10120800E41AA2BF01EB0451294330BD6FEA04047C
:101218001F3C1CDA0C340EDC04F11404C4F1200267
:1012280020FA04F001FA02F340EA030021FA04F379
:1012380045EA030130BDC4F10C04C4F1200220FAD0
:1012480002F001FA04F340EA0300294630BD21FA0E
:1012580004F0294630BD94F0000F83F4801306BFD4
:1012680081F480110134013D4EE77FEA645C18BFC8
:101278007FEA655C29D094EA050F08BF90EA020F5F
:1012880005D054EA000C04BF1946104630BD91EA57
:10129800030F1EBF0021002030BD5FEA545C05D15A
:1012A8004000494128BF41F0004130BD14F5800499
:1012B8003CBF01F5801130BD01F0004545F0FE410D
:1012C80041F470014FF0000030BD7FEA645C1ABF42
:1012D800194610467FEA655C1CBF0B46024650EA79
:1012E800013406BF52EA033591EA030F41F40021A5
:1012F80030BD00BF90F0000F04BF0021704730B52B
:101308004FF4806404F132044FF000054FF00001FF
:1013180050E700BF90F0000F04BF0021704730B5C0
:101328004FF4806404F1320410F0004548BF404295
:101338004FF000013EE700BF42004FEAE2014FEAEA
:1013480031014FEA02701FBF12F07F4393F07F4FC5
:1013580081F06051704792F0000F14BF93F07F4FF7
:10136800704730B54FF4607401F0004521F000413A
:1013780020E700BF50EA010208BF704730B54FF0C0
:1013880000050AE050EA010208BF704730B511F0C5
:10139800004502D5404261EB41014FF4806404F1FD
:1013A80032045FEA915C3FF4DCAE4FF003025FEA7F
:1013B800DC0C18BF03325FEADC0C18BF033202EB07
:1013C800DC02C2F1200300FA03FC20FA02F001FA61
:1013D80003FE40EA0E0021FA02F11444C1E600BF00
:1013E80070B54FF0FF0C4CF4E06C1CEA11541DBFB3
:1013F8001CEA135594EA0C0F95EA0C0F00F0DEF87E
:101408002C4481EA030621EA4C5123EA4C5350EA62
:10141800013518BF52EA033541F4801143F48013B3
:1014280038D0A0FB02CE4FF00005E1FB02E506F044
:101438000042E0FB03E54FF00006E1FB03569CF099
:10144800000F18BF4EF0010EA4F1FF04B6F5007F9F
:1014580064F5407404D25FEA4E0E6D4146EB060611
:1014680042EAC62141EA55514FEAC52040EA5E509A
:101478004FEACE2EB4F1FD0C88BFBCF5E06F1ED844
:10148800BEF1004F08BF5FEA500E50F1000041EB7B
:10149800045170BD06F0004646EA010140EA020028
:1014A80081EA0301B4EB5C04C2BFD4EB0C0541EA4A
:1014B800045170BD41F480114FF0000E013C00F35F
:1014C800AB8014F1360FDEBF002001F0004170BD83
:1014D800C4F10004203C35DA0C341BDC04F114049C
:1014E800C4F1200500FA05F320FA04F001FA05F228
:1014F80040EA020001F0004221F0004110EBD370F5
:1015080021FA04F642EB06015EEA430E08BF20EA20
:10151800D37070BDC4F10C04C4F1200500FA04F3C3
:1015280020FA05F001FA04F240EA020001F0004155
:1015380010EBD37041F100015EEA430E08BF20EAC8
:10154800D37070BDC4F1200500FA05F24EEA020E10
:1015580020FA04F301FA05F243EA020321FA04F03F
:1015680001F0004121FA04F220EA020000EBD370F6
:101578005EEA430E08BF20EAD37070BD94F0000FF6
:101588000FD101F00046400041EB010111F4801F2A
:1015980008BF013CF7D041EA060195F0000F18BFDB
:1015A800704703F00046520043EB030313F4801F17
:1015B80008BF013DF7D043EA0603704794EA0C0FD1
:1015C8000CEA135518BF95EA0C0F0CD050EA4106E7
:1015D80018BF52EA4306D1D181EA030101F0004164
:1015E8004FF0000070BD50EA410606BF104619468C
:1015F80052EA430619D094EA0C0F02D150EA013698
:1016080013D195EA0C0F05D152EA03361CBF1046D8
:1016180019460AD181EA030101F0004141F0FE4177
:1016280041F470014FF0000070BD41F0FE4141F4FB
:10163800780170BD70B54FF0FF0C4CF4E06C1CEAFB
:1016480011541DBF1CEA135594EA0C0F95EA0C0FB0
:1016580000F0A7F8A4EB050481EA030E52EA03356B
:101668004FEA013100F088804FEA03334FF080558C
:1016780045EA131343EA12634FEA022245EA1115B9
:1016880045EA10654FEA00260EF000419D4208BF6A
:10169800964244F1FD0404F5407402D25B084FEA17
:1016A8003202B61A65EB03055B084FEA32024FF4C3
:1016B80080104FF4002CB6EB020E75EB030E22BF20
:1016C800B61A754640EA0C005B084FEA3202B6EBE0
:1016D800020E75EB030E22BFB61A754640EA5C008F
:1016E8005B084FEA3202B6EB020E75EB030E22BF1F
:1016F800B61A754640EA9C005B084FEA3202B6EB20
:10170800020E75EB030E22BFB61A754640EADC00DE
:1017180055EA060E18D04FEA051545EA16754FEA40
:1017280006164FEAC30343EA52734FEAC2025FEA5E
:101738001C1CC0D111F4801F0BD141EA00014FF0ED
:1017480000004FF0004CB6E711F4801F04BF0143BE
:101758000020B4F1FD0C88BFBCF5E06F3FF6AFAEDA
:10176800B5EB030C04BFB6EB020C5FEA500C50F16A
:10177800000041EB045170BD0EF0004E4EEA1131ED
:1017880014EB5C04C2BFD4EB0C0541EA045170BDF4
:1017980041F480114FF0000E013C90E645EA060E38
:1017A8008DE60CEA135594EA0C0F08BF95EA0C0F66
:1017B8003FF43BAF94EA0C0F0AD150EA01347FF4AE
:1017C80034AF95EA0C0F7FF425AF104619462CE785
:1017D80095EA0C0F06D152EA03353FF4FDAE1046E8
:1017E800194622E750EA410618BF52EA43067FF439
:1017F800C5AE50EA41047FF40DAF52EA43057FF4C9
:10180800EBAE12E74FF0FF3C06E000BF4FF0010CD3
:1018180002E000BF4FF0010C4DF804CD4FEA410C37
:101828007FEA6C5C4FEA430C18BF7FEA6C5C1BD004
:1018380001B050EA410C0CBF52EA430C91EA030F85
:1018480002BF90EA020F0020704710F1000F91EAE2
:10185800030F58BF994208BF90422CBFD8176FEAB0
:10186800E37040F0010070474FEA410C7FEA6C5C7E
:1018780002D150EA013C07D14FEA430C7FEA6C5C85
:10188800D6D152EA033CD3D05DF8040B704700BFB1
:101898008446104662468C461946634600E000BFFF
:1018A80001B5FFF7B7FF002848BF10F1000F01BDD1
:1018B8004DF808EDFFF7F4FF0CBF012000205DF89C
:1018C80008FB00BF4DF808EDFFF7EAFF34BF012021
:1018D80000205DF808FB00BF4DF808EDFFF7E0FFBA
:1018E80094BF012000205DF808FB00BF4DF808ED0B
:1018F800FFF7CEFF94BF012000205DF808FB00BF72
:101908004DF808EDFFF7C4FF34BF012000205DF853
:1019180008FB00BF4FEA4102B2F1E04324BFB3F530
:10192800001CDCF1FE5C0DD901F0004C4FEAC0024E
:101938004CEA5070B2F1004F40EB830008BF20F032
:101948000100704711F0804F21D113F13872BCBFEC
:1019580001F00040704741F480114FEA5252C2F141
:101968001802C2F1200C10FA0CF320FA02F018BF8A
:1019780040F001004FEAC1234FEAD32303FA0CFCDD
:1019880040EA0C0023FA02F34FEA4303CCE77FEA6C
:10199800625307D150EA01331EBF4FF0FE4040F4B6
:1019A8004000704701F0004040F0FE4040F4000065
:1019B800704700BF80F0004002E000BF81F00041A6
:1019C80042001FBF5FEA410392EA030F7FEA226CDD
:1019D8007FEA236C6AD04FEA1262D2EB1363C1BF6D
:1019E800D218414048404140B8BF5B42192B88BFDC
:1019F800704710F0004F40F4000020F07F4018BFFF
:101A0800404211F0004F41F4000121F07F4118BF1E
:101A1800494292EA030F3FD0A2F1010241FA03FCC6
:101A280010EB0C00C3F1200301FA03F100F00043AE
:101A380002D5494260EB4000B0F5000F13D3B0F176
:101A4800807F06D340084FEA310102F10102FE2AE5
:101A580051D2B1F1004F40EBC25008BF20F0010055
:101A680040EA03007047490040EB000010F4000F03
:101A7800A2F10102EDD1B0FA80FCACF1080CB2EB96
:101A88000C0200FA0CF0AABF00EBC25052421843F5
:101A9800BCBFD0401843704792F0000F81F400019A
:101AA80006BF80F400000132013BB5E74FEA41036D
:101AB8007FEA226C18BF7FEA236C21D092EA030FD9
:101AC80004D092F0000F08BF0846704790EA010F53
:101AD8001CBF0020704712F07F4F04D1400028BF80
:101AE80040F00040704712F100723CBF00F5000062
:101AF800704700F0004343F0FE4040F40000704798
:101B08007FEA226216BF08467FEA23630146420243
:101B180006BF5FEA412390EA010F40F48000704756
:101B28004FF0000304E000BF10F0004348BF4042FC
:101B38005FEA000C08BF704743F0964301464FF038
:101B480000001CE050EA010208BF70474FF0000394
:101B58000AE000BF50EA010208BF704711F00043D5
:101B680002D5404261EB41015FEA010C02BF8446A5
:101B78000146002043F0B64308BFA3F18053A3F504
:101B88000003BCFA8CF2083AA3EBC25310DB01FA4B
:101B980002FC634400FA02FCC2F12002BCF1004FCF
:101BA80020FA02F243EB020008BF20F00100704760
:101BB80002F1200201FA02FCC2F1200250EA4C00B4
:101BC80021FA02F243EB020008BF20EADC707047FA
:101BD8004FF0FF0C1CEAD0521EBF1CEAD15392EA08
:101BE8000C0F93EA0C0F6FD01A4480EA010C4002E4
:101BF80018BF5FEA41211ED04FF0006343EA50103E
:101C080043EA5111A0FB01310CF00040B1F5000F7F
:101C18003EBF490041EAD3715B0040EA010062F12E
:101C28007F02FD2A1DD8B3F1004F40EBC25008BF18
:101C380020F00100704790F0000F0CF0004C08BF36
:101C480049024CEA502040EA51207F3AC2BFD2F103
:101C5800FF0340EAC250704740F400004FF0000311
:101C6800013A5DDC12F1190FDCBF00F0004070474B
:101C7800C2F10002410021FA02F1C2F1200200FA89
:101C880002FC5FEA310040F1000053EA4C0308BF50
:101C980020EADC70704792F0000F00F0004C02BFA1
:101CA800400010F4000F013AF9D040EA0C0093F01C
:101CB800000F01F0004C02BF490011F4000F013B76
:101CC800F9D041EA0C018FE70CEAD15392EA0C0FE4
:101CD80018BF93EA0C0F0AD030F0004C18BF31F04F
:101CE800004CD8D180EA010000F00040704790F025
:101CF800000F17BF90F0004F084691F0000F91F0C9
:101D0800004F14D092EA0C0F01D142020FD193EA8E
:101D18000C0F03D14B0218BF084608D180EA010016
:101D280000F0004040F0FE4040F40000704740F0F2
:101D3800FE4040F4400070474FF0FF0C1CEAD052C0
:101D48001EBF1CEAD15392EA0C0F93EA0C0F69D01C
:101D5800A2EB030280EA010C49024FEA402037D087
:101D68004FF0805343EA111143EA10130CF000407E
:101D78008B4238BF5B0042F17D024FF4000C8B426E
:101D880024BF5B1A40EA0C00B3EB510F24BFA3EB4E
:101D9800510340EA5C00B3EB910F24BFA3EB91031E
:101DA80040EA9C00B3EBD10F24BFA3EBD10340EA78
:101DB800DC001B0118BF5FEA1C1CE0D1FD2A3FF6BE
:101DC80050AF8B4240EBC25008BF20F00100704773
:101DD8000CF0004C4CEA50207F32C2BFD2F1FF0316
:101DE80040EAC250704740F400004FF00003013A47
:101DF80037E792F0000F00F0004C02BF400010F4EB
:101E0800000F013AF9D040EA0C0093F0000F01F0FE
:101E1800004C02BF490011F4000F013BF9D041EA20
:101E28000C0195E70CEAD15392EA0C0F08D1420253
:101E38007FF47DAF93EA0C0F7FF470AF084676E726
:101E480093EA0C0F04D14B023FF44CAF08466EE7FF
:101E580030F0004C18BF31F0004CCAD130F00042CD
:101E68007FF45CAF31F000437FF43CAF5FE700BF25
:101E78004FF0FF3C06E000BF4FF0010C02E000BF4E
:101E88004FF0010C4DF804CD4FEA40024FEA4103F0
:101E98007FEA226C18BF7FEA236C11D001B052EAA6
:101EA800530C18BF90EA010F58BFB2EB030088BF6C
:101EB800C81738BF6FEAE17018BF40F001007047DB
:101EC8007FEA226C02D15FEA402C05D17FEA236CBD
:101ED800E4D15FEA412CE1D05DF8040B704700BF04
:101EE800844608466146FFE70FB5FFF7C9FF00289B
:101EF80048BF10F1000F0FBD4DF808EDFFF7F4FFD4
:101F08000CBF012000205DF808FB00BF4DF808ED6C
:101F1800FFF7EAFF34BF012000205DF808FB00BF8F
:101F28004DF808EDFFF7E0FF94BF012000205DF8B1
:101F380008FB00BF4DF808EDFFF7D2FF94BF012062
:101F480000205DF808FB00BF4DF808EDFFF7C8FF5B
:101F580034BF012000205DF808FB00BF42000ED20C
:101F6800B2F1FE4F0BD34FF09E03B3EB126209D4CC
:101F78004FEA002343F0004323FA02F070474FF082
:101F88000000704712F1610F01D1420202D14FF0F7
:101F9800FF3070474FF00000704700BF00F026F890
:101FA8000C4880F30888002103E00B4B5B58435032
:101FB80004310A480A4B42189A42F6D3094A02E009
:101FC800002342F8043B084B9A42F9D318F0F4F97D
:101FD8007047000000C00020185A030800000020C5
:101FE8002813002028130020B86200207047FEE75D
:101FF80010B586B0002301244FF46022114801A9CE
:1020080001938DF80930039204938DF808408DF8F8
:10201800144023F0F7FA0B48214623F019FB09482E
:1020280023F020FB074823F022FB0028FAD10548BB
:1020380023F021FB034823F023FB0028FAD106B044
:1020480010BD00BF00240140014610B50D48012213
:10205800032323F023FB0B48012123F015FB7F20EA
:1020680024F052F90748022123F062FB0028F6D039
:102078000448022123F062FB0248BDE8104023F027
:1020880054BB00BF002401400C4A0C2303FB01236E
:1020980010B59C880CB9588010BD5B8803F11304F7
:1020A800844204DA142B07D9133B834204DC0C2343
:1020B80003FB012102238B8010BD00BFF42E0020FA
:1020C8000A4B10B500241C7021464FF4E0720848F2
:1020D800FEF760F9074B43F604501C70064B1C7062
:1020E8000FF01AFD054B187010BD00BFF415002045
:1020F800C01700200B1A0020881900208A19002018
:10210800074B1978013101F01F011970054B1A7836
:102118008A4203D1013202F01F021A70704700BFD1
:10212800881900200B1A002010B50E4A0E2303FB55
:1021380000200D4A014614780C4A03FB042300F1E1
:102148000C0251F8044B914243F8044BF9D10A8828
:1021580000211A800E22FEF71DF9BDE81040FFF796
:10216800CFBF00BFF815002088190020C017002035
:10217800084B1A5C002352FA03F111F0010FD8B290
:1021880002D00130C0B270470133082BF3D10120CF
:10219800704700BFD71A002000F07F0000F5745088
:1021A8002DE9F84309300C46154698460FF0B4FC63
:1021B80000284FD043F63C37002638460FF0ACFCD9
:1021C800C0B25FFA86F988B120280FD04FEA5900CB
:1021D80000F5364037300FF09FFCC0B208B1022836
:1021E80004D10123B340227813432370113743F6F7
:1021F800C43301369F42E0D14BF2DE400FF08CFC35
:10220800C0B280B120280ED02B784BF2CD4043F0DD
:1022180001032B700FF080FCC0B220B1202802D03F
:10222800012388F800304BF20F500FF075FCC0B254
:1022380080B120280ED02B784BF2CD4043F002031A
:102248002B700FF069FCC0B220B1202802D0012306
:1022580088F80030BDE8F883034610465A1E10B5CA
:10226800032A1CD8DFE802F00E0E0207114A527842
:1022780002F0100203E00F4A527802F00802D2B2CC
:1022880072B10BE00C4A927802F04002D2B23AB135
:102298000A4A127802F003029A4200D140B10022A1
:1022A8000748105C984203D00132052AF8D1002172
:1022B800084610BDC8600020F83A0020973F00206B
:1022C800B8170020F8B5064643F63C3500242846E2
:1022D8000FF022FCC0B2E7B268B120280BD0780812
:1022E80000F5364037300FF017FC012803D1A04025
:1022F80033781843307001341135082CE7D1F8BD14
:1023080003780E2202FB0313084AD3189978002396
:1023180051FA03F010F00100DAB202D0501CC0B23A
:1023280070470133082BF3D1704700BFC017002056
:102338002DE9F04101248C40284A29490346E4B29A
:10234800107891F800C019E0264F0E2606FB00769B
:10235800F178A9B996F80680B8F1000F10D196F86F
:102368000580B8F1000F0BD196F80480B8F1000F82
:1023780006D1F67926B9013000F01F00054626E09F
:10238800FBB1012B05D0022B06D10E2101FB0077F2
:1023980039790C4218D014E0042B04D10E2101FB2A
:1023A8000077B9790CE0032B04D10E2101FB0077EB
:1023B800797905E0052B07D10E2101FB0077F97922
:1023C80011B11570BDE8F081013000F01F006045C3
:1023D800BAD11570FF20BDE8F08100BF0B1A0020AC
:1023E80088190020C01700202DE9F043444D454BC3
:1023F8002A780E2101FB0232917A85B0044698466C
:1024080039B101390523594301F56E51443189B277
:1024180001E043F6C431204604220FF08EFB2B78EE
:102428000E2505FB038393F80B80364E344FB8F125
:10243800000F25D131232371073363713B7801A83D
:102448006B430422F15E06F04BFB3B7802A805FBC8
:1024580003630222997A06F043FB3B780DF10A00E8
:1024680005FB03650322697A06F03AFBA01D01A962
:102478000922FEF765FA4FF00F0984F8108012E080
:10248800B8F1010F0FD132232371053363713B7803
:102498004FF0080905FB036393F90130E3713B78BA
:1024A8005D43735BA371002320461A4612E010F8BF
:1024B800011BA1F13005EDB2092D04D8EB18302924
:1024C800DBB203D004E037395B1800E00A33DBB233
:1024D8000132D2B24A45EAD10F21B3FBF1F108012A
:1024E800411A5B1AC3F10F03DBB2092BA35401D8BD
:1024F800303300E03733A35405B0BDE8F08300BFA4
:10250800BE170020C0170020024B1A7842F00102C3
:102518001A707047911D002008B50C4B0C4A1B78A7
:102528000E2101FB0323D97A21B101290CBF09210E
:10253800002100E0102140221346064806F0F4F876
:10254800054B1A7842F002021A7008BDBE17002027
:10255800C01700208B190020911D0020034B1A780A
:1025680002F0F8026FF3C3021A707047911D002041
:10257800024B1A7842F004021A707047911D00202D
:10258800024B1A7842F008021A707047911D002019
:1025980038B5114B1C7814F0010502D1FFF7B4FFD0
:1025A80005E004F00405EDB21DB9FFF7E1FF284688
:1025B80038BD04F00805EDB215B9FFF7E1FFF6E7FD
:1025C80004F00204E4B21CB9FFF7A6FF204638BDA8
:1025D800FFF7C4FF012038BD911D0020014B18787A
:1025E800704700BFF415002030B51E4B85B01B782E
:1025F8000446002B34D11C4D2B78034113F0010FF6
:102608002ED01A4B1A4A1B780E2101FB0323DA78C5
:10261800024112F0010F1CD11B79034113F0010391
:1026280017D110F0010001F1F1014FEA540206D070
:1026380001320091019302926D20FE3905E00132CA
:102648000091019002923C20012103220B460FF0D9
:10265800E1FA012313FA04F42B7823EA04042C701A
:1026680005B030BD8A190020811900200B1A0020FE
:10267800C0170020037830B513F0010F144A4FF04B
:102688000E0419D104FB01210133012212FA03F3CC
:10269800CD7825EA0303CB7004780D79A41812FAD3
:1026A80004F425EA04040C7103789B189A408B788B
:1026B80023EA02028A7030BD04FB0121013B01229A
:1026C80012FA03F38A7822EA03038B7030BD00BF45
:1026D800C017002010B500230278590052FA01F4FF
:1026E80004F00304022C05D1013414FA01F122EAA2
:1026F800010202700133042BEED110BD2DE9F04F19
:1027080085B00192BDF838201C46744B0092DA78E7
:10271800054612F020028B4640F0D9808DF80E2035
:102728008DF80F208DF80D20DCB99B7803F040035D
:10273800DBB21BB101238DF80F3020E0684B5B78CA
:1027480003F00203DBB21BB101238DF80E3016E053
:102758000DF10F010DF10E020DF10D03FFF71CFD38
:102768000DE0012C0BD19B7803F04003DBB223B9B9
:102778000DF10F00FFF7A6FD01E08DF80F409DF861
:102788000F3023B99DF80E00002800F0A38044B94B
:1027980005F07F01490001F574510DF10A00663119
:1027A8000AE0012C0BD1E90101F51C4101F5B471D6
:1027B8000DF10A0001EB4B0102220FF0BEF9BDF941
:1027C8000A3013B9002C00F08480009B33B9454BC4
:1027D800454F93F80080FFF793FC08E0434B444FC4
:1027E80093F8008008F1010202F01F021A700DF13F
:1027F8000F00FFF76FFF002C44D1BDF80A3069B213
:1028080040F6B83212EA210238BF4FF47A72D21871
:102818000E2303FB08F3ADF80A20FA529DF80F9037
:10282800224649460120FE18FFF716FD4946F0707A
:1028380022460220FFF710FD86F8029030719DF8BD
:102848000E90224649460420FFF706FD4946B0711E
:10285800824622460320FFF7FFFC05F07F057071D2
:102868003572BAF1000F00D128B1224B1B7813B989
:102878009DF80D3000E00023F37186F809B0019A45
:10288800B2721CE0012C1AD10E2303FB08F3BDF829
:102898000A202046FA529DF80F6000223146FD18A2
:1028A800FFF7DAFC3146E87000220220FFF7D4FC7B
:1028B80000232871AE70AB716B71EB71AB720E2394
:1028C80003FB0877FC72009B0120BB8102E000201B
:1028D80000E0204605B0BDE8F08F00BFF83A0020C0
:1028E800C860002088190020C0170020F3150020B8
:1028F800F8150020761D002073B5154B04461B788B
:102908000E46D3B11348214622F023F80546A0B954
:10291800012E04F1010606D12046FFF729FC009597
:102928000246812005E02046FFF722FC009502467A
:10293800982031462B46FFF7E1FE2146054821F055
:10294800F2FF0548214602B0BDE8704021F0F6BF0D
:1029580089190020421C0020261A00202DE9F7437F
:102968007B4B04461B7843B17A4B1B7803F0240356
:10297800042B02D1002900F0E880774B774F1B78B1
:10298800002B00F0C7807648214621F0E2FF00289E
:1029980040F0C08007F5C470214621F0DAFF804678
:1029A800002840F0B7803B1993F880302D2B01D0D8
:1029B800532B3AD16B4E357845B30FF00DFC04F12B
:1029C8000108054650B12046FFF7D2FB337802468E
:1029D8001E33009393204146002307E02046FFF76B
:1029E800C7FB00950246414693202B46FFF786FE1B
:1029F8000FF0F2FB014628B1337803201E33009311
:102A0800002101E0009003200A4680E02046FFF7FD
:102A1800AFFB611C02462B4693200095FFF76EFE24
:102A28000095032029462A4671E0542B09D12046F7
:102A3800FFF79EFBCDF800800246611C94204346B8
:102A480066E0462B474D20D12E78BEB10FF0C4FB6F
:102A580004F10109064648B12046FFF789FB2B78A7
:102A680002461E3300939A20494622E02046FFF78B
:102A78007FFB0096024649469A2025E02046FFF74C
:102A880077FB009602469A2039E02E78002E2CD04B
:102A98000FF0A2FB04F11C09064660B12046FFF7BF
:102AA80067FB2B7802461E3369F07F000093C0B2A3
:102AB800611C434609E02046FFF75AFB024669F0CD
:102AC8007F000096C0B2611C3346FFF717FE0FF077
:102AD80083FB21B2024628B12B7803201E330093D2
:102AE800002214E00090032011E02046FFF740FB8D
:102AF800024604F11C0060F07F000096C0B2611C21
:102B08003346FFF7FBFD009603202146324601239A
:102B1800FFF7F4FD124821463F1921F004FF97F80A
:102B280080302D2B0AD0532B08D0542B06D0462B9F
:102B380004D00D48214621F00CFF30B10B48214646
:102B480003B0BDE8F04321F0F9BE03B0BDE8F0835F
:102B5800F6150020301C002089190020202D0020A7
:102B6800421C00209A1C0020A82E00203A1C00209D
:102B7800002302780E2101FB0232044901338A182E
:102B88000021062B9170F4D1704700BFC0170020B8
:102B9800064B00201870064B1A78064B1B789A4291
:102BA80002D00146FFF7C4BBFF207047F415002090
:102BB800881900200B1A00200121814038B5114BDB
:102BC800C9431A78104BC9B202F0030203F5E07446
:102BD800012A04D1DD7801EA0505DD7005E0022A45
:102BE80003D11D7901EA05051D710E33A342EFD10A
:102BF800FFF7FAFC43F604500EF08EFF034B1870F3
:102C080038BD00BF973F0020C01700208A19002058
:102C18002DE9F743A34D8DF807002B78A24C1BB183
:102C28002378C2B29A4204D043F604500EF074FFDF
:102C380028709DF8073023709C4C2278072A00F2F0
:102C48002D81DFE812F008002400360054005D00F2
:102C580072008D00BA00964A3C211170954A1946B7
:102C6800107800F00300FFF763FB934BFF28187000
:102C780000F0368120F06EFB904B002093F8742012
:102C880042F0010283F874208D4B187064E0884B81
:102C98001B78002B00F0248120F024FD012840F04F
:102CA8004D812378142201332370864B01381A7022
:102CB80047E17F4B1B78002B00F01281814E307862
:102CC80008B901234AE020F00DFD022804D020F0C5
:102CD80009FD032840F0328120F03CFB23780422D0
:102CE800013323701D233370774B1A7026E1704B24
:102CF8003C221A707548FFF777FB2378013323705D
:102D08006B4B1B78002B00F0EB806E4B1D78002D71
:102D180040F014811020FFF73BFC002800F01181DF
:102D280023782846013323700BE1614B1B78002B75
:102D380000F0D68005F062FD002800F00281614BAA
:102D48007D221A705E4B002018705C4B93F874203B
:102D580042F0010283F87420237801332370F0E0F5
:102D6800534B1B78002B00F0BB8020F0BBFC0128E4
:102D7800544E03D020F0B6FC03280FD19DF807204D
:102D8800012111FA02F2524B197821EA02021A7053
:102D980064233370237801332370CFE03078002820
:102DA80040F0CC80484A032323701378013BDBB200
:102DB8001370002B00F09480C3E0404A414E92F813
:102DC8006A201AB13278002A40F0B88000223270A6
:102DD800013212FA03F3DFF8E0803E4F98F8001052
:102DE8004FF00E0909FB0172DB4392F803E0DBB2F6
:102DF80003EA0E0E907882F803E092F804E003EA02
:102E08000E0E0340937082F804E00DF10700FFF7FF
:102E180031FC98F8003009FB0372D278DFF89490FF
:102E28002AB999F8002002F00302012A0AD00E22DA
:102E380002FB03721279B2B999F8002002F003027A
:102E4800022A10D10E2202FB0377BA785AB9224F10
:102E58003A789A4207D11848FFF78AFE3B7801333F
:102E680003F01F033B7099F800009DF8071000F06D
:102E78000300FFF75DFA144B0422FF281A7088F844
:102E88000000164B42D0987800F04000C0B20028ED
:102E98003CD1032323701A33337052E00020207092
:102EA8004FE000BF8A190020F7150020F415002014
:102EB80082190020973F0020BE1700201C3F0020E9
:102EC800F5150020F2150020801900208B1900202C
:102ED80081190020C01700200B1A0020F83A0020A2
:102EE800FFF73CFB0023237020F034FA2B78013BDA
:102EF800DBB22B702BB1144B9B7803F04003DBB291
:102F0800F3B19DF80700FFF757FE19E09B780E4ACA
:102F180003F04003DBB22BB1136843F400031360E2
:102F2800FFF7CEF8FFF71AFB20F014FA00232370FE
:102F380043F604500EF0F0FD287001E0002000E098
:102F4800FF20BDE8FE8300BFF83A0020044B1A7842
:102F58000AB1013A1A701B780BB9FFF72DBE7047FA
:102F68008A190020044A054B10781B7803EA501090
:102F780000F00100704700BFF83A0020091C00204B
:102F8800044B054A1B781078C3F3400303EA10107A
:102F9800704700BF091C0020F83A0020034B044A80
:102FA8001B78D078C3F3800318407047091C0020B1
:102FB800F83A0020044B054A1B78D078C3F3C003C5
:102FC80003EA5000704700BF091C0020F83A0020AF
:102FD800044B054A1B78D078C3F3001303EA90002A
:102FE800704700BF091C0020F83A0020044B1878ED
:102FF800044BDB785B005BB2DB1103EAD01070474F
:10300800091C0020F83A002008B50E2104481CF0DD
:10301800D1FB044B5B7803EA000000F0010008BD17
:10302800141A0020091C002070B500241BE030464B
:10303800E9B21CF0FDFB80B14FF4366363433422E0
:1030480002FB05330A4AD3181B7A13F0010F04D088
:10305800084B1878C0F3001070BD0135382DE6D143
:103068000134022C02D0E6B20025E0E7002070BD52
:1030780070400020091C002008B51BF0F5FC034B2C
:103088001B7800EA931000F0010008BD091C00201D
:10309800044B054A1B78D078C3F3401303EAD000E9
:1030A800704700BF091C0020F83A00202DE9F74FAF
:1030B800FFF758FF8246FFF763FF8346FFF76EFF6F
:1030C8000190FFF777FF8146FFF782FF0446FFF77D
:1030D800ABFF0546FFF7DCFF8046FFF7CDFF07464D
:1030E800FFF784FF0646FFF78FFF019B45EA0404BC
:1030F8009B0043EA4B0343EA0A0343EAC90343EA52
:10310800481343EA871343EAC61343EA0023E0B2AD
:1031180043EA0010BDE8FE8F044B987800F00F00DA
:10312800A0F10203584240EB03007047771A0020D1
:10313800044B987800F00F00A0F10102504240EBD8
:1031480002007047771A0020044B987800F00F00AF
:10315800A0F10301484240EB01007047771A0020B4
:10316800054B987800F00F00A0F1060CDCF1000088
:1031780040EB0C00704700BF771A0020514AF0B5A9
:1031880013781446012B29D003D3022B40F09880E2
:103198005EE04D484D4B047819786FF3C304047012
:1031A80001F0F80158786FF3C301197000F080013D
:1031B800C9B2002900F08480012111709C78062290
:1031C80004F00F04544302464148005D60F30602D0
:1031D8005A701A7861F302021A70F0BD3B494D78B3
:1031E8000B4625F07F00002838D00A7802F0080244
:1031F800D2B222B9344A117841F0080111709A7894
:1032080002F00F02012A04D12F4A117841F001017E
:10321800117015F07F0F53D119789E7801F00700CF
:10322800062206F00F0602FB0606294F5D78BE5DF2
:10323800013066F3060500F007005D7090FBF2F5BB
:1032480002FB150262F30201197002232370F0BD1C
:103258001E494D780B4625F07F0028B98B7860F31E
:1032680003038B701070F0BD174A11786FF3C30118
:103278001170997801F00F01012903D111786FF3CA
:103288000001117015F07F0F1AD119789E7801F09E
:103298000700062206F00F0602FB06060C4F5D78B3
:1032A800BE5D013066F3060500F007005D7090FB17
:1032B800F2F502FB150262F3020119700123237073
:1032C800F0BD00BFC61A0020251A0020771A00207A
:1032D800B063020810B51F4A1F4B92F9031009B1D9
:1032E800002231E008B1032119701978032930D878
:1032F800DFE801F00209192C1178002929D01548B6
:1033080081700121197092F90200124920B1134B02
:103318001A786FF3861217E0487808B9032213E089
:1033280088700221197092F902100A4889B90B4A6B
:10333800147861F386141470026861F30F22D1B215
:1033480061F31742026001221A7010BD002111605A
:10335800197010BD9C1C0020231A0020F43D002089
:1033680070B543F6EF23044643F6F020012A08BF60
:1033780018460D460EF0D0FB2678C0B20640164C13
:103388000CD001201CF01AFC43F6EE200EF0C4FB12
:10339800236860F307036FF30F2314E02B781842B8
:1033A80012D030461CF00AFC0C4B43F6EE201A886B
:1033B80066F34D321A800EF0AFFB2368C0B260F39B
:1033C800070360F30F23236094F9003013B1024B15
:1033D8000F22DA7070BD00BF9C1C0020301C00203A
:1033E80008B543F6FB200EF097FB014B187008BD9B
:1033F800241A0020014B1870704700BF131C0020CE
:10340800024B1A5C6FF303021A547047201B00200A
:1034180070B50C46C10001F5CE411B48BF310822EA
:103428000EF08BFB002518482946EEB221F091FAE0
:1034380008B9237823BB154B2278EB5C1A421FD1BD
:103448003046FFF7DDFFF6084BF2DF5030180EF07C
:1034580063FB05F00703C0B2184110F0010F0FD14C
:103468000B48294621F075FA50B12946084821F041
:1034780065FA074B06F5CC40CE30995D0EF042FB5D
:103488000135402DCFD170BD151C0020D71A002062
:103498007A1A002038B546F2167540242046FFF700
:1034A800AFFFA5F5CC43094AD63BD15C11F0100F0C
:1034B80006D06FF30411D154284600210EF022FBE8
:1034C8000134E4B20135E92CE8D138BD201B0020D5
:1034D8003F287FB5054607D800F5E24041300EF099
:1034E8001BFBC3B22BB930E19C4A1478002C00F0C6
:1034F80031819B4E725D02F00F014C1C04F00F04E9
:1035080064F303023F2D725533D8002C00F022815A
:1035180001339C4240F01B81924B5A1992F880204B
:10352800522A725D03D161F3030272550FE16FF302
:103538000302EC081B19725593F8902105F0070354
:1035480052FA03F313F0010F40F00381294686482D
:1035580021F0E9F9844B04F5CC40195DCE30012403
:103568000EF0D0FA2D190223009301940295182029
:103578009EE0002C00F0EE80784B1B7801339C42D3
:1035880040F0E580735D05F5CC406FF30303D6305A
:10359800012173550EF0B6FA735D43F010037355AD
:1035A800A5F14003DBB2072B07D8042200920133B0
:1035B8000232019202931920B3E0A5F14803DBB26D
:1035C800072B07D804220092013303320192029399
:1035D8001A2061E0A5F15003DBB2062B07D80422BC
:1035E800009201330332019202931B2054E0A5F1AB
:1035F8005703DBB2032B07D80422009201330332AE
:1036080001920293212047E0A5F15B03DBB2012B75
:1036180007D8042200920133023201920293222039
:103628007FE05D2D06D1042300930193043B0293B0
:10363800284684E05E2D07D10423009301330193CB
:10364800053B02935E207AE0A5F15F03DBB26F2BA6
:1036580009D8042200920133921801920293332070
:103668000121053A6DE005F13103DBB2072B07D8DC
:103678000422009201330332019202935F200BE08F
:1036880005F12903DBB2012B09D80422009201338A
:1036980003320192029360200121043A51E0DA2DAD
:1036A8000CD1042300930124043B0194029361206C
:1036B8002146032223460EF0ADFA4BE0D92D07D15F
:1036C80004230093023B0193023B0293622036E0FD
:1036D800DD2D08D1042300930322043B01920293B9
:1036E800632001212DE0DB2D06D104230093043B48
:1036F80001930293642022E0DC2D06D10423009379
:10370800043B01930293702019E005F12203DBB218
:10371800032B09D80422009201330232019202934A
:1037280068200121033A0CE01E35EDB2062D10D8B1
:103738000423009301350233019302956A20012185
:1037480003220B460EF066FA03E01C4602E0002452
:1037580000E00124204604B070BD00BF0000002036
:10376800201B0020202D00207A1A0020024B185C14
:10377800C0F30010704700BF201B0020F8B50822D6
:103788000E4600210746FCF705FE46F2BF750024E9
:103798003378234113F0010F08D029460648082240
:1037A8000EF0CBF93846044921F08BF8013408357E
:1037B800082CEDD1F8BD00BF1F1C0020024846F2BE
:1037C800CE6108220EF0B9B97A1A002070B5044605
:1037D80000F56A5044300EF09FF90B4D06462B78E1
:1037E80013F0010F02D1CC2021F0A0FE2B8843F06A
:1037F80001032B80054B1E55054B13F8242042F07E
:10380800010203F8242070BD301C0020571A002044
:10381800361A0020024B185C084100F0010070477E
:10382800D71A002070B505460024094BE0B2E61807
:10383800E35C4BB12946FFF7EDFF28B10023337055
:103848000448214621F07AF80134402CEDD170BDAE
:10385800521C0020671A002038B505460024284667
:10386800E1B2FFF7D7FF10B1044BE35C23B9013491
:10387800082CF4D1002038BD012038BD571A00208B
:1038880038B505460EF0A8FCA0B100242846E1B2E0
:10389800FFF7C0FF40B1084B13F8243013F0010FB5
:1038A80002D0064BE35C23B10134082CEED1002092
:1038B80038BD012038BD00BF361A0020571A002035
:1038C800F8B5114800214022FCF764FD46F2BF75A7
:1038D800002401270D4829460822A7400EF02DF99B
:1038E800FFB200260948314621F033F820B1064BD3
:1038F800F25C47EA0202F2540136402EF2D101345A
:103908000835082CE5D1F8BDD71A00201F1C002067
:103918002DE9FF4100263446B0461A4B1B78234157
:1039280013F00102184B23D0184F1D5D17F82430EF
:10393800A84538BFA84613F0010F1AD0CDB965F3D2
:10394800000307F8243023B20122F71902935B2001
:1039580029462B46009201950EF05CF97B78B878E1
:10396800F9781843621C2B460095FEF7C7FE00E065
:103978001A5501340436082CCFD1054B83F8008042
:10398800BDE8FF81241A0020571A0020361A0020AB
:10399800221A002010B50C4B1B78A3B10B4B1B78D7
:1039A8008BB100240A48214620F0D3FF40B10948D2
:1039B800214620F0CEFF18B920460121FEF7CEFFA0
:1039C8000134402CEED110BD89190020F6150020D5
:1039D8003A1C00201E2400202DE9F043324C334AC3
:1039E800238800266FF386136FF3C4032380304BBC
:1039F800304F85B016701E709146984617F8013BF7
:103A08005BB32278D20052B243EAA2122388402E36
:103A180062F3C40343F0400323801ED000253046E0
:103A2800E9B2FFF7F7FEA8B117F8013C13F0010F50
:103A380006D00122AA4099F800100A4389F800200C
:103A480013F0020F06D00123AB4098F8002013436F
:103A580088F800300135082DE1D10136F6B2412E43
:103A6800CCD1237803F04005EDB2D5B903F0240397
:103A7800042B0BD1FFF78EFFFF230093402029462C
:103A880001222B46019502950EF0C4F823880022E6
:103A98006FF345136FF382036FF3C4032380064B60
:103AA8001A7005B0BDE8F083301C0020483D0020A6
:103AB800783D0020851A0020141C002010B5002431
:103AC8000548214620F045FF08B9044BE05401346D
:103AD800402CF5D110BD00BF0B1C0020851A00201A
:103AE80010B5127804469DF80810DAB1D3B111B1B7
:103AF8000D4920F0DBFEACB1082246F2CE610B483E
:103B08000EF01BF82146094820F0DBFE0749082281
:103B180046F2CE600EF00BF805480449BDE81040A7
:103B280020F0E5BE10BD00BFB82E00200C1A002002
:103B38007A1A002030B5064B04781D7824EA05046B
:103B48000C7001781B7823EA0103137030BD00BFA5
:103B5800241A002038B50A4D002415F8013F2D2BF2
:103B680009D0532B07D0542B05D0462B03D005483A
:103B7800214620F0E3FE0134402CEED138BD00BFD1
:103B88009F2D00203A1C002010B50F4820F086FE1B
:103B980000240E48214620F0DCFE80B10C4BE318CF
:103BA80093F88030482B06D003D82D2B03D0462B12
:103BB80000E0542B03D10448214620F0B4FE013420
:103BC800402CE6D110BD00BFC71A00203A1C0020C7
:103BD800202D0020094A0A4B117831B1997801F05B
:103BE8000F01814201D0002111709A7860F303021D
:103BF8009A705A7842F080025A707047C61A0020AC
:103C0800771A00202DE9FF411E466C4BDDF828800D
:103C1800154604461A780F460023694911F82310FF
:103C280011F0010F03D00121994022EA010201336A
:103C3800082BF2D1634B1A70002C6FD014F0010FCF
:103C48000AD0FF2301210093FF3B019302935220E6
:103C58000A460B460DF0DEFF14F0020F0AD0FF23D0
:103C680001210093FF3B0193029353200A460B4620
:103C78000DF0D0FF14F0040F0AD0FF2301210093A8
:103C8800FF3B0193029354200A460B460DF0C2FFF6
:103C980014F0080F0AD0FF2301210093FF3B019382
:103CA800029355200A460B460DF0B4FF14F0100F8E
:103CB8000AD0FF2301210093FF3B01930293562072
:103CC8000A460B460DF0A6FF14F0200F0AD0FF237A
:103CD80001210093FF3B0193029357200A460B46AC
:103CE8000DF098FF14F0400F0AD0FF230121009334
:103CF800FF3B0193029358200A460B460DF08AFFBA
:103D080014F0800F0AD0FF2301210093FF3B019399
:103D1800029359200A460B460DF07CFFCFB10024D0
:103D28003046214620F015FE60B1FF230093FF3B8B
:103D38000193631C1BB2012102935A200A460B46C9
:103D48000DF068FF21463046013420F0F7FD402C85
:103D5800E6D1BDB100244046214620F0FAFD70B1FD
:103D6800012D0CD104230093DB180193631C1BB2B3
:103D780002937420294603222B460DF04BFF013491
:103D8800702CE8D10F481049104AFFF7D3FE104BAA
:103D980000221A700132009206320192F832029221
:103DA80009490A4A074809F013FF0A4B3C225120E7
:103DB8001A7004B0BDE8F0410EF0FABA241A0020D7
:103DC800361A0020FC1D0020E51E0020D81E002009
:103DD800C11D0020561A002037B5FFF767F90446C1
:103DE8000E4820F089FDD0F1010538BF00250C48A8
:103DF8000E211BF0DFFC10B114F4807F03D124B92D
:103E08005DB1224602E0012200E00022044B204678
:103E180000932946014BFFF7F5FE3EBD181B002015
:103E2800141A0020054B03EBD00393F8903100F0EF
:103E3800070053FA00F000F001007047202D002021
:103E480010B50F4B04461B7813F0010315D0FFF78C
:103E580003FD28B90B4B1B1993F88030462B0DD165
:103E68000EF0BAF918B92046FFF7DCFF30B1064862
:103E7800214620F058FD012010BD184610BD00BF96
:103E8800301C0020202D0020181B0020024B187821
:103E9800003818BF01207047561A002010B5034C8F
:103EA80004EB830358709970DA7010BD361A00203D
:103EB80010B500240948002100190E220E34FCF721
:103EC80069FAB4F5E07FF5D1054A00231370054A75
:103ED800002199520233AA2BF9D110BDF815002000
:103EE800F31500205A1F00207FB5474B04461B7866
:103EF8000E46AA2B78D04548214620F02AFD0546D3
:103F0800002871D12046FFF79BFF00286DD140485B
:103F1800214620F01EFD50B93E48214620F019FDEB
:103F2800054620B92046FFF7D3FA00285DD13A4B61
:103F38001B7823B9394B1B7813F0010F09D1384B83
:103F4800DB7803F02003DBB21BB9364B032283F87E
:103F58004020012E05D82E48214620F0FAFC40B119
:103F680042E0022E07D12B48214620F0F2FC10B186
:103F78003AE0274800E02748214620F0D4FC2A48A8
:103F8800214620F0DBFC022E15D10125294603220B
:103F98002B4600964A206619019502960DF03AFEC6
:103FA8002046FEF7E5F80023024631461820009324
:103FB800FEF7A4FB19E0012E09D102230093631C2C
:103FC80002930196122031460322334609E07EB956
:103FD8000121022300936318029301911120032207
:103FE8000B460DF017FE03E00025284604B070BD0F
:103FF8002046FEF7BDF80246012000232118009351
:104008000125FEF77BFBF0E7131C00207A1A00203D
:10401800261A0020921C0020241A0020551F002078
:10402800F83A0020851A0020421C00202DE9FF479D
:1040380004460D467548214620F08BFC8146002831
:1040480040F0DF802146714820F06DFC7048214621
:1040580020F074FC6F4E0DBB01274FF00208E319E6
:1040680002934246032039463B46CDF8008001972B
:104078000DF0D0FD327862B10EF0AEF8024630B1E4
:10408800337840461E33009321462A4604E00090C8
:1040980000E00092404621463B4628E0012D2BD106
:1040A8005D4B04F5E24041301F5D0DF035FD07F032
:1040B8000F07874209DA631C022202930E20294661
:1040C8002B46009201950DF0A5FD327892B10EF0C5
:1040D80083F8024638B14F4B0D201B7821461E331A
:1040E8000093002202E000900D2021460123FEF7F4
:1040F80005FB5EE00092F7E7022D0BD10123019347
:10410800E3180293142049462A464B4600950DF0C1
:1041180081FD4EE0032D4CD101272A464FF00208BD
:1041280004EB070A4D2039463B46CDF8008001973D
:10413800CDF808A00DF06EFD35783DB30EF04CF8C3
:10414800024630B1337840461E33009321464A4632
:1041580002E00090214640463B46FEF7CFFA0EF0BB
:104168003BF8671C054648B12046FEF701F833784E
:1041780002461E3300931A2039462CE02046FDF7EC
:10418800F7FF0095024639461A202DE021462A46B7
:104198003B4640460095FEF7B1FA2046FDF7E8FF9A
:1041A800514602462B461A200095FEF7A7FA3846D4
:1041B80028E03578EDB10EF00FF804F11C0605463D
:1041C80058B12046FDF7D4FF124B02461B78304603
:1041D8001E330093611C002307E02046FDF7C8FF4B
:1041E800009502463046611C2B46FEF787FA0120EF
:1041F80008E02046FDF7BCFF0095024604F11C00CC
:10420800F1E7002004B0BDE8F08700BF3A1C0020A9
:10421800421C00209A1C0020201B0020064B1B1863
:1042280093F84001492804D0452814BF03200220F0
:1042380070470120704700BF202D00202DE9F04174
:10424800244F00243C702448214620F082FBE5B22C
:10425800224B002837D01E5D3B789E4200D303B91D
:104268003E70002E30D131461C484022FCF792F8AF
:104278001B4B1C4803EBD50393F8888104F0070314
:1042880048FA03F8214608F0010820F062FB68B9F3
:10429800B8F1000F02D02846022101E02846314635
:1042A800FFF7C4FE28460EF083F80DE0B8F1000FC2
:1042B8000AD12846FFF7B2FF0B4BDB7803F0200347
:1042C800DBB20BB9094B18550134402CBBD1BDE802
:1042D800F08100BF9A1C0020671A0020521C0020A1
:1042E800202D00203A1C0020F83A0020851A0020D2
:1042F8002DE9F04F914B8BB01B7813F0010F06D0CE
:104308008F4B1A786FF386121A7001F012BB8D4921
:104318008D4A0B7810788D4D984218BF8C491370D0
:1043280018BF0B706B7803F00803DBB24BB143F690
:10433800CF200DF0F1FB864B18702B886FF3CB2341
:104348002B80844B1B78AA2B08D18349AA3B0B707E
:104358002B8843F080032B8000F028BF6A787B4BC2
:1043680002F01002D2B27D4CA2B11A886FF30C325F
:104378001A807B4B1B7823B97A4B1B7813F0010FFB
:1043880008D1E37803F02003DBB21BB9764B032294
:1043980083F840202368754F6FF3186323603A78D9
:1043A80002F00202D2B232B96B494A781AB16B4AAA
:1043B80043F080731360E67816F0010648D05D205C
:1043C800FFF7D4F900285AD16B78DFF8808103F021
:1043D8000203DBB22BBB5D30FFF77AF8064600BB61
:1043E800B8F80030012143F40073A8F80030042322
:1043F80003220093019302900B460D200DF00AFC56
:1044080045200DF0D5FF3146012233460D20009698
:10441800FEF774F909203146324601230096FEF76B
:104428006DF96B7803F00203DBB243B34C4B1B7896
:1044380023B94C4B1B7813F0010F20D1E37803F01C
:104448002003DBB2DBB9484B032283F8402016E097
:104458006B7803F00203DBB26BB1314632460123BD
:104468000A200096FEF74AF98D203146012233468C
:104478000096FEF743F92B886FF349232B802368B6
:10448800354A6FF35963236093787BB1D37823B9A6
:104498003B7813F00C0F05D108E03B7803F00C03D0
:1044A800042B03D0236843F000732360E17801F004
:1044B8000201C9B200295BD05E20FFF757F9002836
:1044C80065D16B78214F03F00403DBB2EBB95E30A2
:1044D800FEF7FEFF0646C0B93B88012143F480631E
:1044E8003B800423009301330322019302900B467F
:1044F80017200DF08FFB45200DF05AFF0D20314697
:10450800012233460096FEF7F9F86B7803F00403AE
:10451800DBB2002B3BD0124B1B7823B9114B1B7815
:1045280013F0010F33D1E37803F02003DBB273BB40
:104538000D4B032283F8402029E000BFFD1D002019
:10454800F43D00201D1C00201E1C0020301C0020F3
:104558009B1C0020131C002028130020F83A002080
:10456800241A0020551F0020851A00201E2D002027
:104578006B7803F00403DBB22BB18D2001220B46CC
:104588000091FEF7BBF82B886FF38A232B802368F2
:104598004FF05F0B6FF3DF732360002696E00698F9
:1045A800F9B21BF045F9002875D04FF43663734310
:1045B800342202FB0733A749A8F15E0ACB1803F19E
:1045C80008021B7A5FFA8AFA13F001034DD02368B8
:1045D800404643F0004323600592FFF7C7F8059A69
:1045E800002864D1937813F0040F20D14046FEF7D9
:1045F8006FFF059A8146D0B99378012143F00403EF
:10460800937004230093DB180322019332200B4696
:10461800CDF808A00DF0FEFA4A200DF0C9FE0C20D6
:10462800514601224B46CDF80090FEF767F84FF44B
:1046380036637343342202FB0733864AD3189B7AC6
:1046480013F0040F33D0844B1B7823B9834B1B78AA
:1046580013F0010F2BD1E37803F02003DBB233BB57
:104668007F4B032283F8402021E0927812F0040F58
:1046780005D08C20514601220093FEF73FF84FF4F5
:1046880036637343342202FB07337249CB189A7A94
:104698006FF382020AE04FF436637343342202FB5D
:1046A80007336C4AD3189A7A60F382029A720137F8
:1046B80008F10108382F5FFA88F87FF470AF0136E7
:1046C8000BF1380B022E5FFA8BFB04D0F3B2069382
:1046D800D846002763E72368624923F080636FF3B5
:1046E8009E7323600B79002B00F025845E4ADFF867
:1046F8007CB106924FF0CF0800271BF8011F3E46F9
:104708000137002952D0236808F1710A43F0806309
:104718005FFA8AFA23605046FFF728F800285CD130
:1047280018237343DFF8489119F8032012F0100F8B
:1047380023D150460593FEF7CBFE059B8246E0B990
:1047480019F80320012142F0100209F8032004237C
:104758000093023301933BB2032202930F200B46CE
:104768000DF058FA45200DF023FE0D205146012288
:104778005346CDF800A0FDF7C1FF1823734319F87D
:10478800033013F0100F28D0334B1B7823B9334B69
:104798001B7813F0010F20D1E37803F02003DBB27C
:1047A800DBB92F4B032283F8402016E0182373430C
:1047B800DFF8BC9019F8033013F0100F05D08D20E6
:1047C80001220B460091FDF799FF1823734319F84E
:1047D80003206FF3041209F80320069A12F8011F48
:1047E8000692002946D02368404643F08043236060
:1047F800FEF7BCFF002854D14FF0180909FB06F951
:10480800DFF86CA01AF8093013F0200F49D14046A0
:10481800FEF75EFE0646002843D11AF8093001214A
:1048280043F020030AF8093004230093033301936B
:104838003BB2032202934B200B460DF0EBF95020BC
:104848000DF0B6FD19203146012233460096FDF7DA
:1048580055FF26E070400020241A0020551F002034
:10486800851A0020281300204A3C0020763C0020AE
:10487800843C002018237343DFF8A89219F803300A
:1048880013F0200F05D0992001220B460091FDF767
:1048980035FF18235E4319F806306FF3451309F8FE
:1048A800063008F10108082F5FFA88F87FF425AF71
:1048B800974ADFF874B206924FF05008083F1BF889
:1048C800011F3E460137002952D02368A8F16E0A1D
:1048D80043F080635FFA8AFA23605046FEF746FF8A
:1048E80000285CD1DFF8449206EB061319F8032080
:1048F80012F0400F23D150460593FEF7E9FD059BC2
:104908008246E0B919F80320012142F0400209F873
:10491800032004230093023301933BB20322029342
:1049280069200B460DF076F945200DF041FD0D206C
:10493800514601225346CDF800A0FDF7DFFE06EBF5
:10494800061319F8033013F0400F28D0714B1B7869
:1049580023B9714B1B7813F0010F20D1E37803F0D2
:104968002003DBB2DBB96D4B032283F8402016E04D
:10497800DFF8B89106EB061319F8033013F0400F6F
:1049880005D08D2001220B460091FDF7B7FE06EBFE
:10499800061319F803206FF3861209F80320069A04
:1049A80012F8011F0692002933D02368404643F0CD
:1049B80080432360FEF7DAFE002841D1DFF86CA1BE
:1049C80006EB06191AF8093013F0200F38D14046C3
:1049D800FEF77EFD064698BB1AF80930012143F020
:1049E80020030AF8093004230093033301933BB2F0
:1049F8000322029310200B460DF00CF950200DF005
:104A0800D7FC19203146012233460096FDF776FE81
:104A180016E0DFF8189106EB061319F8033013F0C7
:104A2800200F05D0992001220B460091FDF766FE64
:104A380006EB061619F806306FF3451309F8063029
:104A480008F10108072F5FFA88F87FF438AF344A75
:104A5800DFF8DCB006924FF05708073F1BF8011F3C
:104A68003E460137002967D02368A8F1790A43F048
:104A780080635FFA8AFA23605046FEF777FE0028C3
:104A880071D1DFF8B09006EB061319F8032012F085
:104A9800400F23D150460593FEF71AFD059B824629
:104AA800E0B919F80320012142F0400209F8032077
:104AB80004230093023301933BB20322029367203D
:104AC8000B460DF0A7F845200DF072FC0D2051465D
:104AD80001225346CDF800A0FDF710FE06EB0613A1
:104AE80019F8033013F0400F3DD00A4B1B7823B957
:104AF800094B1B7813F0010F35D1E37803F020033D
:104B0800DBB283BB054B032283F840202BE000BFB8
:104B1800FB3A0020241A0020551F0020851A002087
:104B28003D3B0020843C0020313C0020BB3B002062
:104B3800313B0020593B0020DFF8B49306EB061305
:104B480019F8033013F0400F05D08D2001220B46D1
:104B58000091FDF7D3FD06EB061319F803206FF358
:104B6800861209F80320069A12F8011F06920029F6
:104B780033D02368404643F080432360FEF7F6FDB8
:104B8800002841D1DFF868A306EB06191AF80930A6
:104B980013F0200F38D14046FEF79AFC064698BB22
:104BA8001AF80930012143F020030AF809300423D8
:104BB8000093033301933BB2032202931F200B4659
:104BC8000DF028F850200DF0F3FB19203146012292
:104BD80033460096FDF792FD16E0DFF8149306EBD6
:104BE800061319F8033013F0200F05D0992001227D
:104BF8000B460091FDF782FD06EB061619F8063004
:104C08006FF3451309F8063008F10108042F5FFA1D
:104C180088F87FF423AF4FF000084FF05B094FF09E
:104C2800D70A4646AB4B08F10108F15CAA4F0029A8
:104C380049D02368484643F080632360FEF796FD19
:104C4800002852D113237343FA5C12F0200F22D1AB
:104C580048460593FEF73CFC059B8346D8B9FA5CA9
:104C6800012142F02002FA540423009302330193F5
:104C78000FFA88F30322029320200B460CF0CAFF98
:104C880045200DF095FB0D20594601225B46CDF8D5
:104C980000B0FDF733FD13237343FB5C13F0200FC3
:104CA80023D08E4B1B7823B98D4B1B7813F0010F43
:104CB8001BD1E37803F02003DBB2B3B9894B03229D
:104CC80083F8402011E013237343FB5C13F0200F9B
:104CD80005D08D2001220B460091FDF70FFD13230F
:104CE8007343FA5C6FF34512FA547F4BF15C002969
:104CF80033D02368504643F080432360FEF736FDE7
:104D080000283ED1132303FB06735A7812F0200FB4
:104D180037D150460593FEF7DBFB059B834680BBE6
:104D28005A78012142F020025A7004230093033379
:104D380001930FFA88F3032202934C200B460CF0E0
:104D480069FF50200DF034FB1920594601225B46BB
:104D5800CDF800B0FDF7D2FC13E0132303FB067374
:104D68005B7813F0200F05D0992001220B460091A3
:104D7800FDF7C4FC132303FB06735A786FF345123F
:104D88005A705A4B1322F35C002B43D002FB06F3F4
:104D980017F803B0CBF3801BBBF1000F22D143F609
:104DA800DE2005930CF0B8FE059BD8B1FA5C012112
:104DB80042F04002FA5404230093DB1801930FFADF
:104DC80088F3032202932F200B460CF023FF472081
:104DD8000DF0EEFA0920414601225B46CDF800B0FD
:104DE800FDF78CFC13237343FB5C13F0400F22D0B8
:104DF8003A4B1B7823B93A4B1B7813F0010F1AD1A1
:104E0800E37803F02003DBB2ABB9364B032283F817
:104E1800402010E07243BA5C12F0400F05D08920A0
:104E2800414601220093FDF769FC13237343FA5CA2
:104E38006FF38612FA5401360AF1010A09F10109E1
:104E4800022E5FFA8AFA5FFA89F97FF4EBAEDFF88F
:104E5800A4A04827023E1AF8011FB04601360029CF
:104E68004CD02368384643F080432360FEF77EFC2D
:104E780000285CD14FF01E0909FB08F9DFF878B06B
:104E88001BF8093013F0200F51D13846FEF720FBEC
:104E9800804600284BD11BF80930012143F020033C
:104EA8000BF80930042300930333019333B2032230
:104EB800029313200B460CF0ADFE50200DF078FA4B
:104EC8001920414601224346CDF80080FDF716FC23
:104ED8002DE000BF483C00200C3B0020241A002095
:104EE800551F0020851A0020393C0020433B002034
:104EF800593B0020B23B0020133E00201E2303FB39
:104F080008F3DFF8C09119F8033013F0200F05D02B
:104F1800992001220B460091FDF7F0FB1E2303FBAD
:104F280008F819F808306FF3451309F80830013705
:104F3800082EFFB28FD1A67806F00806F6B2002E2A
:104F480040F03481594A06925FFA86F8B8F1000FAA
:104F58000CBF4023702347F61B410993079149F67C
:104F68001E59002447464FF4E07A0AFB06FA4F4AD6
:104F78002146524410465FFA84F808921FF0E9FC73
:104F880048B94A480AF1700A504421461FF0E1FC2A
:104F9800002800F0F880454B4FF4E07A0AFB063A07
:104FA8000AF1E00A504621461FF0D3FC002840F0E1
:104FB800EA80504621461FF0B6FCDFF80CA10FB975
:104FC800484600E007980CF0A7FD8AF800009AF818
:104FD8000000DFF8F4B0002800F0D5800138C0B236
:104FE8008BF800000BF0A2FE002840F0CC809BF864
:104FF800000000F56A507C300CF08EFD2C49C0B2E0
:10500800087027B92B4B4B4413F85EAC03E0069AA3
:10501800131993F850A100EA0A0ABAF1000F00F038
:10502800B280089821461FF094FCDFF894B000B3D2
:105038001E4B4FF4E07000FB0630214670301FF025
:1050480088FCB0B91C49012F0B784AEA030A8BF88F
:1050580000A055D13823B8FBF3F203FB12834FF4B9
:1050680036614A43DBB2342101FB0323134AD318C8
:1050780040E00E4B4FF4E07000FB063021467030E4
:105088001FF067FC38B1089821461FF062FC10B980
:1050980009490B7804E0084A13781AEA030F15D077
:1050A80023EA0A0A8BF800A02AE000BF982900200A
:1050B800961E00202091FF1F241A00207040002017
:1050C800FC1D0020133E0020171B00204AEA030A9B
:1050D800012F8BF800A013D13823B8FBF3F203FBA0
:1050E80012834FF436614A43DBB2342101FB0323B8
:1050F8009C49CB1893F8302042F0200283F83020E6
:1051080099489A499A4AFEF715FD984B1B781BB1A6
:10511800FDF7CCFF002836D19448964912F0DCFE02
:1051280068B10DF059F870BB924808F0BDFD50BB4E
:105138000123904890498D4A0093FEF7D1FC002343
:1051480000938E4A01330193137887480293874965
:10515800874A894B08F03CFD012F14D13823B8FB4E
:10516800F3F203FB12884FF436635A435FFA88F868
:10517800342303FB08237B49CB1893F8312042F0F2
:10518800010283F831200134079A0999E3B2053204
:105198008B4209F101090792FFF4E5AE069A013640
:1051A80002F5E072022E06927FF4CEAE744E73784A
:1051B8006FF3C71373702B7803F08002D2B2002A02
:1051C80000F002816F490C78002C40F0FD8003F05C
:1051D8002403042B0BD1FEF7DDFBFF2300934020B3
:1051E800214601222346019402940CF013FD2B88DA
:1051F80000246FF3C7136FF3820364F3451364F35A
:10520800410364F30003604A64F3492364F38A2387
:1052180014702B805D4B1A7842F0C0021A705A78CD
:1052280064F3C3025A70FEF795FC59481FF036FB29
:1052380058481FF033FB58481FF030FB57482146A9
:105248004122FBF7A7F818236343554A0134D15C80
:10525800082C01F0DF016FF30411D154F3D10023BE
:10526800504903EB0312885C013300F0DF006FF351
:105278008610072B8854F3D14B4B1A786FF34512DD
:105288001A709A7F6FF345129A7793F83C206FF360
:10529800451283F83C2093F85A206FF3451283F89F
:1052A8005A2093F878206FF3451283F8782093F802
:1052B80096206FF3451283F8962093F8B4206FF385
:1052C800451283F8B42093F8D2206FF3451283F87F
:1052D800D220364B1A7802F0DF026FF386121A706A
:1052E8005A7C02F0DF026FF386125A7493F8222078
:1052F80002F0DF026FF3861283F8222093F833203E
:1053080002F0DF026FF3861283F83320284B5A78B5
:105318006FF345125A701A7802F0BF026FF3451204
:105328001A701A7D6FF345121A75DA7C02F0BF0203
:105338006FF34512DA74002311E04FF436615943D4
:10534800342000FB02111B48013209188878382ADA
:105358006FF382008870F0D10133022B2CD0002229
:10536800EBE700BF70400020FC1D0020E51E002078
:10537800D81E00202E1A0020C11D0020961E0020D5
:10538800771A002028130020141C0020F43D002068
:10539800921C0020261A0020671A0020851A002077
:1053A800843C0020BB3B0020133E0020593B0020DA
:1053B8000C3B002078400020082272480021FAF7B0
:1053C800E9FF714B00221A70704C2378002B48D1EA
:1053D80029786F4A01F00201C9B2D9B16D48118824
:1053E800477863F34D3163F3C30741F08001477099
:1053F8001180CA2020F09AF8C62020F097F820F0F3
:10540800E3F8654A13780BB90DF05EF8FEF742F839
:10541800FEF74EFD614A2B8811786FF341036FF355
:1054280000016FF3000311705D48002140222B80BA
:10543800FAF7B0FF5B481FF031FA5B481FF02EFA0D
:105448005A481FF02BFA5A481FF02CFA08224D48E8
:105458000021FAF79FFF4C4A00231370554A137036
:105468006AE02F7807F00203DBB293B917F001075F
:105478000FD14C481FF012FA2378F8B23B4113F0D1
:10548800010F03D0FEF7A2F90CF09CFE0137082F9C
:10549800F2D12B783E4F13F0010F25D0FEF79CFC7C
:1054A8003B8843F002033B80FEF732FA364B93F811
:1054B8000080B8F1000F14D1CA2020F037F8CD20B1
:1054C80020F034F83B883C4868F300033B80334BBA
:1054D8001A7842F001021A701FF0E0F9FDF7DAFFBE
:1054E80002E00120FEF776FB2B7803F00202D2B22D
:1054F80012B3304A12782AB113F0010F02D10220F8
:10550800FEF768FBFEF79AFE2C4927481FF0E4F9DE
:10551800254926481FF0CAF9FEF736FB22492848D4
:105528001FF0C4F9274926481FF0CBF9FEF7C6FA41
:105538001F481D491FF0DBF9204923481FF0B6F921
:1055480015490B780BB9FEF747FA737803F0800317
:10555800DBB2002B40D12B7803F02403042B06D1B7
:1055680043F6EC200CF0D8FA08B1062032E0FEF73A
:105578008DFC08B105202DE00DF090F830B3032024
:1055880028E000BF571A0020221A0020241A002001
:10559800301C0020F43D002028130020251A00208C
:1055A800521C0020653200200B1C0020671A0020C6
:1055B8004A1C00209A1C0020181B00207A1A002080
:1055C8003A1C0020C71A00205F1A002001F07EF85C
:1055D80010B10420FEF7FEFA694B1B781BB17378F3
:1055E8006FF3C7137370674A137813B1664B1B7850
:1055F800CBB12B78654E03F04403402B13D1002127
:10560800BF3300933F200B460222019102910CF018
:1056180001FB338843F6CE2043F0040333800CF0BB
:105628007BFA5B4B187057495A4E0B789BB1564B17
:10563800197881B92A78554B02F04002D2B252B19A
:105648001A8861F382021A80337823B943F6CE2090
:105658000CF062FA30702A78DFF8308102F004002A
:10566800C0B24D4B00287AD002F02000C0B2484F9B
:1056780090B11A78002042F0C0021A70FDF72AFE95
:105688003B78002B71D1B8F8002063F3820263F3F2
:105698004512A8F8002068E0D20052B21978921199
:1056A800D2B241F0C00112F0010F197003D0C9B293
:1056B80060F3C711197012F0020F03D01A786FF354
:1056C80086121A701B78344A03F04003DBB24BB9D8
:1056D800537843F00803537023781BB12B8843F4A5
:1056E80000532B800120FDF7F5FD43F6CD200CF08B
:1056F80013FAC0B20128307002D1264B02221A7068
:105708003C78002C31D1FEF745F9FF2301220093A4
:10571800402021462346019402940CF07BFA2B8802
:1057280043F6CD2043F020032B800CF0F5F9184BFD
:105738001A4A1870144B14701A780AB1013A1A7080
:10574800197891B90F4A13787BB1FF230093412050
:1057580002220B46019102910CF05CFA05E01A78DE
:1057680042F0C0021A70FDF7B5FD0CF047FF0C4877
:105778001FF0C2F80B4BB8B91A7860F3820216E032
:10578800AE5A00201D1C00209B1C0020301C00204D
:10579800141C0020841A0020F43D00202813002047
:1057A800CF1A0020251A00201A7842F004021A7035
:1057B8006A78614812F001011A780CBF61F341025E
:1057C80042F002021A705D491FF091F85C495A488C
:1057D8001FF077F858485B491FF073F83378012BAE
:1057E80040F0A7802B8800246FF349236FF38A23A6
:1057F8002B80554B21461C7041225448FAF7CAFDAC
:1058080053481FF04BF8FEF7A5F94D481FF046F82E
:105818004C481FF043F8182363434E4A0134D15CC7
:10582800082C01F0DF016FF30411D154F3D10023E8
:10583800494903EB0312885C013300F0DF006FF382
:105848008610072B8854F3D1444B1A786FF345120E
:105858001A709A7F6FF345129A7793F83C206FF38A
:10586800451283F83C2093F85A206FF3451283F8C9
:105878005A2093F878206FF3451283F8782093F82C
:1058880096206FF3451283F8962093F8B4206FF3AF
:10589800451283F8B42093F8D2206FF3451283F8A9
:1058A800D2202F4B1A7802F0DF026FF386121A709B
:1058B8005A7C02F0DF026FF386125A7493F82220A2
:1058C80002F0DF026FF3861283F8222093F8332068
:1058D80002F0DF026FF3861283F83320214B5A78E7
:1058E8006FF345125A701A7802F0BF026FF345122F
:1058F8001A701A7D6FF345121A75DA7C02F0BF022E
:105908006FF34512DA74002311E04FF436615943FE
:10591800342000FB02111448013209188878382A0B
:105928006FF382008870F0D10133022B01D000227E
:10593800EBE70BB0BDE8F08FEA3600203A1C0020F8
:10594800261A0020921C0020841A0020851A0020A4
:10595800671A0020843C0020BB3B0020133E002037
:10596800593B00200C3B0020784000202DE9FF41E6
:1059780004460D460CF06CFEA04B1A1992F8807084
:105988009F4A98461278AA2A0AD1A7F14F03DAB299
:105998000B2A00F2AD819B4A5BB29A4040F1A88184
:1059A800994B0C2202FB04335A7A0833AA42C0F0FE
:1059B8009F81FF2A00F09C81FF229A70934808EB90
:1059C800D403214693F888511EF0C3FF06460028E9
:1059D80040F08E8104F007031D41502F05F00105AA
:1059E80000F0268114D8462F00F0F28009D8412F04
:1059F80000F09E80452F00F01B812D2F40F076810E
:105A080034E0482F00F0C5804F2F40F06F810EE042
:105A1800542F67D006D8522F00F08A80532F40F0B9
:105A280065811CE0A7F15903012B00F25F817848DA
:105A380021461EF08EFF0646002840F059815A2F55
:105A480001D1744802E0592F04D1734821461EF051
:105A58006AFF54E121466F481EF065FFF5E76F487D
:105A680021461EF076FF002800F042816C4821464E
:105A78001EF06FFF8046002840F03A8121466848B2
:105A88001EF051FF674821461EF058FF02270126E5
:105A980055B1A419142041463A4643460097019649
:105AA80002940CF0B7F82AE129463A46334604F145
:105AB80001080A2000970196CDF808800CF0AAF892
:105AC8002046FCF755FB414602462B46132000951D
:105AD800FCF714FE384629462A4633460095FCF75B
:105AE8000DFE0CE14E4821461EF033FF0746002804
:105AF80040F005810126022231463346A5193E2091
:105B08000092019602950CF085F82046FCF730FBD0
:105B1800294602463B4614200097FCF7EFFD214634
:105B28003F481EF000FF21463E481EF007FFE6E012
:105B38003A4821461EF00DFF0646002800F0DF8097
:105B4800374821461EF005FF064628B92046FDF7CE
:105B5800BFFC002840F0D380002D40F08E80204606
:105B6800FEF76EF9002840F0C5802046FEF756FB88
:105B78002D4BDB7803F02003DBB20BB92B4B185508
:105B8800412F00F08880522F40F0B080204601213C
:105B980083E0234821461EF0DCFE28B92046FDF7A5
:105BA80097FC002840F0A480002D66D12046FEF71F
:105BB80047F9002840F09E801B4BDB7803F0200358
:105BC800DBB2002B67D1194B032283F8402062E037
:105BD800134821461EF0BDFE064628B92046FDF7AB
:105BE80077FC002840F08B802046FEF729F9002832
:105BF8007ED1002D41D1204603214EE0202D0020EA
:105C0800131C002000003080F42E00207A1A002097
:105C1800782A002098290020082A00200B1C002040
:105C28003A1C0020421C0020F83A0020851A002067
:105C3800354821461EF08DFE064600285FD02046D6
:105C4800FDF71EFE20B1214630481EF06CFE4FE0E5
:105C5800502F28D12E4B1B782BBB2046FDF7FCFD7F
:105C680008BB2C4821461EF074FE064620B9204683
:105C7800FDF72EFC002842D115B1204602210CE088
:105C88002046FEF7CBFA244BDB7803F02003DBB287
:105C98000BB9224B185520460021FEF7C7F9061EFE
:105CA80018BF01262BE02046FDF7D6FD0546F8B9BA
:105CB8001B4821461EF04DFE0646D8B92046FDF782
:105CC80007FC0746D8B9164821461EF02CFE154A8F
:105CD800135D8BB910494E7806F02006F6B26EB9FE
:105CE80008EB040393F80031135508E0012606E099
:105CF800002604E02E4602E03E4600E01E463046FE
:105D080004B0BDE8F08100BF0B1C0020181B002068
:105D18009A1C00203A1C0020F83A0020851A00201E
:105D2800671A0020521C0020032210B505490648B6
:105D3800FAF706FE054806490222BDE81040FAF7C0
:105D4800FFBD00BFF6260020040200200902002043
:105D5800F426002070B5844C237813F0010F0AD084
:105D68000CF042FA38B10020804902F093FE804BD3
:105D78008048197849E0804D2B78002B4AD00CF0E8
:105D880039FA002846D07D4B1B7873B97C4B5B7879
:105D980013F0010F09D00CF01FFA30B9237803F083
:105DA8002403042B01D10330BEE0764C207870B177
:105DB8000020754902F06EFE21780122734802F036
:105DC8008FFE00201021621C07F0BCFA02E0704927
:105DD80002F060FE6F4C684807F004FB2378002B44
:105DE80000F018810CF000FA002800F013816A49CD
:105DF8006A481022FAF7A4FD68485B21FAF748FBC5
:105E0800002800F00781217801308322BDE8704026
:105E180002F066BE624C237803F00503012B5DD1C6
:105E28000020604902F036FE202110225E48FAF771
:105E3800B1FA601D5D490322FAF72CFD40BBE01C56
:105E48005B490222FAF726FD30B95A48FAF7F2FC04
:105E58005849024654480BE0E01C57490222FAF719
:105E680019FD40B95548FAF7E5FC544902464E4831
:105E7800FAF766FD0EE0E01C51490222FAF70AFD26
:105E880030B95048FAF7D6FC4E4902464648EFE783
:105E9800FFF74AFF6278303AD3B2092B00F2BA8092
:105EA8003F4B9B78303BDBB2092B00F2B3800A21D1
:105EB80001FB0231C9B2002900F0AC80374BFF2248
:105EC8000C291A7740F2A68010295A7740F2A2804E
:105ED80013299A7740F29E80DA7770BD3A4C23787E
:105EE80003F00203DBB213B1002038498EE0234EE1
:105EF8003378EBB9224B5B7813F0010F18D00CF014
:105F08006BF9A8B932481EF0F7FC60B12268314B32
:105F180002EA03033BB918F0A7FD20B9E37803F0C0
:105F28004003DBB223B10020BDE870400AF0D6B9C7
:105F3800337863B90CF050F948B1274B1B7803F05C
:105F48000603042B03D02B780BB90120ECE7FDF7EF
:105F58009DFF10B10020214958E0214B1D78002DEC
:105F680042D0204952E000BF301C0020B9FA020894
:105F7800221A002000020020241A0020941E00206B
:105F8800551F0020DE1D0020CCCF0208050200208E
:105F98008ACF02089A1C0020ABCF0208F401002027
:105FA800F1260020D3D40208040200202457030855
:105FB8002857030836D502082B57030815D50208B9
:105FC8002E570308F4D40208F83A00202AE40208FD
:105FD800CF1A00203000000F251A00205CE20208CA
:105FE8002D130020EDCF02080B4802F002FD0A48ED
:105FF80002F0F6FC094802F0F3FC1DF029F9E378F9
:1060080003F02003DBB22BB105492846BDE87040F8
:1060180002F040BD70BD00BFE81E0020081E002031
:10602800E5CE0208054B1B78D8019B015BB2DB115A
:1060380040B243EAE070C0B2704700BF301C002095
:1060480070B50E4686B041000122054601F5E9719A
:1060580005A80BF072FD0021012E8DF815104FF0E8
:10606800FF0205F1010305D1009201910293092075
:10607800FB3A04E00092019102931E2004220B4691
:106088000BF0C8FD05A83D49FAF788FA50B105A8F4
:106098003B49FAF783FA28B105A83A49FAF77EFA94
:1060A800002867D105A83749FAF778FA364B04462D
:1060B800F8B95A78214642F010025A70FF2302229A
:1060C80000930190FE3B02903D200BF0A3FD4D2074
:1060D8000CF06EF9691C0122234612200094FCF78B
:1060E8000DFB12202146224601230094FCF706FBF3
:1060F80003E05A786FF304125A700024E0B2552175
:1061080015F092FE38B12846214616F02EF810B147
:10611800204616F019F80134112CEFD13EBB1B486C
:106128001B491C4AFDF706FD19481B4911F0D4FE0E
:1061380068B10CF051F850B9174807F0B5FD30B9FF
:10614800012315481549124A0093FDF7C9FC144B61
:106158000F491D700023009305330193114B0D4A1D
:106168001B780A4802930D4B07F032FD02E00E4BF4
:1061780000221A7005A806B070BD00BFB557030805
:1061880031570308C1590308F43D0020FC1D0020C5
:10619800E51E0020D81E00202E1A0020C11D002058
:1061A800033F0020961E0020561A002007B5410024
:1061B800012201A801F5E9710BF0BFFC002301A839
:1061C80004498DF80530FAF7E9F9D0F1010038BF34
:1061D80000200EBDB557030807B54100012201A8EC
:1061E80001F5E9710BF0A9FC002301A804498DF819
:1061F8000530FAF7D3F9D0F1010038BF00200EBD01
:106208007E59030870B5154B04461B1893F8805047
:10621800B1B1134821461EF09CFB88B911482146AC
:106228001EF081FBA5F15903DBB2012B0CD94F2DD0
:106238000AD0542D08D021460B481EF074FB07E005
:10624800084821461EF07AFB074821461EF076FBD7
:1062580004480649BDE870401EF028BB202D0020E8
:106268007A1A0020CF1A00206F1A00204A1C00203A
:10627800024B1878C0F38000704700BF251A002031
:10628800024B1A8860F308221A807047301C0020DD
:10629800034B5878C00140B2C011C0B2704700BF6C
:1062A800301C0020014B1878704700BF241A0020CA
:1062B80030B5457800230021C218917055FA03F1D2
:1062C80011F0010F08D0064959188C7C017804EAAE
:1062D8000101A14208BF91700133042BEBD130BDFD
:1062E800DE1D002046F6A93104220BF026BC000072
:1062F80070B5104C0546112220460021FAF74AF8DD
:10630800002004F8010C2A78103414F8011FC3B2D5
:1063180091420BD152B10849013301F8013B1122D6
:1063280046F6F953BDE8704002F000BB013004287E
:10633800EBD170BDDF1D0020DE1D00201FB520B190
:10634800134B1A8842F480521A80124B00245A7850
:10635800214642F010025A70FF23022200933D208A
:10636800FE3B019402940BF055FC4D200CF020F8F4
:1063780040210122234612200094FCF7BFF9122085
:106388002146224601230094FCF7B8F91FBD00BF3F
:10639800301C0020F43D00202DE9F3412D4C07224C
:1063A800E37849F6B44702FB003349F6D540DBB23F
:1063B80018180BF0B1FB257964795FFA80F800268C
:1063C80048FA06F313F0010F3AD03946042201A81F
:1063D8000BF0B3FB9DF804009DF805309DF80610FE
:1063E8009DF8072000282BD0002929D0002B27D082
:1063F800002A25D0934204D19C4221D185421FD343
:106408000FE09A4210D99C421AD3944218D89C4261
:1064180001D994421AD39C4201D1854216D29442A2
:106428000ED18D420CD811E09C4201D185420DD28B
:10643800944201D18D4209D99C4207D8944205D390
:1064480001360437082EBBD1002000E00120BDE84A
:10645800FC8100BF1C58002010B5044649F60D50B9
:1064680000EBD4000BF058FB04F00704C0B2204145
:1064780000F0010010BD70B5C30849F60D555D194F
:10648800044628460E460BF047FB04F00704C0B24A
:10649800012126B9A14040EA0101C9B202E0A140A8
:1064A80020EA01012846BDE870400BF02BBB000034
:1064B800F0B57E4B95B0DD78082200EBC505EDB24E
:1064C800E90001F5084104A801F59E710BF035FBC0
:1064D800774B784E1A78002304A9C95C312905D175
:1064E8003039994041EA0202D2B205E0302903D19D
:1064F8002F39994022EA01020133082BECD132707E
:106508006C486D496D4AFDF715FB6B4B1B7813B949
:106518006A4B1B78F3B16848694911F0DDFC68B132
:106528000BF05AFE50B9664807F0BEFB30B901239C
:1065380063486449604A0093FDF7D2FA0023009348
:1065480002330193FD3302935A485B495B4A5D4B22
:1065580007F03EFB05EB0511002401F50A413470F4
:1065680004A8FC3111220BF0E8FA2646E0B25421C7
:1065780015F05AFC002838D004AB1B5D312B03D131
:10658800204615F0E7FC38B104AB1B5D302B2CD14D
:10659800204615F0DFFC40B34EB9FF2300933420AA
:1065A800314604223346019602960BF033FB04AEC3
:1065B800305D2146303815F0DBFC335D0126312B88
:1065C8004FF0030306D10093A3191BB2019602935F
:1065D800352005E00093631C1BB201960293362018
:1065E800002104220B460BF015FB0134112CBDD100
:1065F800A90101F50E4104A8B43140220BF09DFA1F
:10660800113C04AD274615F8013BE6B20134302BA6
:1066180003D13046FFF720FF38B115F8013C312B84
:106628002CD13046FFF718FF40B34FB9FF23009332
:106638003420394604223B46019702970BF0EAFAC8
:1066480015F8011C30463039C9B2FFF714FF15F8A8
:10665800013C0021302B4FF0FF0305D1009323B2FA
:1066680001910293372004E0009323B20191029331
:10667800382004220B460BF0CDFA0127402CC2D15A
:10668800114D6B7803F00403DBB263B1403C204644
:10669800FFF7E2FE38B90134E4B2402CF7D16B7849
:1066A80060F382036B7015B0F0BD00BF1C5800206A
:1066B800241A0020FC1D0020E51E0020D81E002002
:1066C8002E1A0020C11D0020F43D0020014B18782F
:1066D800704700BF2D1300202DE9F04F4E4B0022CC
:1066E8001A704E4A85B01678002E40F091804C4BB7
:1066F8004FF4B468DA78997808FB02F24FF03C0856
:1067080008FB01285A78474F90441FFA88F8BA4680
:106718006CE03AF815303C24DAB2544304EB132405
:106728004C44A4B2042CEEB207D842F25A739845EE
:1067380003D904F51C546034A4B2444511D949F670
:10674800D4400BF0E9F9C8EB0403834209DC364B6B
:106758001A787B1993F87030934302D02E4901239D
:106768000B702F4AD378B34232D142F26073B4FB34
:10677800F3F203FB12439BB2434523D12B4B9B7887
:1067880013F0090F44D12A4B5B7803F08003DBB286
:10679800002B3DD1274B5B7803F00203DBB2002BC3
:1067A80036D1254B1A781BEA020F11D101990098AE
:1067B80041EA02021A70FFF7EFFD48B90098FFF7A7
:1067C80077FE05E01C4B02991A7801EA02021A705A
:1067D800013509F5B469072D1FFA89F999D1039E86
:1067E80007370136082E0AF10E0A11D04FF0010BB7
:1067F8000BFA06FB5FFA8BF301936FEA0B03F2B215
:10680800DBB24FF00009009202934D46039680E7F1
:1068180005B0BDE8F08F00BF2D130020A11C00209B
:106828001C580020A21C0020241A0020F83A00203E
:10683800033E0020E2340020A01C002073B50C4663
:1068480001EBC001C9B2C90001F50841054608229B
:10685800684601F59E710BF070F9104B002003EBB0
:10686800C402121B521982F870001DF80020312A48
:106878000AD10121814003EBC402121B521992F87C
:106888007060314382F8701001300828EDD16946F4
:10689800312230231EF065F8C0B27CBDA21C002056
:1068A80000B501EBC001C9B2890191B001F50E41F3
:1068B800B431402268460BF040F940206946312245
:1068C80030231EF04EF8C0B211B000BD7FB501EB09
:1068D800C001C9B201EB011101F50A41FC311122D5
:1068E80001A80BF02AF9112001A9312230231EF04A
:1068F80038F8C0B207B000BD2DE9F8430026344689
:106908002BE021462846FFF799FF21468146284675
:10691800FFF7C6FF214640EA09092846FFF7D6FFD8
:106928005FFA89F949EA000010F0FF0F05D04046E8
:10693800394602220BF001F903E04FF0FF33A8F8C3
:1069480000300135EDB20237072D08F10208D8D121
:106958000134E4B20E3E082C07D0054BC6F50847B3
:10696800C6EB0308CC370025CBE7BDE8F88300BFAA
:10697800A21C002010B51FF05BF84FF480301FF008
:1069880077F81FF08FF90128044628D110201EF04F
:1069980071FF02201EF062FF00201FF0A9F80020FE
:1069A8001FF0BAF84FF480601FF0ACF84FF4404085
:1069B8001FF0BCF84FF480304FF4E0111FF074F86A
:1069C80020461FF07DF839201FF058F90028FAD02A
:1069D80002201FF07BF81FF083F80828FBD17C20E9
:1069E80001211FF015F946F6012001211FF010F9C9
:1069F8000C4801211FF018F90B4801211FF014F968
:106A0800042001211FF010F97E201FF037F938B15A
:106A18001FF05EF9054B04211A7861F344021A70DD
:106A280010BD00BF0340060020080818915A002036
:106A380010B50C46014620B110220C48F9F780FF2A
:106A480004E00A4820211022F9F7A4FC34B10848D0
:106A580021461022BDE81040F9F772BF04482021F2
:106A68001022BDE81040F9F795BC00BFF4010020E2
:106A78000402002010B5FF2B1446029A03D04218D6
:106A880002F8013C08E06FF07F439A4204D01314E7
:106A9800437013128370C2701BF0CAFA02E07F20A1
:106AA8001FF032FC1BF0B0FA0028F8D1ACB10B484B
:106AB80090F82010163001F00F011BF0B9FA02E02F
:106AC8007F201FF021FC1BF09FFA0028F8D1044B0F
:106AD80093F8693013F0010FE9D110BD580C00206C
:106AE800AC59002010B50A4B002203EBC003013B50
:106AF8001046084951184C7813F8011F8C4205D1EB
:106B08000130C0B20C320828F3D1F73010BD00BFF5
:106B1800DA630208F42E002070B50D4C05460E46C7
:106B28004FF4007200212046F9F734FC2A4631461A
:106B380004F50070F9F786FB642024F8035C1CF068
:106B480059FE0023A4F82D33024B64221A6070BD4D
:106B5800155B0020FC26002010B5054C00212046BE
:106B68004FF40072F9F716FC0023A4F82D3310BD7A
:106B7800155B0020164B2DE9F0415D8A0746284633
:106B8800FAF7CEFF1349FBF7D7F8134B134E1860EB
:106B9800D723B5FBF3F5EDB2822229460446F01956
:106BA80001F09EFF2846FAF7BFFF01462046FAF794
:106BB80005FF0B49FBF70CF8FBF7D0F90337BE19B3
:106BC800C1B281223046BDE8F04101F089BF00BF63
:106BD80030320020000057434C1D0020F4010020F3
:106BE800000020410000000070B54B4D2868FAF7FE
:106BF800A3FB45A3D3E90023FAF73EFAFAF78AFE86
:106C0800FAF79AFB42A3D3E90023FAF7E9FB3EA37C
:106C1800D3E90023FAF70EFDFAF77CFEFAF78CFBAE
:106C2800FAF796F9FAF776FE3C4906462860FBF72C
:106C380077F920B13046FBF791F9C4B25EE03046EF
:106C48003649FBF781F950B130463549FBF768F909
:106C580028B13046FBF782F9C0B2441C4EE03046FA
:106C68002F49FBF771F950B130462E49FBF758F917
:106C780028B13046FBF772F9C0B2841C3EE03046BA
:106C88002849FBF761F950B130462749FBF748F925
:106C980028B13046FBF762F9C0B2C41C2EE030467A
:106CA8002149FBF751F950B130462049FBF738F933
:106CB80028B13046FBF752F9C0B2041D1EE0304639
:106CC8001A49FBF741F950B130461949FBF728F941
:106CD80028B13046FBF742F9C0B2441D0EE03046F9
:106CE8001349FBF731F948B130461249FBF718F957
:106CF80020B13046FBF732F9C0B2841D0A20214684
:106D0800BDE870400AF0FEBE736891ED7CFF7F40DD
:106D18000000000080842E41501D0020000010411A
:106D28000000F0410000484200008E420000B842D6
:106D38000000E0420000F2422DE9F04F9DB01BF048
:106D48000DF909201CF0F2FE1CF0D8FC4FF461404C
:106D58001CF028FF09201CF0A5FF0022A3484FF4CF
:106D680080411EF0ECFDA24800211FF0B5F9A149B1
:106D780004224B78DFF8A0E26FF300034B709E4BC0
:106D88009E4C1A705A715A709A70DA701A719A7108
:106D9800DA719B4B033A1A709A4B00201F328EF817
:106DA800000020705A7105900546069006467F201F
:106DB8001FF0AAFA23780E2B01F2B681DFE813F050
:106DC8000F004F009500E0007902DE0330048504CF
:106DD800EA06DC07EF075808B108D00882098A4E8E
:106DE8008A48317801F00F01013149014118FFF754
:106DF8001FFE337813F00F0308D1854A92F8012358
:106E0800012A41F09181834A138024E0012B03D1A8
:106E18007F4B93F819330BE0022B04D17C4B93F88A
:106E28000D33032B05E0032B06D1794B93F80D3373
:106E3800012B41F079810EE0774901220A707748E9
:106E48004FF400711EF07BFD754BC8221A60337831
:106E58006FF30303BFE333785A1C01F05FB8704B3C
:106E68001A6822B96D484FF400711EF068FDDFF80A
:106E780098816C4898F8001001F00F010131490120
:106E88004118FFF7D5FD36B198F800305A1C62F367
:106E9800030388F800305F4B00221A8098F800102E
:106EA80001F00F02022A03D11A7842F010020AE018
:106EB800042A03D11A7842F0040204E0052A05D115
:106EC8001A7842F040021A7001F02EB9062A04D14D
:106ED8004D4B6FF3030119707EE301F00F0101229E
:106EE80012FA01F1198001F01FB9474E4E48317866
:106EF80001F00F01013149014118FFF799FD96F89A
:106F0800008008F00F08B8F1070F27DC18F0010F10
:106F1800464B02D00020588002E04FF0FF315980E4
:106F28004FEA6809062209F1010902FB09394FF005
:106F3800FF32A9F802204046FFF7D4FDFF2806D00B
:106F48003B4B03EB40005823437401F0EDB800239A
:106F5800A9F8023008F1010801F08AB800211022CE
:106F680013A8F9F717FA0FA800211022F9F712FA57
:106F780023780133237033786FF3030301F07BB870
:106F8800DFF884A09AF8008018F00F0840F03F81DD
:106F9800284E337803F04003DBB2F3B926486FF08C
:106FA8007F43817A0122009301F00F01FF23FFF74D
:106FB80061FD224B93F8692012F0400F08D093F836
:106FC8006C3013F0040F03D0337843F04003337070
:106FD8007378142262F3C7037370737813F0F80F91
:106FE80030D0174800F12001A7E300BF0018014086
:106FF800002C014052320020202D0020561D002078
:107008002B130020843C0020551D00201A64020820
:10701800F42E0020F43D00202C270020000C014015
:10702800FC260020BA6402089A6502087A3D00200E
:10703800F4010020E33A0020580C0020AC5900204D
:10704800BA660208BC4B1B7803F04003DBB2002B86
:1070580000F0D980DFF80483DFF8049398F8003053
:1070680013F00C0B30D1B54E6FF07F4396F82B1010
:1070780006F12100009301F00F0101220523FFF71B
:10708800F9FC96F84C104FF4860A06F1420001F01C
:107098000F010122FF23CDF800A0FFF7EBFC96F8C3
:1070A8004110FF2306F1370001F00F015A46CDF8D1
:1070B80000A0FFF7DFFC042389F8003098F80030BF
:1070C80043F0080301F02EB803F00803DBB2002BED
:1070D80039D099F800A0BAF1000F03D0984800F110
:1070E800400138E0954E6FF07F4B717D06F10B0043
:1070F80001F00F010122FF23CDF800B0FFF7BAFC21
:1071080096F82B1006F1210001F00F010122072348
:10711800CDF800B0FFF7AEFC96F836104FF48603B2
:10712800009306F12C00FF2301F00F015246FFF7F0
:10713800A1FC98F800306AF3C303DBB243F0040300
:1071480088F800305AE099F800C0BCF1000F08D068
:107158007B4800F16001FFF76BFC99F800203032A2
:1071680008E2764E6FF07F40717DFF23009001F0BA
:107178000F0106F10B000122CDF80CC0FFF77AFCD5
:107188009AF80030DFF8C4B103F0100A5FFA8AFAFF
:10719800DDF80CC0BAF1000F0CD098F800206CF3A1
:1071A800820288F800205A1C62F303038BF800302F
:1071B80000F0BABF96F82B106FF07F42009206F1EC
:1071C800210001F00F0101220C23FFF753FC96F870
:1071D80036104FF4860300935246FF2306F12C0025
:1071E80001F00F01FFF746FC9BF8003083F0100216
:1071F800C2F3001262F304138BF80030042389F8F9
:10720800003000F091BF4E4800F1800195E2B8F1DE
:10721800010F3CD14A4800F1A001FFF709FC002EFC
:1072280000F082879AF80030444E5A1C62F3030338
:107238008AF8003096F82B106FF07F4906F121008C
:1072480042460F2301F00F01CDF80090FFF712FC22
:1072580096F82B1006F1210042460E2301F00F018B
:10726800CDF80090FFF706FC96F82B1006F12100E8
:10727800424601F00F010F23CDF80090FFF7FAFB0B
:107288003048802142461EF05AFB00F04DBF2C4882
:1072980000F1C001FFF7CCFB002E00F045872A4B18
:1072A80096221A609AF800306FF303038AF80030C8
:1072B80092E1264E317811F00F0A16D1244800F1D8
:1072C8002001FFF7B5FB204B1B68002B40F02C87F3
:1072D80013A8F9F7AFFA40221346014613A801F0A4
:1072E80023FA3378012200F019BEBAF1010F39D11F
:1072F80012486FF07F4390F8201000220093163058
:1073080001F00F01FF23FFF7B5FB01F077FA002822
:1073180000F00A873378022262F3030333700D4BBF
:107328001A7842F080021A700B4B5A7842F0020227
:107338005A7000F0F9BE00BFE33A0020580C002054
:10734800BA66020800100140FC260020551D0020E6
:107358009A670208E83A0020923F00203061002036
:10736800B762002001F00F0101F10E0303F00F03D3
:10737800012B44D89B4849014118FFF759FB9A480B
:107388006FF07F4390F8201000221630009301F030
:107398000F01FF23FFF76EFB1BF0F8FF337803F0B4
:1073A8000F03022B13D117F02BFB002800F0BC862B
:1073B8008E4B1A7842F040026FF304121A705A7812
:1073C8006FF345125A703378032200F0A7BD17F007
:1073D80001FB78B117F0A0FB17F058FA844B002096
:1073E8001A7858816FF3C7121A703378042262F33F
:1073F800030333707F4B1A786FF3000263E5BAF129
:10740800040F4DD1DFF8DC914901DFF810824944BF
:107418004846FFF70DFB98F80010774B01F004027F
:10742800D2B27AB941F004016F4883F800A088F815
:10743800001090F836104FF4860300932C3001F0BA
:107448000F01EEE293F800A0BAF1000F40F06C864D
:1074580065486FF07F45417D01220B3001F00F0137
:10746800FF230095FFF706FB64480122817AFF237A
:1074780001F00F010095FFF7FDFA98F8003005229A
:107488006AF3820388F800303378484662F30303CE
:10749800337009F1A001FFF7CBFA554600F044BE5E
:1074A800DFF84481FF2398F8201000226FF07F490D
:1074B80008F1160001F00F01CDF80090FFF7DAFA95
:1074C8002BB2072B18D1337808F121006FF303038F
:1074D8003370237801220133237098F82B100E2380
:1074E80001F00F01CDF80090FFF7C4FA444880215D
:1074F80000221EF024FA0025424E96F86B3013F055
:10750800040F00F0118698F857106FF07F4300229F
:1075180000933D48FF2301F00F01FFF7ABFA96F8FF
:107528006B303A4A03F00F03012B137003D1002D7F
:1075380008BF01250CE0022B04D12BB2012B08BF98
:10754800032505E0032B03D12BB2032B08BF072526
:10755800ABB213F0010F02D02D4A3121517713F04D
:10756800020F02D02A4A3221917713F0040F00F05B
:10757800DB853322264BDA7700F0D6BD1948254E35
:1075880000F1C001FFF754FA96F80090DFF85C802C
:1075980019F00F090CD117F093F898F8003069F337
:1075A800000388F8003033785A1C62F30303337001
:1075B80017F018F998F8003013F0010F00F0B485AF
:1075C8000022154880211EF0BAF90A4B00225A7091
:1075D800337862F30303337023780133237000F0A8
:1075E800A3BD00BF9A670208580C0020923F0020F4
:1075F800E83A00200A3F0020B7620020010000207E
:1076080000100140AC590020A50C0020E23A0020EF
:10761800F4010020551D00200018014030610020B1
:107628008648874E00F1E001FFF702FA0FA8F9F744
:1076380001F90FA902468348F9F782F90021824827
:10764800B18090F8C5106FF07F4300220093BB30E3
:10765800FF2301F00F01FFF70DFA7C4A92F86B1037
:1076680092F86C30327843EA012312F0010FB380AC
:1076780010D0A3F1EB0292B20A2A04D9A3F5E6735B
:107688009BB2282B02D8F3880133F38033786FF349
:10769800000333707378002B40F04685684AD2881F
:1076A8007AB16B4A1BA8117863F303011170227831
:1076B8008DF86F300132227028228DF86C201EF070
:1076C8005DF90022F28000F02FBD624EDFF8ACA118
:1076D800337803F004085FFA88F8B8F1000F15D181
:1076E80009A841461522F8F755FE5B4BCAF80080F9
:1076F8001B684546CDF827303368474643F00403F6
:107708003360564BA3F8368300F00EBD03F08003B8
:10771800DBB2002B67D1DAF80010002940F00485AD
:107728004F48FFF785F94F484FF480511EF0FDF898
:10773800012806D04A4800F1A001FFF779F900F0C6
:10774800F3BC4649B1F83623002A43D009314648EC
:10775800013AF9F7F5F8444B03F1100113F8012B3E
:107768000D2A01D00A2A02D1202203F8012C8B42CB
:10777800F4D13E4B4FF03C0808FB073808F11E08CF
:107788004046F9F757F8414602463948F9F782F872
:10779800D8B9022F03D1336843F0100304E0032F54
:1077A80003D1336843F040033360327853005BB24F
:1077B80003EAC263DB173268DBB263F3C7123260D5
:1077C8001BB1FFF7C9F900F0AFBC0137FFB2042FB6
:1077D80008BF0227254B3C2606FB07363046F9F73B
:1077E80029F8314626E0DAF80080B8F1000F40F0B9
:1077F8009B84737803F02002D2B2002A40D11D4B3B
:1078080009A81A889B781C498DF82630ADF82420E1
:10781800F8F71AFE114B5B7A302B07D1FFF79CF96A
:10782800336843F40053336000F07EBC09A8F9F7CD
:1078380001F809A9FFF770F900F076BC9A67020809
:107848000A3F002008020020580C0020AC590020F4
:10785800551D002000270020335703080C5B00202B
:107868009A68020800080140040200200C00002069
:10787800155B0020385703083C570308FC260020F6
:1078880003F04003DBB2002B40F08980B14800F1DF
:107898006001FFF7CDF8B048F8F7CCFF8046AE4955
:1078A800AE484246F8F7F6FF002873D1AC4B434484
:1078B8005B7A302B6ED1FFF74FF93368DFF8D0923F
:1078C80043F48043336099F82B106FF07F430093A3
:1078D80009F12100082301F00F010122FFF7CAF87E
:1078E8006423CAF800307F201EF00EFDDAF800305D
:1078F800002BF8D1984699F88E10D633994E89F80E
:1079080086304B3B6FF07F4A89F88730964801F004
:107918000F0142467433CDF800A0FFF7ABF896F894
:10792800B91106F5D670033001F00F014246FF2366
:10793800CDF800A0FFF79EF896F8C41106F5DD70A3
:1079480001F00F014246FF23CDF800A0FFF792F89F
:1079580096F8CF1106F5E270013001F00F014246AA
:10796800FF23CDF800A0FFF785F896F8DA1106F5A1
:10797800E87001F00F014246FF23CDF800A0FFF7A1
:1079880079F899F899107948CDF800A001F00F011D
:10799800424646E07648F8F74DFF75494AE796F8BB
:1079A80002B0DFF8EC910BF0020B5FFA8BFBBBF136
:1079B800000F3AD199F82010FF236FF07F4809F1A2
:1079C800160001F00F015A46CDF80080FFF752F873
:1079D800684B93F86B3003F00803DBB2002B00F020
:1079E800A38399F82B10012209F1210001F00F015E
:1079F8000323CDF80080FFF73DF83368554843F47A
:107A0800003300F180013360FFF712F855485A46F9
:107A180090F8E51100F5EC70CDF80080033001F026
:107A28000F01FF23FFF726F87EE3CAF8008099F8D4
:107A380020106FF07F4300934246FF2309F11600A0
:107A480001F00F01FFF716F82AB241F211139A421A
:107A58001DD1434B5B7A302B13D1FFF77DF8336888
:107A6800454668F3514368F38E3368F34D3333600A
:107A7800414B1A7868F303021A7023780133237094
:107A880052E33E48F8F7D6FE3C49FFF745F8394E31
:107A980096F86B3013F0040F00F0468325B9384888
:107AA80020211022F8F776FC7F201EF02DFC99F893
:107AB80057106FF07F43002200933248FF2301F0F4
:107AC8000F01FEF7D7FF96F86B202F4B02F00F023D
:107AD8000D2A1A7005D125B92C4A412191754FF408
:107AE80080551A78062A08D12AB2B2F5805F04D1E7
:107AF800264A3621D1754FF488551A78082A08D1B4
:107B08002AB2B2F5885F04D1204A3821117641F2B1
:107B180010151B780B2B09D12AB241F210139A4287
:107B280004D11A4B2A225A7641F211150D486FF0EA
:107B38007F4390F8F0110022009300F5F370FF23C3
:107B480001F00F01FEF796FF96F86B3013F0010F66
:107B5800AAD0E9E29A6802081A010020155B002001
:107B68000C5B002001000020DC0C0020E70C00204A
:107B7800FC000020AC590020551D002038010020D1
:107B880004020020A50C0020E23A0020F4010020A5
:107B9800580C0020A34B1A7842B300221A700F2009
:107BA800FAF752FA06460A20FAF74EFA9E4B9F4910
:107BB80058824A7812F0010F18D06436301A588368
:107BC8009B4B1A78642A01D19B321A701B78984E05
:107BD800FF2B0BD00A21B3FBF1F1964B1931198019
:107BE80095481EF079FA337801333370DFF86482F0
:107BF80098F8003013F00F0612D18E4B19228B48DB
:107C08001A804378192143F0010343708A481EF013
:107C180063FA8A4800F12001FEF70AFF04967CE225
:107C2800012E68D1804B5A8BA2F1690189B21129C2
:107C380008D8049911F0010F04D141F00101C9B22B
:107C480004910592049A12F0020F0DD15B8A7C4AC6
:107C58001380A3F5C263023B9BB2D72B04D80498C8
:107C680040F00203DBB204931B20FEF783FF059963
:107C7800744B0AB2632A05DD642192FBF1F23032BB
:107C88001A7401E0092A0CDD059A11B2642291FBED
:107C9800F2F002FB10120A2012B292FBF0F230321C
:107CA8005A74059802B2642092FBF0F100FB11218E
:107CB8000A2209B291FBF2F002FB101230329A74D8
:107CC8005B4B1B78FF2B08D158495B484B786FF307
:107CD80000034B7000211EF0FFF9049A032A40F0BC
:107CE80023825248002143786FF3000343705248BF
:107CF8001EF0F2F911E2022E03D1534BC8221A608A
:107D08000BE2032E16D1504B1B68002B40F00C825F
:107D18004A4800F14001FEF78BFE1B20FEF72AFFC0
:107D2800414B5B8AA3F51E630F3B9BB2542B00F2B9
:107D3800FB81F2E1042E0CD13B4B988A0FF0D0FC6A
:107D4800002840F0F1813D4800F16001FEF770FE27
:107D5800E3E1052E07D1344B988A0FF0C1FC0328C4
:107D680040F0E281D9E1062E40F0D78122786FF306
:107D7800030301322270D5E1344800F12001FEF7F7
:107D880057FE334B1B78002B00F0CE81237801334C
:107D98002370304B1A786FF30302FFF794B82D4E17
:107DA800DFF8A480337813F00F021AD12A4800F1C3
:107DB8002001FEF73DFE2948F8F73CFD2749024619
:107DC8002748F8F73FFA2548F8F734FD254BA3F87C
:107DD800160233785A1C62F3030333701BF08CFFCE
:107DE80091E0012A16D1D8F80030002B40F09C8190
:107DF8001BF0AEFF012840F097811B48F8F71AFDE9
:107E0800194902461948F8F745FD002840F08C81C9
:107E180011486FE0D8F80020002A40F085810B2136
:107E28007BE000BF2E1300203032002052320020A9
:107E3800641D0020540C0020002C01405A690208DF
:107E4800581D0020F4010020FC260020DA690208F1
:107E5800541D0020551D00201A6A020874010020D4
:107E6800D0380020B05E002092010020B15E0020D2
:107E7800874E337813F00F080CD186484146FEF739
:107E8800D7FD33785A1C62F303033370824BA3F88F
:107E9800028049E1B8F1010F18D1804804211DF092
:107EA80044FD002800F040817A4800F12001FEF7E7
:107EB800BFFD33784FF0FF315A1C62F30303337070
:107EC800774B64221A60744B59802DE1B8F1020F88
:107ED800DFF8CC811BD1D8F80030002B40F024818A
:107EE8006E4804211DF021FD002840F01D816A4BD9
:107EF8005880684800F14001FEF79AFD33785A1C13
:107F080062F3030333706423C8F800300CE1D8F837
:107F18000020002A40F008810C21217062F303033D
:107F2800A9E0604910234FF40052CB700D3B8B70D1
:107F38000A805D481DF0AAFC0A2200215B48F8F778
:107F480029FA80201DF006FC237801332370504B5A
:107F58001A786FF303021A70514BC8221A60E3E0D3
:107F68005348DFF848A100F12001FEF761FD9AF8B7
:107F78000030002B00F0D8804E48DAF80020444E3C
:107F88000260BAF8042082809AF80620827131785B
:107F980011F00F0159D1DFF80881D8F80010002935
:107FA80040F0C2809AF80410A2F5A6524FF0640B74
:107FB800103A0BFB01229AF805004FF00A0909FB59
:107FC80000200393F9F7ACFD3B49F9F7B5FE0246EB
:107FD8009AF80200039BA0F5A65010380BFB030B80
:107FE8009AF80100354B09FB00B018600392F9F7C5
:107FF80097FD039A01461046F9F7E2FC304B1860EA
:10800800F9F79AF91EA3D3E9002382468B46F9F7BC
:108018006DFC002800F08880504659461AA3D3E921
:108028000023F9F759FC00287ED0FEF7DDFD3378F0
:1080380048465A1C62F303033370C823C8F800305B
:1080480009F06AFDC0B207906EE001296CD10D30CD
:108058000799832200F044FD114BD3F80080B8F152
:10806800000F61D140461DF075FB23780133237062
:10807800337868F30303337056E000BFAFF3008032
:10808800736891ED7CFF7F400AD7A3703D00804064
:10809800551D00207A6A02087A3D0020000C014034
:1080A800FC2600204E320020001001406C1D0020EC
:1080B800DA6A02080402002000007A44681D0020E1
:1080C800501D00208448854E00F12001FEF7B0FCC9
:1080D800F37913F0010F27D0DFF8488298F8009061
:1080E80019F00F0920D17E4B0A22597818781039D7
:1080F80002FB0011B1701979D878103902FB001110
:108108007170D9799B79103902FB0312327018F01B
:1081180037FFF37969F30003F37198F800305A1CBC
:1081280062F3030388F80030DFF8FC9199F80060E7
:1081380016F001063EF43BAE6A4B01221A701AF0A3
:108148006FFD2378092B01D00D2B28D1012066491A
:1081580012F0A2FA654B664A5B7803F01F03D35C02
:10816800644A522B137002D1634B01221A70634B7D
:10817800634A03F1200153F8040B8B4242F8040BC5
:10818800F9D1002117A812F0B1FA17A80D211BF098
:108198004FFD5C4B1A78013202F003021A7099F80D
:1081A800006006F00206F6B2002E00F08B800FF099
:1081B800F3FC13F067FE06980322431C93FBF2F2CC
:1081C80002EB42029B1ADBB20693002B79D1DFF84F
:1081D800488198F84960C246002E4DD0022E03D13E
:1081E80098F80130312B49D023780E2B13D146480B
:1081F80046490522F8F74EFB8246002840D1B21FB7
:1082080037484349F8F79CFB344B5646DA7942F035
:108218000102DA7135E00D2B03D13E483A490722B5
:1082280027E0032B22D13C4B002713F8012F2C2ADF
:1082380003D00137FFB2B742F7D113A832493A4603
:10824800F8F77EFB7B1C07E00AEB03025278303A12
:10825800D2B2092A03D80133DBB2B342F4D30AEB12
:108268000701FA430FA80231D21802E0264909A8EB
:10827800721EF8F765FB03E0069E02E0012600E0A7
:1082880000261E4B204A03F1100153F8040B8B42C1
:1082980042F8040BF9D1214B214A03F1100153F89C
:1082A800040B8B4242F8040BF9D1402388F81130B3
:1082B8001C3B88F82230023B88F84B301BF040FA10
:1082C80000E0002699F8003003F0F5036FF300038F
:1082D80089F80030FEF76BBD1A6B02081C580020A5
:1082E8005A1D00202E1300204D5E00204C5E0020F9
:1082F8000CA20208A53B0020541D0020F401002018
:10830800573C0020033B0020BB5A00203F5703087E
:10831800C05A00206C1D0020BA5A00200402002018
:10832800CC5A0020551D0020945A0020AFF300803D
:1083380010B5044640181146F8F71EFA2046F8F71B
:1083480079FAC0B210BD42540131C8B2704700007A
:1083580010B50D4B0D4A1B780C460E2101FB03236B
:10836800997A39B101390523594301F56E514431E0
:1083780089B201E043F6C4310019042209F0DDFB9B
:10838800201DC0B210BD00BFD1600020C017002062
:1083980010B5054B0C46197800190131042200F07C
:1083A8009FFB201DC0B210BDD160002000F53440F5
:1083B80008B5CB3009F0B0FB10F0FF0F14BF002058
:1083C800012008BD10B50A4600210446FFF7B0FF9A
:1083D80001462046FFF7DCFF114A01462046FFF719
:1083E800A7FF232201462046FFF7ADFF014620469E
:1083F800FFF7AEFF5B2201462046FFF7A4FF2322CA
:1084080001462046FFF79FFF01462046FFF7A0FFE1
:108418007C2201462046BDE81040FFF794BF00BF0C
:108428004557030810B55D220446FFF78CFF0D225F
:1084380001462046FFF787FF0023235410BD38B5B7
:108448001D460C4640182C1911461A4600F048FBE8
:10845800E0B238BD2DE9F04118490446FFF7B2FFF4
:10846800174F0E263B78174D73430146EA5A2046AC
:108478000423FFF7E4FF202201462046FFF763FFAD
:108488003B78014606FB035320469A7A0223FFF7FE
:10849800D6FF202201462046FFF755FF3B780146CC
:1084A80006FB035520466A7A0323FFF7C8FF0146F7
:1084B8002046BDE8F041FFF7B5BF00BF48570308A5
:1084C800D1600020C01700202DE9F047264E0E226B
:1084D8003378264F534337F90380FA1824494FF469
:1084E8007A73044698FBF3F8157AFFF76BFF4E2270
:1084F80001462046FFF727FF1E4B1C2202FB0535CD
:108508005FFA88F8B8F1030F01460CBF05F11202B3
:1085180005F108022046FFF70BFFA146804600251B
:1085280019E019F8013BA32B07D133780E2202FB7F
:108538000373204629465A7A08E0242B09D1337858
:108548000E2202FB03739A7A204629460223FFF77C
:1085580076FF0135EDB24545E3D120462946BDE811
:10856800F047FFF75FBF00BFD1600020C0170020B1
:10857800525703082CA20208074B187800F0040091
:10858800C0B240B11A686FF382021A60034B00222E
:108598001A70034B18787047F83A0020901D002095
:1085A800781D0020054B00211970054B05481A68F5
:1085B80061F382021A601222F7F7ECBE901D0020C8
:1085C800F83A0020781D002038B5084C0849227870
:1085D8000546F7F737FE23780021E954054B1A685A
:1085E80061F382021A60207838BD00BF901D002018
:1085F800781D0020F83A0020064A07491378112B05
:10860800C85401D801331370044A136843F00403B3
:1086180013607047901D0020781D0020F83A002054
:10862800054B1B7813F0010F05D1044B181810F8EF
:10863800010CFFF7E1BF7047911D00205A6B02083B
:108648002DE9F041334C002314F8101094F82A2037
:1086580001F00F0161F3030284F82A2004EB4000C3
:1086680084F8293084F828304378DFF8B88063F339
:108678000712638C4FF4D277E38498F800302A26E7
:108688007B4306FB0133244D2448E95A84F82A2009
:108698001DF020FD98F8003094F82A207B4302F062
:1086A8000F0206FB0233EB1859881C48013989B2BE
:1086B8001DF014FD01210A4618481DF0DBFC0121BC
:1086C80016481DF0C8FC98F8003094F82A207B431F
:1086D800120906FB02331248E95A1DF0FBFC98F810
:1086E800002094F82A3057431B0906FB0376AD197E
:1086F80069880B48013989B21DF0EEFC01210A4650
:1087080007481DF0B7FC06480121BDE8F0411DF0FF
:10871800A2BC00BF921D0020666B02080008004042
:1087280000340140BE1D002030B5164C94F82B5083
:10873800A38445F00105002384F82B50628484F853
:10874800211084F8203019E0C55CA5F13002D2B2BE
:10875800092A08D9A5F14102D2B2052A9ABFA5F182
:108768003702D2B22A46084D013305EB420292F88D
:10877800495392F84823257062700234DAB28A426B
:10878800E2D330BD921D0020666B0208124B10B573
:108798009A8C0024DA8483F8294083F828402246FA
:1087A80001210E481DF066FC64210C481DF092FC66
:1087B80032210A481DF092FC0121224608481DF08A
:1087C80059FC642106481DF085FC05483221BDE8A6
:1087D80010401DF081BC00BF921D00200008004021
:1087E8000034014010B500212C220348F7F7D2FDD0
:1087F800BDE81040FFF7CABF921D002070B5214C9C
:108808002378042B39D8DFE803F0030D152A30004C
:108818001D4B012093F82B3013F0010F30D020703E
:10882800013870BD184B93F82000FFF709FF0223A9
:10883800237022E0144DEE8CFEB9FFF7A7FF95F8E0
:10884800203095F821200133DBB29A4285F8203098
:1088580001D8042300E003232370304670BD0A4B7F
:10886800D88C50B90123237070BD074BDD8C35B906
:10887800FFF7B8FF2570012070BD002070BD0020F3
:1088880070BD00BFBF1D0020921D0020044B0022B8
:108898005A701A709A7842F001029A70704700BFB5
:1088A800E81E0020202102480A46F7F773BD00BFE2
:1088B800F401002038B5044608460D46F7F7BAFF1C
:1088C80098B10319202B094BC8BFC4F120001C190B
:1088D800002308E014F8012BE02A14BFEA5C2022E8
:1088E80004F8012C01338342F4DB38BDF401002085
:1088F8000D4B46F669321B689B6893420FD043F6CE
:10890800FC2293420BD0122B09D0B3F5E97F08D093
:1089180046F60D401B1A584240EB030070470120F1
:1089280070470120704700BFF81D0020F0B51F46B2
:1089380087B006460C46084600211546F7F72AFD7B
:10894800244B07B19F80B3F9041005A801EB8601F9
:10895800042209F0F2F8002605AB9B5D013BDBB26F
:10896800B92B35D81D2B4FEA031209D8D31803F5B4
:108978002641684601F5BF71112209F0DEF80BE0C7
:108988001549D3185B186A4603F110071868596827
:108998000833BB4203C2F9D12046F7F74BFFC7B2F1
:1089A8006846F7F747FF3818A84203D8E019694620
:1089B800F7F7E2FE6846F7F73DFF7B1C1B18AB4252
:1089C80003D2E0190549F7F73FFD0136042EC3D15C
:1089D80007B0F0BDE81E0020503903086A570308A5
:1089E80010B500216C220446F7F7D4FC0123A370CC
:1089F80010BD002343700370837843F00103837034
:108A0800704700002DE9F0419378804613F0010F7C
:108A18000D4614463AD06FF3000393701AF068FEBF
:108A28006378002B32D123780BB90A336370A378AB
:108A3800174F6FF30003A3701AF05AFE217807EB63
:108A480008066118073130462A46F7F779FF30469D
:108A5800F7F7F0FEC6B2AE420DD80AD20023237053
:108A680006EB08000A33637038182021AA1BF7F7B1
:108A780091FCAE420AD12278A3181B7A1BB10132AD
:108A88002270BDE8F08123700A236370BDE8F0818D
:108A9800F4010020054B1A780AB100221A701B78DD
:108AA80046F68A4202FB0311FFF704BFDB1D0020D4
:108AB800F8B505460C460818002109F023F8013CD2
:108AC800E4B26719384609F027F8C6B2202E03D851
:108AD8003846002109F016F80CB1202EEFD9F8BD60
:108AE80002F00F03032B22F07F0230B5D2B20CD96B
:108AF8004FF47A7491FBF4F42025E4B2057002B1C6
:108B080014B13034047000220130B1F57A7F05DBEE
:108B18004FF47A7491FBF4F504FB1511022B0BD971
:108B2800642491FBF4F42025E4B2057002B114B179
:108B38003034047000220130632904DD642491FB81
:108B4800F4F504FB1511012B0AD90A2391FBF3F361
:108B58002024DBB2047002B10BB130330370013052
:108B6800092904DD0A2391FBF3F203FB12113031CA
:108B7800017030BD13B5104B01461B689A899C7B68
:108B880012F0100214BF0220012034B10B4C9B7C60
:108B98002478634303FB001109B23AB10DF10600D2
:108BA800022208F0CAFFBDF8060002E0084608F0F5
:108BB800B3FF00B21CBD00BFF81D0020871E0020B7
:108BC80010B50F4B1B689A899C7B12F0100214BFDA
:108BD8000221012134B10B4C9B7C2478634303FBB5
:108BE800010000B22AB108490222BDE8104008F08D
:108BF8009EBF054B1968BDE8104008F083BF00BF51
:108C0800F81D0020871E0020A01E00203038C0B2AA
:108C1800092894BFFF20002070470000024B1A78F3
:108C28006FF300021A707047D71E002070B5FFF767
:108C3800F5FF884B1A781E2A01D91E221A70864C15
:108C48002678254606F0F006202E72D109F0C4FADF
:108C580000286ED1814B1B7833B92378C3F30312F4
:108C6800013262F307135EE07D4B1B7803F080034B
:108C7800DBB2002B59D07B48F7F7DCFDC5B27A4C44
:108C8800BDB1204679493246F7F75AFE0A2D0BD86E
:108C98002A4620467349F7F753FE60193146C5F155
:108CA8000A02F7F777FB04E020466E490A22F7F735
:108CB80047FE6F4B1B7813F0010F01D0472300E0EC
:108CC8002023E372684C042204F10C00A521F7F775
:108CD80061FB684B1A7852B1FF23012A237306D926
:108CE800022A637303D0032AA37318BFE373624C89
:108CF800257815F0600502D194F8A33013B95F48C0
:108D08005F4902E05D4804F1A3010622F7F718FE67
:108D18005C4B1B78452B40F09A81002D40F09781E1
:108D2800237843F08003237070BD4F48564932467C
:108D380082E12C7804F0F004102C3FD109F04CFAB1
:108D480000283BD1202251494748F7F7F9FD46480A
:108D58004E492246F7F7F4FD4D4B1B7813F0010FEF
:108D680006D04C48F7F766FD4A4902464A4805E0EE
:108D78004A48F7F75FFD494902464748F7F7E0FDDB
:108D8800364B1B781BB946484649102254E14448E3
:108D980045491022F7F7D4FD314B1B7803F08003C7
:108DA800DBB22BB13B48F7F745FD02463F484FE0A1
:108DB8003A48F7F73FFD02463C4842E02B7803F07B
:108DC800F003302B7ED109F007FA00287AD1264C1F
:108DD800202237492046F7F7B3FDA521052204F1E3
:108DE8000B00F7F7D7FA334B1B78042B02D9FF2374
:108DF800E37300E002D1FF23A37301E0032B02D148
:108E0800FF23637301E0022B02D1FF23237300E0E9
:108E18000BB1FF23E372284B5B7813F0600F05D08A
:108E28003F23E37223736373A373E373234B1B78AA
:108E380003F02003DBB233B11848F7F7FBFC024616
:108E48001F481649F8E01348F7F7F4FC02461C4897
:108E58001049F1E0E31E0020D71E00202C27002037
:108E68000027002004270020F40100203CFF02080E
:108E7800C8600020F9270020342700200E020020B7
:108E880057D50208C01D0020FAFE02083F35030826
:108E9800923F00208936030801020020AA36030801
:108EA800040200200C3B030860350308110200206F
:108EB800FCD502081F2D002058320020F83A002067
:108EC8000F0200202B7813F0F0030CD12022604908
:108ED8006048F7F735FD604B5E4819888322BDE886
:108EE8007040FFF7FDBD602B1ED109F075F9D8B9A8
:108EF8005A4920225748F7F723FD5948F7F79AFCB3
:108F0800574902465748F7F71BFD5748F7F792FCB1
:108F1800554902465548F7F713FD5548F7F78AFCB7
:108F280053490246534887E02B7803F0F003102B8F
:108F380006D109F051F918B146484F4920227BE083
:108F48002B7803F0F004402C02D0502C78D108E0A4
:108F580040484A492022F7F7F3FC494B1B784BB9A4
:108F68004CE03C4847492022F7F7EAFC464B1B787F
:108F78003BB943E0454B5A7882B11B78022B14D198
:108F880005E0434B1B7813F0010F07D00DE0414873
:108F9800F7F750FC3F4902463F4835E03F48F7F7AE
:108FA80049FC3E4902463C482EE03D48F7F742FC62
:108FB8003B4902463848F7F7C3FC402C0BBF334BFC
:108FC800384B5B78DB78022B0AD0042B0FD0012BAF
:108FD8001CD13548F7F72EFC3349024633481BE0CD
:108FE8003348F7F727FC32490246304814E0314845
:108FF800F7F720FC2F4902462C480DE02E48F7F7DA
:1090080019FC2D4902462448F7F79AFC2B48F7F734
:1090180011FC2A4902462548F7F792FC284B1B7891
:10902800ABB9202107222148F7F7B4F92248F7F70E
:1090380001FC214902461D48BDE87040F7F780BC95
:10904800204A6FF3071313701F4B00221A6070BD7C
:1090580099D50208F4010020D61D002078D5020811
:1090680078CE0208F801002082CE0208080200200B
:109078007DCE02080F020020DBD5020881350308E7
:10908800E03A0020A23503082C270020F236002001
:10909800C860002047360308FD010020EC360308AD
:1090A80089360308D4260020C33503080D020020A2
:1090B800E435030805360308CB36030826360308CB
:1090C800D7340020D71E0020F81D0020204B70B593
:1090D800F022204D1A702B7813F0010F0BD01E4C84
:1090E800207810F0010006D11C49FFF7D3FC237843
:1090F80043F0010323701A4E3378532B0ED1164CCC
:10910800237813F0010F07D000201649FFF7C2FC9F
:1091180023786FF300032370FFF780FD3378232B48
:1091280014D10D4B1B7813F0010F0FD1FFF776FD0B
:109138002B780D4A43F006032B701378013BDBB202
:1091480013700A4A52F82320094B1A6070BD00BFF9
:10915800E31E0020D71E0020FD1D0020102B030851
:10916800C01D0020EF2A0308B71E0020C41E0020DF
:10917800F81D00202DE9F0415E4BF0225E4D1A707B
:109188002A7802F01003DBB2002B2DD15B4963F380
:1091980047120B601C462A70594A9A5C2D2A01D046
:1091A8000134E4B20133112BF6D1564E3A21304640
:1091B800F7F76EF938B1801BC0B20130301821467C
:1091C8000222FFF78DFC504B1B78452B40F08F8017
:1091D80000242046013412F0ADFE112CF9D12B7871
:1091E80043F010032B703CE0484C237813F0010F38
:1091F80017D1424E4648FFF7F3FB424F31683846D5
:1092080001310222FFF76CFC2D23BB70307846F643
:10921800955340496522FFF789FB237843F0010302
:10922800237003200D213A4AFFF7ECFB2D78324ECC
:1092380015F0E00545D110203749FFF72BFC324BDC
:109248001B78442B11D12D4A136801331121B3FB2C
:10925800F1F101EB01115B1A2949C95C2D29F4D000
:109268001360BDE8F041FFF7D9BC532B0DD132781C
:109278004E3B63F347123270204A28491268062091
:1092880000FB02125380BDE8F081232B2FD11B4B2A
:109298001D60337803F0EF0365F347133370FFF76E
:1092A800BDFC23781E4A43F0060323701378013B64
:1092B800DBB213701B4A52F823201B4B1A60BDE81F
:1092C800F081104C10201949FFF7E4FB04F110005D
:1092D8002821F7F7DDF850B1001B3178C0B2013012
:1092E800201849098022BDE8F041FFF7F9BBBDE825
:1092F800F08100BFE31E0020FD1D0020A01E0020FD
:10930800493D0020F4010020C01D0020D71E002088
:10931800E81E0020EF1E00208C2A03087A3D00205A
:10932800B71E0020C41E0020F81D0020AD2A030827
:10933800454B2DE9F041F022444E1A703378444DE4
:1093480043F0010333702B68424C9B7C022B06D1FF
:10935800414B1B7803F04003DBB23BB10FE0012B1C
:109368000DD13E4B1B7813F0010F08D109F0ACF872
:10937800236800206FF355532360394944E0A378EC
:10938800344F03F02003DBB2C3B909F09DF8F87835
:1093980000F02000C0B288B92968324B897C1A785D
:1093A80061F301021A703B682D4943F400133B60D6
:1093B800FFF770FB2C4B802283F843200DF040FD13
:1093C800804678B12B689B7C012B08D1234B5B78B6
:1093D80003F01003DBB213B10020244914E000208D
:1093E800234911E00DF05CFD074610B140462149C4
:1093F8000AE00DF09DFD10B138461F4904E01A4BF4
:1094080093F8433013B91D49FFF744FB1C4B1B78F5
:10941800232B16D1FFF702FC337843F00603337091
:1094280009F052F823686FF3555323600CF0FCFBE6
:10943800144A1378013BDBB21370134A52F82330F5
:109448002B60BDE8F08100BFE31E0020D71E00207E
:10945800F81D0020F83A002000270020923F002045
:10946800312B0308973F002081220020732B03082B
:10947800522B0308B52B0308942B0308D62B03089B
:10948800C01D0020B71E0020C41E00202DE9F34196
:109498006E4B6F4DF0221A702B686E4C9B7C1BB97B
:1094A800637843F0100302E0637843F008036A4EE0
:1094B8006370337843F001033370238823F47E63A9
:1094C80023F01E03DB04DB0CB3F5805F08D0634B8D
:1094D8001B7883B15F4B5B7803F00803DBB253B1B1
:1094E800637800206FF341035D496370FFF7D2FA98
:1094F800F8F7E6FD84E06378564F03F00203DBB229
:10950800FBB9BB78EBB9574B93F8008018F001080A
:1095180017D1F8F7D5FD7B7843F002037B702B68F1
:10952800B3F91030022B7B780CBF43F0040368F3C7
:10953800820300217B70082001220B460091F9F775
:10954800DDF8A378434A032B28D003D8012B0BD08E
:109558000DD806E0052B2DD0517825D3FF2B32D11D
:109568002BE000203E4949E000203F4946E03F48C3
:10957800F7F760F9DFF82C81C7B23C4908F1100011
:109588003A46F7F7DDF90F2F3AD807F110004044B3
:109598002021C7F11002F6F7FDFE31E0344B1878B0
:1095A80000282DD1334929E06FF341015170002083
:1095B800314923E00020314920E06FF34101517027
:1095C80000202F491AE0053BDBB26FF34101022B63
:1095D800517002D100202B4910E0012B02D100204C
:1095E80029490BE0032B02D10020284906E0052B6E
:1095F80002D10020264901E026490020FFF74AFA57
:10960800637803F00203DBB20BB9F8F759FD224B7C
:109618001B78232B18D1FFF701FB3378002243F086
:10962800060333706378A27003F0E50362F38203E4
:109638006370F8F745FD194A1378013BDBB21370E4
:10964800174A52F823302B60BDE8FC81E31E002046
:10965800F81D0020C8600020D71E0020F236002028
:10966800312B0308CE60002074270308D760002040
:10967800CC60002095270308392C03081928030813
:109688007C280308B6270308D7270308F827030808
:109698003A2803085B280308C01D0020B71E0020D5
:1096A800C41E0020F40100207B4B2DE9F341F02279
:1096B8007A4E1A7033787A4D43F0010333702B6871
:1096C800784C9B7C022B11D1774B1B7803F040031D
:1096D800DBB293B1754B1B7803F02003DBB2BBB14F
:1096E800A37803F04003DBB23BB111E0012B0FD1AB
:1096F8006F4B1B7813F0010F0AD1F8F7E1FC2368D0
:10970800002023F480036FF3D753236069498FE067
:10971800A778DFF8908107F04003DFB2002F34D13B
:10972800F8F7CEFC2968644B897C1A78384661F3CF
:1097380001021A70D8F800305E4943F4800367F3D9
:10974800D753C8F80030FFF7A5F92B68198A21B953
:109758000091082001220B4615E00BB2022B0CD118
:1097680001223B46082039460097F8F7C7FF534BBC
:109778001A7842F008021A7007E0012B05D1009709
:109788000E2039463A46F8F7B9FF0DF059FB07465F
:1097980078B12B689B7C012B08D1454B5B7803F093
:1097A8001003DBB213B10020454941E000204549D0
:1097B8003EE0414B3946187800F00300F8F7B8FD51
:1097C800FF280FD13D4B1B7803F01803182B31D01D
:1097D800A07800F08000C0B210B138463A4927E0BE
:1097E8003A4925E00DF05CFB8046E0B1334B187830
:1097F80000F008085FFA88F8B8F1000F0AD1F8F706
:10980800EDFEC0B2022801D840460AE0062811D869
:10981800404604E000F01000C0B210B138462C49B0
:1098280006E02C4904E00DF083FB18B12A494046B4
:10983800FFF730F9294B1B78232B29D1FFF7EEF9D5
:10984800337843F006033370F8F73AFC236823F4BF
:1098580080036FF3D7532360184B1A786FF3C30252
:109868001A701F4A1378013BDBB213701D4A52F875
:1098780023302B60104B1B7803F00303022B02D11B
:109888000DF0B4FA20B102B0BDE8F0410CF0CCB94B
:1098980002B0BDE8F08100BFE31E0020D71E002003
:1098A800F81D0020F83A0020002700203427002067
:1098B800923F0020312B0308973F00201020002002
:1098C800732B0308522B0308392C03085A2C03085E
:1098D800182C0308F72B0308942B0308C01D00203D
:1098E800B71E0020C41E002010B5FFF797F90A48DC
:1098F8002523C377094B0A4A1B6813219B7C1C301C
:1099080001FB03235B78093903F00F0359438322D2
:10991800BDE81040FFF7E4B8F4010020F81D00206E
:109928000C3B00202DE9F047514D524F2B78F02287
:1099380043F001032B70504BDFF878911A703B68A5
:109948009C6847F2F373E21A544244EB0204132171
:1099580061434A4A565C5318C6F300065FFA86F814
:109968009246B8F1000F23D140464549FFF792F8D7
:1099780099F80030232B79D1FFF750F92B78414A19
:1099880043F006032B701378013BDBB213703E4A99
:1099980052F823303B603D4B1E703D4B1E703D4BD3
:1099A8001E703D4BC3F800803C4B1E70BDE8F0872D
:1099B80099F80020232A21D19A786FF300029A702F
:1099C8000EF096F9FFF72AF92B782E4A43F0060392
:1099D8002B701378013BDBB213702B4A52F82330FB
:1099E8002A4A3B6000231370294A1370294A1370CE
:1099F800294A1360294A1370BDE8F087532A13D106
:109A08009A7812F001010FD172206043244D42F080
:109A180001022E5C61F300062E549A701E4B01223F
:109A28001A60204616F0C0FC132303FB04A39B789E
:109A380013F0010F02D000201A4913E0164B1B68DF
:109A480073B9382102221848FFF74AF8204615F062
:109A580045FF014615480222BDE8F047FFF740B828
:109A680013490020BDE8F047FFF714B8BDE8F087B8
:109A7800D71E0020F81D0020E31E00200C3B00200C
:109A8800C7E30208B71E0020C41E0020DD1D002009
:109A9800061E0020871E0020A01E0020921E002007
:109AA800305700206A2E0308120200200D02002001
:109AB800492E0308C01D00202DE9F0412D4E2E4FE0
:109AC800307800F5E240F13008F026F83B78C4B26F
:109AD80013F0010F26D0294D2B78552B0AD1EC2CE9
:109AE80001D0013CE4B23078214600F5E240F13083
:109AF80008F008F82B78442B0DD1A4F11403DBB23D
:109B0800D72B01D90134E4B23078214600F5E24080
:109B1800F13007F0F7FF2B78532B03D1FFF77EF8CE
:109B28000EF0E6F8164B1B7803F08003DBB253B156
:109B38003B7813F0010F06D0124820210422BDE81B
:109B4800F041F6F727BC14F0800F0F4805D12B23FE
:109B58000A2103746143113006E02D230374373B57
:109B68005C43113004F520610322BDE8F041FEF7A3
:109B7800B7BF00BF871E0020D71E0020C01D0020D1
:109B8800F83A002004020020F40100201FB5204B01
:109B980020491A781AB1087840F00100087009784D
:109BA8001C4C11F0010F31D01B490978532901D001
:109BB8000AB103E082B901221A700DE023290BD102
:109BC800002018701549FEF765FFFFF727F823787E
:109BD80043F00603237019E01B78012B16D12021CE
:109BE8000A460F48F6F7D6FB0E4B68461B6810224C
:109BF800996807F0A2FF002409491DF8040001EB49
:109C0800440101341AF0C0FE102CF5D11FBD00BF6D
:109C1800871E0020D71E0020C01D002082310308A7
:109C2800F4010020F81D0020034B1B78532B01D1B1
:109C3800FEF7F4BF704700BFC01D0020084BFF2887
:109C48001A68936807D1917B41B10649927C0978DB
:109C580001FB023302E0927C02FB00331846704796
:109C6800F81D0020871E00204328F8B504460D463D
:109C7800174608D1114B0A261A7891FBF6F66FF3AE
:109C8800C3021A7000E00E462046FEF7BFFF90B1EF
:109C98000A4B303C1A780A2602F00801C9B200299A
:109CA80018BF002506FB05466FF3C30236B21A70CB
:109CB800BE42A8BF3E4630B2F8BD00BFD71E002046
:109CC800624B2DE9F3411A689846157C977C604CE5
:109CD8002DB1604821780222FEF702FF00E02570CE
:109CE800FF01237807F51C4707F5B47707EB43070F
:109CF800594E0BB90DB10FE015B901A8394601E06D
:109D080001A8B91E022207F018FF9DF80430F37568
:109D18009DF80530337605E006F117003F21022251
:109D2800F6F738FB5B23B375023373764B4B1B781E
:109D380013F0010F5DD04A4B1B78A3F13002D2B269
:109D4800092A31D822780AB9002D3CD1454A117820
:109D580096469942444A01D000211170434811782F
:109D6800A3F1300490F800C004EB840404EB01086C
:109D780002A801318444C9B23D48641810F808802B
:109D8800005D0CF8048C117008B1032901D9002179
:109D980011708EF800300DB9384600E0B81E01A9E0
:109DA800022207F0C4FE17E0232B04D12F4B1A78A8
:109DB80092B9013205E02A2B05D12C4B1A785AB1F9
:109DC800013A1A7008E0532B06D12A4A533B137004
:109DD800264A1370FFF728FF274B1B7803F08003F0
:109DE800DBB2002B2FD0214B1B78F6182023F375FC
:109DF80029E045B31A4B1878A0F13003DBB2092BE0
:109E080010D81C4A137803B92370013303F00103F7
:109E18001370D8F800302178B3F91020FFF724FF29
:109E2800207005E0432803D1124B1B7803B9237037
:109E3800114B1B7803F08003DBB223B105482021C6
:109E48000222F6F7A7FABDE8FC8100BFF81D002042
:109E5800071E002002020020F4010020D71E002067
:109E6800C01D0020DA1D0020061E0020D81D00207D
:109E7800D46E0208921E0020F83A0020F7B5384E3A
:109E8800384D3378384C6FF34103337019F022FAA8
:109E9800FFF7CAFE02238DF807302B7883B1334AC7
:109EA800D17941F00101D171314A207802EBC30325
:109EB8005F6B93F839203978FFF7D6FE38700DE0DC
:109EC800337813F0010F06D02378303BDBB2062B32
:109ED8009CBF264AD37003238DF80730337813F0DC
:109EE800010F12D0234B1B7803F08003DBB263B160
:109EF80029781F4B204803EBC10393F838309DF8AD
:109F08000720C0182021F6F745FA2378232B09D11A
:109F18001A4A2B781268927C013A934202DA114A63
:109F28000133137023782A2B04D12B7813B10D4AEF
:109F3800013B13702378532B0FD117F021F80B4BEB
:109F480000212970DA7961F30002DA71FFF76CFEFB
:109F58000B4B9A7942F004029A7100232370FEBDDC
:109F6800D71E0020921E0020C01D00201C58002073
:109F7800D46E0208F83A0020F4010020F81D0020F1
:109F8800042000202DE9F74F924E934C3378934DDF
:109F9800232B934F25D12368986843F6F1239842E1
:109FA80017D1DFF86082296898F8000000F56A5038
:109FB800713007F0A7FD98F80000013000F00100AB
:109FC80088F8000000F56A50713007F0A5FD286098
:109FD80007E000B2FEF7CEFD28603B7843F00803A7
:109FE8003B703378532B40F06781236849F615524C
:109FF8009B68934202D12A687A4B15E04BF2B6422D
:10A00800934202D12A68784B0EE04BF233429342D6
:10A0180002D12A68754B07E049F66652934204D18B
:10A028002A68734B02B101221A7023689A6843F6B2
:10A03800DD239A420AD16F4B29681A7861F300022E
:10A048001A7008F0C9F808B108F0E4F8236843F674
:10A05800E0229B68934206D1664B29681A7861F31F
:10A06800C7121A7019E043F6EA22934206D1614BEF
:10A0780029685A7861F300025A700EE043F6E72225
:10A0880093420AD129685C4B19B11A6842F0005210
:10A0980002E01A6861F35D721A6023689A684BF2ED
:10A0A8004C539A420AD12968544B19B11A7842F094
:10A0B800200202E01A7861F345121A7023689A6840
:10A0C8004BF2D9539A4202D1287819F06BFE2368D3
:10A0D80043F6DA229B68934203D12A68484B1A70E8
:10A0E80008E049F61E52934204D12B6813B93B4B42
:10A0F80001221A6023689A684BF2DA539A420BD10C
:10A10800404A2B6812784049032B8B5404D13F4BAB
:10A118005A7942F010025A71236849F65E529B68D8
:10A12800934202D129683A4A05E049F661529342BE
:10A1380003D12968374A117016E049F662529342F2
:10A1480003D12968344A117015E049F664529342E4
:10A1580003D12968314A11701CE049F665529342CF
:10A1680002D12A682E4B13E043F60852934202D1DB
:10A178002A682C4B0CE04AF26C72934202D12A688E
:10A18800294B05E04BF2CA42934203D12A68274B78
:10A198001A700AE049F61652934206D12A68244BEF
:10A1A80001201A7001460EF0ABFB2368986843F64D
:10A1B800F12398423ED1DFF84C80296898F80000D6
:10A1C80000F56A50713007F09DFC002388F80030D4
:10A1D80033E000BFC01D0020F81D0020A01E002095
:10A1E800D71E00202C270020E03A0020D73400207A
:10A1F800BE1D0020551F0020F83A0020C86000202E
:10A20800AA5A0020871E0020B8170020D426002054
:10A218006440002062400020953F0020093F002054
:10A2280084200020F6150020A11C0020761D0020A7
:10A23800023E002000B2FEF7C3FC23689A6843F68A
:10A2480098139A4236D12968DFF8A8B2DFF8D0A26D
:10A258000BEBC1031B79DFF8A082C3F34113012B79
:10A26800DFF8C09221DD98F8000000F56650203034
:10A2780007F048FC98F80030DAF8001009EB030200
:10A2880011720BEBC1021279C2F34112032A0CD1ED
:10A29800974A126890681030C01807F033FC98F895
:10A2A8000030DAF800204B441A7498F800302A6815
:10A2B80009F80320FFF7B8FC3B78DFF86C8213F04D
:10A2C800010F00F0DC80216843F698128B689342F6
:10A2D8007FD1884A2B68914602EBC3010979C1F303
:10A2E8004111012906DD844A1278072A02D9FEF7AE
:10A2F80095FCD0E03278442A36D15FFA83F82DE015
:10A3080008F101087B4B5FFA88F803EBC8031B7957
:10A31800C3F34113012B06DD784B1B7823BB764B27
:10A328001B78072B20D8DFF8D0A19AF800303F2BF4
:10A3380008D807F051FF70B109EBC8031B7913F077
:10A34800100F08D19AF800303F2B07D909EBC80342
:10A358001B79DB0902D0C5F8008005E009EBC803CA
:10A368001B7913F0080FCBD03378552B40F093802E
:10A378002E782BE0013EF6B209EBC6031B79C3F336
:10A388004113012B08DD5D4B1B78002B40F08380C7
:10A39800594B1B78082B7ED8DFF85C8198F8003081
:10A3A8003F2B08D807F018FF70B109EBC6031B79DB
:10A3B80013F0100F08D198F800303F2B06D909EB9D
:10A3C800C6031B79DB0901D02E6064E0002ED1D1D1
:10A3D80061E04BF2DA5293420AD005DCA3F534422D
:10A3E800CA3A012A0ED803E04BF23762934209D1E8
:10A3F80033782F2B4FD9B1F91020303293424ADCF1
:10A40800303B30E043F6F122934207D13A4B1B78B8
:10A4180023B13078B5F900103B222CE007F0DCFEC0
:10A4280018B3236843F6C4219A688A4203D047F2D6
:10A4380001118A4204D13078B5F900102D221AE0B2
:10A44800A2F56A516139052903D943F6E9218A42FF
:10A4580001D1012307E043F6E0218A4202D00A3104
:10A468008A4203D100232B6015E023683078B5F9C0
:10A478000010B3F91020FFF7F7FB28600BE0236802
:10A48800B3F90800FEF776FB286098F8003043F02F
:10A49800080388F80030FFF7C7FB236843F6D22289
:10A4A800986890420BD12B6813B91548154901E0FB
:10A4B800134815490222F6F743FA0226C8E14BF27F
:10A4C800376290420AD12B6813B91048104931E01D
:10A4D800012B0E480CBF0F490F492BE04BF2DA5203
:10A4E800904236D12B68012B20D108480B4921E036
:10A4F800F81D002014040020871E00204A0D0020AB
:10A5080012020020386F02083A6F02080402002085
:10A51800661D0308A81D0308871D03083D1C0308C2
:10A52800A01E0020202D0020D71E0020022B05D1C0
:10A53800A548A6491022F6F703FA88E1032B02D1B1
:10A54800A148A349F6E7042B9F480CBFA149A2499B
:10A55800F0E74BF2CA4290420AD12B6813B99A48E5
:10A568009E49E7E7022B98480CBF9D499D49E1E7C2
:10A578004BF2CB4290420AD12B6813B992489A49C0
:10A58800D8E7012B40F063818F489849D2E749F614
:10A598006352904203D043F6EE2290420ED12868CF
:10A5A8000A21B0FBF1F201FB1201914B3031D9774E
:10A5B80030322E2199775A77032649E143F6F12262
:10A5C80090423ED18B4B1B78E3B9022229688A4816
:10A5D800FEF786FA43F6F220FEF7CCFA022201468D
:10A5E8008648FEF77DFA3B7813F0010F00F0808172
:10A5F800834B1B7803F08003DBB2002B00F07881DB
:10A608007D4819E0FEF7B6FA022201467A48FEF7BD
:10A6180067FA022279482968FEF762FA3B7813F054
:10A62800010F00F06581764B1B7803F08003DBB2E5
:10A63800002B00F05D81714820210222F5F7AAFE67
:10A6480056E143F69812904240F0B5802B686D4E63
:10A65800DFF8A08156F8331010225B48F6F770F93E
:10A668000DF1060298F800000DF1070110F098F9B5
:10A678004246334620B316786349895D03291FD0C3
:10A68800296803EBC1010979C1F34111012917D1E7
:10A69800072E15D95D490B225D48F6F751F95D483B
:10A6A800711C0222FEF71CFA9DF807105A48013166
:10A6B8000222FEF715FA9DF806105848013118E0F5
:10A6C8002E68157803EBC601097903EBC6063679BF
:10A6D800C1F34111012906F00706C8BF05F00705B7
:10A6E800012E0ADC4E494A480B22F6F729F9494857
:10A6F800691C0222FEF7F4F9A9E0022E0BD14949A0
:10A708000B224348F6F71CF932464248691CFEF70B
:10A71800E7F90E369CE0032E0BD143490B223C4847
:10A72800F6F70EF93B48691C0222FEF7D9F90D36F7
:10A738008EE0042E11D13D490B223548F6F700F979
:10A748003448691C0222FEF7CBF9334805F10901A8
:10A758000222FEF7C5F90C367AE0052E11D13449EC
:10A768000B222B48F6F7ECF82A48691C0222FEF760
:10A77800B7F9294805F109010222FEF7B1F90B36AC
:10A7880066E0062E63D12B490B222148F6F7D8F84C
:10A798002048691C0222FEF7A3F91F4805F10901A8
:10A7A8000222FEF79DF9244805F111010222FEF765
:10A7B80097F90A364CE0B3F91060092E3EDD632E96
:10A7C800CCBF032602263AE0040200205E1C0308E0
:10A7D8007F1C0308A01C03081C1C03080B1E03088D
:10A7E8004D1E03082C1E03088F1E0308B01E030805
:10A7F800F4010020871E00200F0200201202002012
:10A80800F83A002014040020202D0020F437030813
:10A81800F9010020FA010020FE01002001020020B9
:10A82800B23703080D370308913703084F37030879
:10A838002E370308703703080202002001262D482E
:10A848002968801B46F08002FEF74AF900E01026CE
:10A858003B7813F0010F0BD0274B1B7803F08003D4
:10A86800DBB22BB123482021801B3246F5F792FD3D
:10A87800224EB37803F00203DBB2002B38D0FEF788
:10A8880037F81F4D034628B92878F11D6522FEF7D1
:10A898004DF808E0B2792978B388F01D01FB023140
:10A8A80009B207F04AF9236847F201129B689342FC
:10A8B80013D006DC43F6C42293420ED043F69E52D0
:10A8C80009E047F28112934207D049F61E5293429B
:10A8D80003D047F2411293420AD105200B21074ABF
:10A8E800FEF790F82978074801310222FEF7F8F8B8
:10A8F800BDE8FE8F14020020F83A0020E81E002070
:10A90800871E0020F5010020F0B5114B1F78114B70
:10A91800303F1E680DE0D6F814C01CF803C00133A0
:10A92800644501D112E00023DAB28242F3D3013543
:10A938000D70094B0622094902FB07330D785B1994
:10A9480093F86840002CEED10C70F9321046F0BD37
:10A95800C01D0020F81D0020D46E0208061E00202D
:10A968002DE9F74F964C974E23689A6843F609539A
:10A978009A4203D133780BB9013333702368924F6D
:10A9880099689B7C3A78B3F1010848BF03F106083F
:10A998004FEAE808337808F1010812F0010F03FBC9
:10A9A80008188A4D00F0AD80894B1A789946432AD9
:10A9B8004DD128780FFA88FA0AEBD00007F0ACF8E6
:10A9C8002268844B916846F2C8629142186001D1AE
:10A9D8002A783AB12A78012102F0070211FA02F224
:10A9E80050401860287819780AEBD00007F08AF8E8
:10A9F800236847F2E1129B68934209D1734B1A7896
:10AA0800754B03EBD203734A126883F8A0211EE04A
:10AA180046F6A932934205D13178002001310EF073
:10AA2800CBFA14E046F2BF7A4FF0000B23689B681C
:10AA3800534504D101200BEB00010EF0BDFA0AF1D9
:10AA4800080A46F2FF739A450BF1010BEED199F80B
:10AA58000030232B10D122682B78927C013A934244
:10AA68000ADA5A4A013313705C4B9B7803F00203ED
:10AA7800DBB20BB1FDF70AFF99F800302A2B0CD195
:10AA88002B7853B1514A013B1370544B9B7803F018
:10AA98000203DBB20BB1FDF7F9FE99F80030552B34
:10AAA80014D12368997C0F2910D92A7808398A4249
:10AAB800464B01DA083200E000221A70474B9B78B7
:10AAC80003F00203DBB20BB1FDF7E0FE99F80030AA
:10AAD800442B42D123689A7C0F2A3ED929783B4BD4
:10AAE800072902D90839197001E0083A1A703B4B56
:10AAF8009B7803F00203DBB2002B2ED0FDF7C6FED5
:10AB08002BE049F6D54399420ED1314B1B78A3F17E
:10AB18003101C9B2072907D842F006023A70072264
:10AB28005343284A573B137023689A6843F60953DE
:10AB38009A4212D133781B2B08D9284B46F69542F6
:10AB48009A809A7842F002029A7006E05901C91870
:10AB5800234B0020C918FDF79DFFFFF765F8214A30
:10AB68002B7811789346994288BF137012780F3268
:10AB7800934202DD1B4A0F3B137023684FF0000A13
:10AB880093F81290B9F10F0F9ABFC9F120095FFA33
:10AB980089F94FF010099BF800004FFA8AF318184A
:10ABA8000FFA88F202EBE000019306F0B5FF9BF87C
:10ABB8000020019B5FFA80FC9B1803F007032AE042
:10ABC800F81D0020871E0020D71E0020921E00209E
:10ABD800C01D0020A01E0020202D0020E81E0020FF
:10ABE800C0200308891E00204CFA03F06549013390
:10ABF80000F0010000280CBFA520DB20DBB201F823
:10AC080009000AF1010A09F10109082B5FFA8AFA19
:10AC18005FFA89F903D0B9F1200FE5D109E0B9F15C
:10AC2800200F06D023684FFA8AF19B7C8918994235
:10AC3800B1DB3B7813F0010F15D0236852499B7C98
:10AC480009780F2B01F0800198BFC3F11003C9B236
:10AC580094BFDBB2002331B1297810318A1A4949EF
:10AC6800CB185F219954DFF8288198F802304746BD
:10AC780003F00203DBB2002B64D0FDF739FE034674
:10AC880000BB226846F6A93192688A4206D0243170
:10AC98008A4203D043F6E5118A4204D130783B4911
:10ACA8006522002309E043F609518A4208D1307829
:10ACB8001C38C0B208F107016522FDF737FE18E01D
:10ACC8002878F7E7236846F669329B68934203D0F1
:10ACD80043F6FC22934202D1BA79317801E0BA797D
:10ACE8002978BB88294801FB0231BA7909B206F0F4
:10ACF80024FF23689A7C102A02D905200B211EE024
:10AD08009B6846F6693293420ED006DC43F6E5129C
:10AD1800934209D043F6FC2204E046F6A932934256
:10AD280002D02432934201D1102007E043F60952A1
:10AD3800934202D10020102101E000200721144A8B
:10AD4800FDF760FE226846F60D4193688B4216D0E7
:10AD580046F6C7218B4212D043F6ED218B4202D131
:10AD6800084BDB219977937C102B08D9297809485F
:10AD78000131022203B0BDE8F04FFDF7B1BE03B0C8
:10AD8800BDE8F08FF4010020F83A0020EF1E002003
:10AD9800E81E0020F5010020114B002270B50D4679
:10ADA8001A7118B11B7803B920234370BDB10D483F
:10ADB800F5F740FD0446681C5CB10A492246F5F7E0
:10ADC80041FA022C0BDC601C28182021C4F1030274
:10ADD80001E020210322BDE87040F5F7DBBA70BD21
:10ADE800741E0020751E002038B50546002408E0B2
:10ADF800601906F091FE3038C0B2092808D801342D
:10AE0800E4B2044B1B78303B9C42F1DB012038BD97
:10AE1800002038BDDC1D002008B506F07DFE0023AB
:10AE2800C0B2064AD25C824201D1202804D1013343
:10AE3800082BF6D1002008BD012008BD786F020854
:10AE480070B506460D4600240DB12D232B55A019CB
:10AE58000021013406F056FE062CF5D170BD000025
:10AE68002DE9F04F954C964E226896F8009093681D
:10AE780092F8128099B208FB091848F63C108342F0
:10AE880087B01FFA88F80BD18E490878497800F006
:10AE98000700C1F3420101EBC00108EBC10825E03E
:10AEA80048F6FC2083420CD1864908784D7800F09A
:10AEB800070088214843C5F34205773901FB05019E
:10AEC8000DE048F6B46083420BD17E490878497892
:10AED80000F00700C1F3420101EBC0018901884479
:10AEE80004E0B3F5E97F08BF01EB4908764F774DD9
:10AEF800397811F0010F52D147F20902934204D078
:10AF080046F60962934240F04681714A12782A2A2D
:10AF18003CD1704A92F800A00AF1010A0AF0010A2D
:10AF280082F800A0BAF1000F1BD046F609629342DE
:10AF380008D1694B46F695429A809A7842F0020207
:10AF48009A7028E1202110226448F5F723FA4FEA85
:10AF580049139944624B002009EB0301FDF79AFD60
:10AF680019E15D48FDF73CFD236850469A6846F6AE
:10AF780009639A420CBF5B495B49FDF78BFD317849
:10AF88005A4801310222FDF7ABFD04E1552A02D0EF
:10AF9800442A40F000814F4B00221A70FBE05069B0
:10AFA800F5F748FC4A4B834693F800A09946BAF156
:10AFB800450F02D14E4B00221A705046FDF726FE6F
:10AFC80000284FD04B4B5FFA8BFB1A7852450ED1B5
:10AFD8005846FFF799FCFF2804D15846FFF794FC20
:10AFE800FF283FD0444B1A7801321A7015E0DFF879
:10AFF80008A100228AF8002058460593FFF784FC30
:10B00800FF28059B04D09AF8002001328AF8002016
:10B0180099F80020FF281A7024D02168374A4B6914
:10B0280010601B5C886847F20901884213609246E9
:10B0380010D1562B01D0542B0CD13378123BDBB2F4
:10B04800022B07D82B780FFA88F0C01806F064FD99
:10B05800CAF800002B780FFA88F0C018DAF8001048
:10B0680006F050FD99F80030552B17D12368997CCC
:10B078000F2913D92A7808398A42144B01DA083281
:10B0880000E000221A70144B9B7803F00203DBB235
:10B098000BB1FDF7FBFB184B00221A7099F8003032
:10B0A800442B3AD123689A7C0F2A36D92978074B42
:10B0B800072925D90839197024E000BFF81D002098
:10B0C800871E00208D1E0020D71E0020921E002003
:10B0D800C01D0020E21E0020E81E0020F401002010
:10B0E800E3180308F416030836170308F5010020CF
:10B0F800D81D0020DA1D0020061E0020A01E0020FA
:10B10800083A1A70964B9B7803F00203DBB20BB136
:10B11800FDF7BCFB934B00221A7099F80030432BC3
:10B128000DD123680FFA88F05B6919788E4B196086
:10B138002B78C01806F0E6FC8A4B00221A7099F8A2
:10B148000030232B13D122682B78927C013A93424A
:10B158000DDA864A01331370824B00221A70804B35
:10B168009B7803F00203DBB20BB1FDF78FFB99F874
:10B1780000302A2B0FD12B786BB17C4A013B13701E
:10B18800784B00221A70764B9B7803F00203DBB2EF
:10B198000BB1FDF77BFBFEF747FD754A2B7811785D
:10B1A8009246994288BF137012780F32934202DD9B
:10B1B8006F4A0F3B137023684FF0000B93F81290FF
:10B1C800B9F10F0F9ABFC9F120095FFA89F94FF059
:10B1D80010099AF800000FFA88F3181858440593D4
:10B1E80006F09AFC634A02F8090009F101095FFABE
:10B1F80089F9B9F11F0F059B05D821680BF1010BDF
:10B20800897C8B45E5DB397811F0010F17D021686F
:10B218005948897C00780F2900F0800098BFC1F157
:10B228001001C0B294BFC9B2002140B128789AF881
:10B2380000C010305218CCEB00005F211154226876
:10B2480090684AF26A7290420AD14C4B1B78532B91
:10B2580030D106F061FC4A4B187006F057FD29E022
:10B26800B0F5E97F26D1454A1278532A22D11846EB
:10B27800FFF7D2FD8046E8B93378DA00D31A03F134
:10B288001200FFF7B1FD68B1FF2300933D4BCDF8E5
:10B2980004801B78792001330293414604224346F7
:10B2A80006F0B8FC33780021DA00D31A03F1120053
:10B2B800FFF7C6FDDFF8A89099F80230C84603F0FA
:10B2C8000203DBB2002B68D0FDF712FB034688B9F6
:10B2D800226848F6B46192688A420BD046F6096142
:10B2E8008A4214BF2878307809F107016522FDF7F2
:10B2F8001DFB12E0236898F806209B682248B3F5E6
:10B30800E97F0CBF31782978B8F8043001FB0231A5
:10B3180098F8062009B206F010FC23689A7C102AD7
:10B3280013D89B6848F63C1293420BD13B7813F034
:10B33800010F01D010202CE0202107221348F5F737
:10B3480029F82AE0B3F5E97F02D105200B2121E095
:10B3580046F6096293421BD1002010211AE000BF73
:10B36800E81E0020061E0020A01E0020921E0020BD
:10B37800891E0020F4010020F83A0020C01D00209A
:10B38800DC1D0020871E0020EF1E00200402002084
:10B3980000200721094AFDF735FB23689B7C102B09
:10B3A80008D9297806480131022207B0BDE8F04FD4
:10B3B800FDF796BB07B0BDE8F08F00BFE81E002080
:10B3C800F50100202DE9F04F794E8BB033689D6868
:10B3D80093F81290122D01D00B2D09D1754A122D18
:10B3E80092F80090A9F130095FFA89F915D01DE0AB
:10B3F8004BF2E7539D4203D028339D4240F05383DC
:10B408006D482821F5F744F88046002800F04E835F
:10B4180001302821F5F73CF848E39F7B37B9674BA3
:10B42800B846D879FEF70AFC044615E00027B84666
:10B43800FF20FEF703FC4BF2D8339D4204460BD1A4
:10B448004BF2B74006F068FBC0B2099020B15B4BE5
:10B458009B790BB1FDF7E2FB3368594D9A68122AC4
:10B468001AD19B7BC3B12B7813F0010F08D120466A
:10B47800FFF7BAFC534B10B101221A7000E01870A4
:10B488004E4B9B7943B12046FFF7AEFC20B14D4BA4
:10B498001B780BB1FDF7C2FB2978DFF844A111F046
:10B4A800010100F087819AF80030DFF838B11846BA
:10B4B8000793FDF7ABFB079B002800F0B5804249D6
:10B4C800002008704148424A90F800C013609C452B
:10B4D800404940F0898033689B8903F00F03032BB0
:10B4E8001ED13D4BACF1300C18784FF00A0E059088
:10B4F8003A480EFB0C00DDF814E000EB0E0C0EF1E0
:10B50800010E5FFA8EFE70449CF8ADC090F8AD0055
:10B51800C2F800C083F800E0002872D1187070E00B
:10B52800082B2CD12C4BACF130001B7800EB800C95
:10B538000CEB030E294BDFF8A0C013F80E3008936C
:10B548000BB98CF800309CF800E000EB8000059007
:10B5580070440EF1010E5FFA8EFE8CF800E01F4B6E
:10B56800DDF814C01B5C08900CEB0E00DFF86CE0F3
:10B5780013601EF80030002B43D1174811E0072B49
:10B5880011D1BCF1300F10D11348037823B14FF01B
:10B598002B0EC2F800E001E0C2F800C0013303F04E
:10B5A800010303702DE0062B2BD10B78013327E024
:10B5B800F81D0020DC1D002004020020961E00203B
:10B5C800D71E00202F130020AF5A0020DA1D0020BC
:10B5D800A01E0020921E0020061E0020D46E020825
:10B5E800C01D0020DD1D0020DFF898E203709BF8E5
:10B5F80000304FF0010C8EF800C013B10B78634493
:10B608000B7040238BF800300B784B4503D39B4BD2
:10B6180009F1FF30187008781168201806F072FADE
:10B628002B7843F004032B709AF80030232B2FD18A
:10B63800924B09F1FF311A788A4229DA72B93268D5
:10B648004BF2E75192688A4208D028318A4205D0E5
:10B658002046079306F060FA079BC8B118780130B6
:10B66800C0B21870201806F057FA28B9834B202169
:10B678001878201806F046FA814B40221A702B7869
:10B68800804A43F004032B7000238BF800301370BA
:10B698009AF800302A2B10D1784B1A786AB1013AFF
:10B6A8001A70774B40221A702B78764A43F00403BD
:10B6B8002B7000238BF8003013709AF80030432B5E
:10B6C8001FD16E4B1878484505D2201820210793C2
:10B6D80006F018FA079B9BF800203AB91B7809F185
:10B6E800FF32934202DA654A013313702B78644AB9
:10B6F80043F004032B7000231370624A8BF8003068
:10B7080013709BF8003013B15F4A013B13709BF82C
:10B718000030012B0ED1594B1A784A4501D201321B
:10B728001A70584A002313702A7842F004022A70CB
:10B738008BF800302B7803F00402D2B2002A71D0C3
:10B74800524A6FF382031370002111225048F4F714
:10B7580021FE504A494B11781B78994288BF1370D3
:10B7680011780F318B4202DD4A490F3B0B7011787B
:10B7780047481022611806F0E0F94548F5F75AF8ED
:10B7880033684BF2E7519B68C2B28B4202D0283132
:10B798008B4205D122B94048F5F74CF8421CD2B289
:10B7A8000F2A3FD83A4820218018C2F11002F4F736
:10B7B800F1FD37E0DFF8D8B011225846F4F7EAFD7A
:10B7C80033684BF2E7529B68934202D02832934287
:10B7D80009D1214604222E4806F0AFF940463946E1
:10B7E800FFF7DAFA1EE021461022584606F0A5F9BE
:10B7F8005846F5F71FF802462021C2F110025844B6
:10B80800F4F7C8FD21464A46244806F096F9244A2A
:10B818001020937882F8069043F002039370014653
:10B82800FDF7F0F89AF80030532B75D133689A6811
:10B838004BF2D8339A4208D1204606F06DF920B170
:10B848004BF2B740012106F05DF93368DFF838A004
:10B858009B68122B40D12046FFF7C6FA8346002882
:10B8680030D0104BFF2219780F4BF9B90092019193
:10B878001B78782001330293FB3A1FE0921E0020C8
:10B88800AF5A0020061E0020DD1D0020D71E002014
:10B89800741E0020891E0020751E00200F1E002027
:10B8A800081E00202F130020871E00200021009270
:10B8B80001911B787A200133029304220B4606F08B
:10B8C800A9F909E08AF800007D492046FFF7B8FA8F
:10B8D8007C4B83F800B0EFE020464946FDF7E8F8D6
:10B8E800794B0020187033688AF800009B684AF288
:10B8F8007E72934202D10090013005E04BF2FA3299
:10B90800934206D1012300930146024603460DF0F7
:10B918007FFB6E48FDF764F8FEF786F92B7813F085
:10B92800010F17D033684BF2E7529B68934202D05D
:10B938002832934204D140463946FFF72DFA09E0F0
:10B948005F4B634A03F1100153F8040B8B4242F832
:10B95800040BF9D133689A68122A1ED19B7BE3B194
:10B968002046FFF741FAC0B12B7813F0010F14D12C
:10B97800584B9A7922B9DA79574B1B789A420CD0EE
:10B98800564B1A780023303A05E055492A20C91841
:10B9980001330874DBB29342F7DB326893680B2BF0
:10B9A80001D0122B0AD14A4B991D13F8010B2028FC
:10B9B80002D10D3003F8010C8B42F6D192684BF29C
:10B9C800D8339A4214D1434B9B798BB1099878B1FB
:10B9D8004FF0000909EB040006F09EF818B1404B3F
:10B9E8002A224B441A7409F10109B9F1100FF1D157
:10B9F8002B7813F0010F25D03A4B1B7803F0800306
:10BA0800DBB2FBB133689A684BF2E7539A422D4B8D
:10BA180003D04BF20F618A420CD11B7833B9B8F1CD
:10BA2800000F0FD05F3388F801300BE057B15F2269
:10BA3800FA5407E0244A1B78127810339B1A284AD4
:10BA48005F21D154284CA37803F00203DBB2002B0A
:10BA580032D0FCF74DFF2049034628B90878652203
:10BA6800E11DFCF763FF12E03068B4F90430A279F5
:10BA780084680978122C01FB023105D1807B18B942
:10BA88001449C97902FB0131184806F056F83368A1
:10BA98009B68122B10D10820134A01460BB0BDE851
:10BAA800F04FFCF7AFBF0027B84600E0074609F1A2
:10BAB800FF395FFA89F9BBE40BB0BDE8F08F00BF2E
:10BAC800741E0020921E0020891E0020081E0020DF
:10BAD80004020020961E0020871E0020DC1D002086
:10BAE800F4010020F83A0020E81E0020EF1E002094
:10BAF80024282DE9F041144626D16B4B43F63C32FD
:10BB08001B686A4D9B686A4E934206D12B7813F0E6
:10BB1800010F0ED02438674909E04BF20F629342B7
:10BB28000AD12B7813F0010F03D063490020FCF7EA
:10BB3800B1FF2978490800E029783019013102223B
:10BB4800FCF7CEFF0234AAE0E72809D1574B584842
:10BB58001978801801310322FCF7C2FF03349EE0F4
:10BB6800A3282AD1514D2B783F2B15D8104653497D
:10BB7800FCF790FF5148F4F75DFE2A2124184C4841
:10BB8800E4B2F4F785FC002800F08A8029780222C4
:10BB98000131FCF7A5FF83E05901494DC91869181F
:10BBA80001F582411046DF31FCF774FF05F592403C
:10BBB800FE30F4F73FFE241871E0F22821D13B4F04
:10BBC8003B4D3978072605EB0208B1FBF6F14046F4
:10BBD80001310222FCF784FF39782D23B1FBF6F6F8
:10BBE80088F80230F3009E1B8B1B364FDBB207EB45
:10BBF80083031988E21CA9529B78A818837006341D
:10BC08004DE025280BD1304B46F695429A804522C7
:10BC18009A719A78053842F002029A703CE05E28E0
:10BC28000BD1294B46F695529A8045229A719A78FB
:10BC38003E3842F002029A702EE07C280BD1224B4B
:10BC480046F248129A8011229A719A785C3842F02A
:10BC580002029A7020E0EC280BD11B4B46F6D95211
:10BC68009A8045229A719A78CC3842F002029A70EA
:10BC780012E0A7280BD1144B46F6F9529A804522B8
:10BC88009A719A78873842F002029A7004E0E028A4
:10BC980001D1541C03E018B1054B18550134E4B226
:10BCA8002046BDE8F08100BFF81D0020871E002057
:10BCB800F40100204811030806110308C2180308FC
:10BCC800C4CE02083DFB0208E81E002038B50A4B26
:10BCD80046F68A451B78002405FB030507E0074B59
:10BCE80022461978FFF704FF041B2D19044628780B
:10BCF80008B11F2CF3D938BDDB1D0020871E00209A
:10BD080070B5002543F62064204605F005FF064679
:10BD180004F1080005F000FF16F0FF0F06D020F030
:10BD28007F0010F0FF0F01D00135ADB246F23F138E
:10BD38009C4201D00934E7E7284670BD38B5B0F910
:10BD480000500B4C05EBC50505F5785528352846F8
:10BD580005F0E2FEC1B211F0800F07D02388284613
:10BD6800013B01F07F01238005F0CCFE208838BD1F
:10BD7800D61D0020454B2DE9F74F1B88444A044641
:10BD880089461788DFF80C8123B14FF0000A0AE0D2
:10BD98009A4608E00529FBD198F8003043F00403DF
:10BDA80088F8003070E098F8003013F0030F0BD0DB
:10BDB80013F0010F02D0B4F1FF3F05D103F00203E5
:10BDC800DBB21BB1012C01D03F19BFB23BB2B3F1BA
:10BDD800FF3F04D0B3F57A7F08BF002701E040F2A7
:10BDE800E7370FFA87FB0BEBCB0303F5785303F127
:10BDF8002000019305F090FE10F0FF0F019B16D074
:10BE0800B9F1050F09D103F1280005F085FE20F0EE
:10BE18007F0010F0FF0FC6D022E0B9F1000F1FD04D
:10BE280003F1280005F078FE00F07F0618E00AF11B
:10BE3800010AB4F1FF3F1FFA8AFA04D198F80030DA
:10BE480043F0010305E0012C05D198F8003043F0D8
:10BE5800020388F80030BAF57A7F0DD03D46A2E794
:10BE68004E4505D0B9F1000F02D0B9F1050F9AD1AE
:10BE7800BAF1000F05D000E03D46054A2DB2156025
:10BE880002E0034BC3F800B0BDE8FE8FD61D0020CA
:10BE9800A01E0020A41E0020F0B503789BB05A1EF7
:10BEA800D2B2792A0F4600F2C8805E01644AF318BC
:10BEB8009B18644A46F68A461278457806FB02368D
:10BEC800E7213046F4F7E4FA0446F0B930467C211D
:10BED800F4F7DEFA0446C0B930462521F4F7D8FA5B
:10BEE800044690B930462421F4F7D2FA044660B9E2
:10BEF80030464021F4F7CCFA044630B93046F921EF
:10BF0800F4F7C6FA0446002876D0A41B0FB14E48B1
:10BF180000E04E4831462246A619F4F711FD304696
:10BF2800E721F4F7B5FA30B128466946652246F6A6
:10BF3800D953FCF7FBFC30467C21F4F7A9FA50B141
:10BF4800691EC9B201EB011101F5C24168464831C9
:10BF5800112205F0F2FD30462521F4F799FA38B19F
:10BF6800681EC0B26946652246F69543FCF7DEFCBA
:10BF78003046F921F4F78CFA38B1681EC0B2694628
:10BF8800652246F69553FCF7D1FC30464021F4F77C
:10BF98007FFA50B1691EC9B201EB011101F5E84100
:10BFA80068463B31112205F0C8FD30462421F4F7DC
:10BFB8006FFA50B10FB1244800E02448001929460F
:10BFC8000222FCF78DFD02340BE00FB11E4800E0A1
:10BFD8001E4800196946F4F7CFFB6846F4F72AFCB7
:10BFE8000419002F29D01A4A9378141943F0020330
:10BFF80093700023E37116E03046F4F71BFC054606
:10C008001FB9124831462A4615E0102810DD2A4685
:10C018000D483146F4F794FC0D4A9378551943F0CE
:10C0280002039370EC7110200146FCF7EBFC04E06E
:10C03800084831461022F4F783FC1BB0F0BD00BF5E
:10C04800A7000308DB1D0020EF1E00206E33002030
:10C05800E81E0020040200200C4B1B7813F001029C
:10C0680002D000200A4905E003F00200C0B218B16E
:10C0780008491046FCF70EBD03F00403DBB20BB110
:10C088000549F7E705480121FFF706BFA41E002070
:10C0980080D602085FD60208A1D60208D91E002061
:10C0A80070B5124D124C00201249FCF703FC2846CB
:10C0B800A1780222FCF714FDE81CE1780222FCF7C3
:10C0C8000FFD05F1080021790222FCF709FD05F1B1
:10C0D8000B0061790222FCF703FDA17905F10E003E
:10C0E8000222BDE87040FCF7FBBC00BFF401002051
:10C0F800D91E0020E56F02082DE9F341504F514C3D
:10C108003B689D7C237813F0010F2FD1022243F660
:10C118001E610DF1060005F010FD4B4EBDF806300E
:10C128004FF0FF3033602946FFF724FE237843F0B1
:10C1380001032370454B1B7813F0030F14D1B6F994
:10C148000010434801EBC10101F578512031092263
:10C1580005F0F3FC3F4B1B881BB13046FFF7EEFDA3
:10C1680010B90020FAF78CF8FFF79AFF3A4E3378A7
:10C17800552B0DD1DFF8D4803848FCF731FC98F8FE
:10C1880000304FF0FF306FF3410388F800300DE0C6
:10C19800442B2BD1DFF8B4803048FCF721FC98F809
:10C1A800003001206FF3000388F800302946FFF7BC
:10C1B800E1FD98F8003013F0030F15D1224D244803
:10C1C800B5F90010092201EBC10101F578512031C0
:10C1D80005F0B3FC1F4B1B881BB12846FFF7AEFDCB
:10C1E80010B90020FAF74CF8FFF75AFFFFF734FFB1
:10C1F8003378232B22D1154B184E1A7802F0FC0203
:10C208006FF382021A70FCF709FDB3786FF34103EC
:10C21800B370134B1D7835B9FCF738FB3046FCF783
:10C22800DFFB3D600AE02278013DEDB242F00602F4
:10C2380022701D700B4B53F825303B60BDE8FC8124
:10C24800F81D0020D71E0020A01E0020A41E0020DC
:10C25800D91E0020D61D0020C01D0020E81E002089
:10C26800B71E0020C41E00202DE9F0411646104AD2
:10C278000F4653780E21C3F342034B43117803F55D
:10C288000843CC330B4D01F00701044603EB410191
:10C29800022205F052FCE81921780222FCF720FC62
:10C2A8006178A8190222BDE8F041FCF719BC00BF6B
:10C2B8008D1E0020F4010020044B02225978044B03
:10C2C800C1F3420118180131FCF70ABC8D1E002089
:10C2D800F401002010B5074B074C1B78074A03F000
:10C2E800070304EB83031C88111814529B788B7086
:10C2F80010BD00BF8D1E00203DFB0208F401002088
:10C30800084B1B789B0902D0012B06D102E01020B4
:10C31800054904E01020054901E005491020FCF713
:10C32800B9BB00BF8D1E002022E3020843E30208C8
:10C3380064E302082DE9F041DFF868800F4698F8B9
:10C348000010174DC1F382010446164605F1080096
:10C3580001310222FCF7C4FB98F80010042201F016
:10C368001C0101F51C41B431204605F0E6FBE81933
:10C3780021780222FCF7B4FBF81C28186178022205
:10C38800FCF7AEFBA819A1780222FCF7A9FBF01C68
:10C39800E17828180222BDE8F041FCF7A1BB00BFF4
:10C3A800F4010020D91D0020064B1B7803F0800300
:10C3B800DBB233B1435C04482021C0180222F3F7F2
:10C3C800E9BF7047F83A0020F40100202DE9F7434F
:10C3D800654D664C2B6821789B68022203EB41016E
:10C3E8000DF1060005F0A9FB2B68A9469A6843F6EB
:10C3F800F4239A4208D100205D49FCF74BFBBDF8B5
:10C4080006804FF4B46303E0BDF806804FF461631F
:10C41800B8FBF3F103FB11883C221FFA88F8B8FB3C
:10C42800F2F302FB1388CFB2DEB20222514839463A
:10C43800FCF756FB5FFA88F802224F483146FCF7B2
:10C448004FFB02224D484146FCF74AFB4C4B1B78F8
:10C4580013F0010F6ED04B4B4B4D1878232804D1A5
:10C468002B78012B62D8013305E02A2805D12B78D7
:10C47800002B5BD0013B2B7058E0A0F13003DBB2FE
:10C48800092B01D943284BD12B7873B9D9F800303F
:10C4980039B29A6843F6F4239A4201D10A2200E09D
:10C4A8001122FDF7E1FBC7B216E0012B0ED1D9F836
:10C4B800003031B29A6843F6F4239A4201D1172228
:10C4C80000E03B22FDF7D0FBC6B205E041463B2227
:10C4D800FDF7CAFB5FFA80F8D9F800309A6843F68E
:10C4E800F4239A4209D13C235E434FF4B46303FB1F
:10C4F8000767B844ADF8068006E03846314642463C
:10C508000FF06FFEADF80600D9F8003020789B6870
:10C518000DF1060103EB4000022205F008FB05E0DF
:10C52800532803D100232B70FDF77EFB1748297889
:10C53800FFF73AFFD9F800309A6843F6F4239A4295
:10C5480010D02078124965220023FCF7EFF9052066
:10C558000B21104AFCF756FA21780F4801310222C4
:10C56800FCF7BEFABDE8FE83F81D0020871E0020F8
:10C5780047150308040200200A02002012020020C6
:10C58800D71E0020C01D0020921E0020F66F020852
:10C59800EF1E0020E81E0020F501002073B5994B1E
:10C5A800994D1A7812F0010F05D12A7812F0380245
:10C5B80004BF2A706A701A78924E42F001021A700B
:10C5C8002B78914C13F038023ED1904909785529BF
:10C5D80004D113F0070F2FD0DA1D0AE044290CD13B
:10C5E80003F0070201323D3992FBF1F1C800411A0C
:10C5F800521A62F3020323701EE053290AD1C3F3CF
:10C60800C201013161F3C5032370637862F3430308
:10C61800637011E023290FD1FCF700FB33787C4AC3
:10C6280043F0060333701378013BDBB21370794A89
:10C6380052F82320784B1A6000207849FCF72AFA30
:10C648001C20FFF747FEDBE0082A2CD174490020A4
:10C65800FCF720FA0620FFF72FFE0C20FFF73AFE22
:10C668001521182201A8FFF7FFFD684B1B78552BF1
:10C6780006D1637803F0FE03C3F34202013A07E0F0
:10C68800442B09D1637803F0FE03C3F3420201325D
:10C6980062F343036370B3E0532B28D0232B40F09D
:10C6A800AF802378A6E0102A51D15D490020FCF71D
:10C6B800F1F90620FFF700FE0C20FFF70BFE15210D
:10C6C800182201A8FFF7D0FD6178564801F0010152
:10C6D800FFF76AFE4D4B1878232801D02A2804D189
:10C6E8006378DA4362F30003D4E7532804D123784C
:10C6F800C3F3C202013280E0A0F13003DBB2092BA0
:10C7080001D943287CD16B7802AA03F001033B21AD
:10C71800D41883F001024B43172606FB023214F8A3
:10C72800041CFDF7A1FA04F8040C6B780E22C3F37D
:10C7380042035343287803F50843CC3300F007003D
:10C7480003EB400001A90C3A05F0F1F958E0182A6A
:10C758004DD133490020FCF79DF90620FFF7ACFDC9
:10C768000C20FFF7B7FDFFF7CBFD284B1B78552BA7
:10C7780007D1237813F0C00F42D0C3F38112013AD6
:10C7880006E0442B07D123789A09012A38DC0132C4
:10C7980062F3871333E0232B04D12378C3F3C20257
:10C7A800023A2AE0532B2BD1FCF738FA33781E4A89
:10C7B80043F006033370164B1648197840F82120C9
:10C7C800013119702378C3F3C201013161F3C50344
:10C7D800C3F381112370104B11B1012904D101E079
:10C7E8001C3202E0114A00E0114A1A6008E0114ABE
:10C7F80000211170C3F3C202013A62F3C50323702A
:10C808007CBD00BFD71E00208D1E0020C01D00204B
:10C81800B71E0020C41E0020F81D0020E0E2020818
:10C8280001E30208F96F0208FC6F0208347002087D
:10C8380050700208921E002073B5494B494D1A7872
:10C8480012F0010F04D12A7812F0030208BF2A70EF
:10C858001A78434E42F001021A702B78414C13F0BB
:10C8680003022ED1404A1278552A03D1C3F382021B
:10C87800013A04E0442A06D1C3F38202013262F38A
:10C888008403237017E0532A03D15A1C62F301036F
:10C89800F7E7232A0FD1FCF7C1F93378334A43F07D
:10C8A800060333701378013BDBB21370304A52F839
:10C8B8002320304B1A6001A810211B22FFF73AFDF4
:10C8C8004CE0012A4AD101A810211A32FFF732FDA3
:10C8D800254B1878232804D12378C3F34112013259
:10C8E80005E02A2807D12378C3F34112013A62F3FD
:10C8F800461323702CE0532804D12378DA1C62F302
:10C908000103F6E7A0F13003DBB2092B01D9432874
:10C918001ED12B7802AAC3F34113D4180C215A1C38
:10C9280003F001034B4302F001021F2614F8041C14
:10C9380006FB0232FDF798F904F8040C287801A9DF
:10C9480000F01C0000F51C40B430042205F0EFF89C
:10C9580029780948C1F34111FFF726FD7CBD00BFC6
:10C96800D71E0020D91D0020C01D0020B71E0020A2
:10C97800C41E0020F81D00206C700208064B1B78AE
:10C9880003F08003DBB233B1435C04482021C018B4
:10C998000322F3F7FFBC7047F83A0020F4010020A7
:10C9A8004328F8B504460D46174606D1104B002615
:10C9B8001A786FF3C3021A7000E00E462046FCF79F
:10C9C80025F990B10A4B303C1A780A2602F0080182
:10C9D800C9B2002918BF002506FB05466FF3C3023C
:10C9E80036B21A70BE42A8BF3E4630B2F8BD00BF8C
:10C9F800D71E00202DE9F3416E4F6F4E3B7843F070
:10CA080001033B70347844B94BF22F4005F084F8A9
:10CA18006A4B6B491860204617E0012C02D10020B0
:10CA2800684912E0022C02D1002067490DE0032C6E
:10CA380002D10020654908E0042C02D10020644995
:10CA480003E0052C03D163490020FCF723F8317873
:10CA5800D9B9614B1B78312B01D1013101E0302B61
:10CA680005D1564B4BF22F40196005F04BF85B4B44
:10CA78001A785B4B02F08002D2B20AB1202202E09F
:10CA88004E4A12683032DA776EE001290BD002295B
:10CA98000CD003290DD004290ED04BF22B450529C3
:10CAA80018BF00250AE04BF21B4507E04BF21F4573
:10CAB80004E04BF2234501E04BF2274529460422C6
:10CAC80001A805F03AF8474B474A03F1100153F81B
:10CAD800040B8B4242F8040BF9D1032243489DF81A
:10CAE8000410FBF7FDFF032241489DF80510FBF7F2
:10CAF800F7FF03223F489DF80610FBF7F1FF3E4879
:10CB080003229DF80710FBF7EBFF334B3B4C1878DB
:10CB1800232804D12378022B22D8013304E02A28C1
:10CB280004D12378E3B1013B237019E0A0F130036D
:10CB3800DBB2092B01D9432812D194F8008002AA4C
:10CB4800904418F8041CFF22FFF72AFF08F8040C89
:10CB5800207802AA131813F8041C281804F0D2FF2E
:10CB680027482178FFF70AFF1B4B1B78532B1FD14F
:10CB7800224B00221A7033780133DBB2062B337054
:10CB880004D0012B14D10D4B1B688BB1FDF74CF869
:10CB9800002333703B781B4A43F006033B7013783D
:10CBA800013BDBB21370184A52F82320174B1A6066
:10CBB800BDE8FC81D71E0020871E0020A01E002093
:10CBC800CD2E0308F62F0308173003083830030862
:10CBD800593003087A300308C01D0020F83A0020B5
:10CBE800F40100205C57030804020020050200201D
:10CBF800090200200D02002011020020921E0020D0
:10CC080070700208B71E0020C41E0020F81D002006
:10CC180070B5174C0D460646002120464FF4C172E8
:10CC2800F3F7B8FBFF2D0AD1B10001F5D841204632
:10CC38009531042204F081FF23789BB970BDFE2D45
:10CC480001D1173E02E0FD2D02D10136267009E020
:10CC5800B60006F5D8409530401904F05DFFC0B223
:10CC6800207020B10248BDE8704018F0E9BB70BDE3
:10CC7800FC2000202DE9F04118F014FC60B11020D0
:10CC88008F49FBF707FF8F4B1B78432B40F0EF8151
:10CC9800BDE8F04118F028BC18F016FC002826D092
:10CCA800894C23786BB110208849FBF7F3FE88483C
:10CCB8002D211030F3F7ECFB002800F0D881217803
:10CCC80010E010208349FBF7E5FE81482D21103044
:10CCD800F3F7DEFB0446002800F0C98118F00CFCCD
:10CCE800014620468222BDE8F041FBF7F9BE7A4CA6
:10CCF80043F6CC2223689B68934250D0774E744DFC
:10CD0800307803EB800004F007FF032201467448E3
:10CD1800FBF7E6FE2368986846F6F95398422BD04D
:10CD2800203B984228D03378013000EB830004F090
:10CD3800F3FE0322014605F11500FBF7D1FE236837
:10CD480030789B68023303EB800004F0E5FE032291
:10CD5800014605F11900FBF7C3FE236830789B688C
:10CD6800033303EB800004F0D7FE0322014605F1EC
:10CD78001D00FBF7B5FE0EE02D2103225948F3F7FD
:10CD880009FB2D2103225848F3F704FB57482D21AE
:10CD98000322F3F7FFFA20232B772B762B75544BBE
:10CDA8001B7813F0010F00F0BD80236843F6CC22F6
:10CDB8009B68444D934261D04E4E484F3278387844
:10CDC800D31803EB800004F0A7FE4B4B0146186014
:10CDD80028789846A0F13002D2B2092A01D943280E
:10CDE8000FD109B2BA22FCF73FFF236832789B685B
:10CDF8000146C8F800003878D31803EB800004F027
:10CE080081FE2B782A2B04D1337813B1394A013BA0
:10CE180013702B78232B0ED13378022B0BD8226872
:10CE280046F6D95192688A4205D020318A4202D00A
:10CE3800304A013313702B78552B01D0442B0FD176
:10CE4800236831789B68A3F5D843B3F1950248BFAE
:10CE5800A3F192023B7803EBA202D0B2FFF7D8FE0F
:10CE6800264B1B7803F08003DBB23BB13278184BBA
:10CE780003EB820320225A749A74DA742B78532BAA
:10CE880006D023689A6843F6CC239A4240F0EF8094
:10CE9800FBF7C4FE236846F695429B68934203D18C
:10CEA8000E4B0220197806E046F6F952934227D134
:10CEB8000A4B002019780131BDE8F0410CF07CB82C
:10CEC800FC170308C01D0020F0150020D316030826
:10CED800F40100201D180308F81D0020871E0020FB
:10CEE80005020020090200200D0200201102002086
:10CEF800D71E0020921E0020A01E0020F83A002015
:10CF080046F6D952934204D15A4B01201978091890
:10CF1800D2E746F69552934240F0A980554B03203C
:10CF28001978C8E723684AF27E729B6893423FD11A
:10CF3800504E10205049FBF7ADFD31784F4D01EBB5
:10CF4800011101F5264101F5BF711022284604F0B0
:10CF5800F4FD2B4605F110012A461078474F78B9A1
:10CF68004749FBF797FD3846E721F3F791FA78B17F
:10CF78003178401B381801310322FBF7B1FD07E077
:10CF880013F8010B10B9203003F8010C8B42E4D1DF
:10CF98003C4D2B782A2B03D13078FD21FFF738FE42
:10CFA8002B78432B63D1307823680130C0B259E025
:10CFB80043F6CC229342334E1AD010203249FBF765
:10CFC80069FD33782A2B52D1304B1B689B68A3F537
:10CFD800D843B3F1950248BFA3F19202254BFF2134
:10CFE8001B7803EBA202D0B2BDE8F041FFF710BEF8
:10CFF8003378204D552B04D12B78142B01D1033BCA
:10D008002B703378442B05D12B78122B02D1194B76
:10D0180015221A702B78DFF878805901C918414415
:10D0280001F5944100201F31FBF734FD08F59241CA
:10D03800102017312F78FBF72DFD3378112F8CBF77
:10D04800032700272A2B05D12878FE21C01BC0B250
:10D05800FFF7DEFD3378432B09D12B78173BDF1B15
:10D068002368F8B2997CBDE8F04118F003BABDE82E
:10D07800F08100BF871E0020DB170308F4010020A1
:10D08800EBF80208C01D002099170308F81D0020BE
:10D09800C4CE020810B50E4B1B78452B17D10D4B8B
:10D0A8001A7842F006021A700B4A1378032B0ED82E
:10D0B8000A490B4C086844F823000133137083684D
:10D0C8000B60FBF7EFFBBDE81040FBF7A7BD10BDF9
:10D0D800C01D0020D71E0020B71E0020F81D00200C
:10D0E800C41E002010B50C4B04462146D8790FF019
:10D0F8003CF860B1204655210EF096FE48B1204616
:10D108000EF028FFD0F1010038BF002010BD02202A
:10D1180010BD022010BD00BF961E002008B50FF0FC
:10D1280013F8C0B208BD00002DE9F047634B644C0A
:10D138001A78994612F0010F624D65D02078FFF7F2
:10D14800D1FF614A2B181178604F93F8A031604ED7
:10D1580044293870336090460AD12D2B08D038B94D
:10D1680095F8A11101233B7031602078FFF7D6FFB5
:10D1780098F80030552B10D133682D2B0DD03B7803
:10D188005BB1013B514ADBB21370EB1893F8A01165
:10D198004F4B20781960FFF7C1FF98F80030232B18
:10D1A80019D14C4B20781B689B7C013B984212DAC2
:10D1B800434B0130C0B21870FFF794FF387028183D
:10D1C80090F8A0313360444B9B7803F00203DBB244
:10D1D8000BB1FBF75BFB98F800302A2B14D12078B1
:10D1E80090B1374B0138C0B21870FFF77BFF387029
:10D1F800281890F8A0313360374B9B7803F002036E
:10D20800DBB20BB1FBF742FB344EFCF70DFD237884
:10D2180032789A4288BF337032780F32934202DDF7
:10D228002E4A0F3B1370DFF8C48000273078381877
:10D23800C0B2FFF757FF281890F8A0310137102F18
:10D2480008F8013F07D0254B1A78224BBA181B68FB
:10D258009B7C9A42EADB99F8003013F0010F13D057
:10D268001F4B1A781F4B02F08002D2B22AB12278E3
:10D2780031781032521A5F2105E022783178103265
:10D28800521A134909689954134DAB7803F00203F5
:10D29800DBB25BB12078E91D652246F69553FBF7B2
:10D2A80045FB05200B212A46FBF7ACFB21780E48ED
:10D2B80001310222BDE8F047FBF712BCD71E00205F
:10D2C800921E0020D46E0208C01D0020D81D002028
:10D2D800A01E0020F81D0020E81E0020891E002046
:10D2E800F83A0020F4010020F50100200302002094
:10D2F80038B5054600240123A3402A78E0B29A42B3
:10D3080005D10E49102246F6D953FBF70FFB01341D
:10D31800082CF0D1083C0A4BE0B2E3189A782B7835
:10D32800934206D12BB10549102246F6F953FBF773
:10D33800FDFA0134042CEED138BD00BFC21D002017
:10D34800961E00202DE9F041074610460D4614466A
:10D35800F3F770FAC3B28046B3B1AB4214D80B4EA0
:10D3680020212A46F019F3F715F82046F3F762FA58
:10D37800C8EB05056D08EDB2EF1902462146F01914
:10D38800BDE8F041F2F75EBFBDE8F081F40100208E
:10D39800F0B5134B0C781A1895781F46E5B10023A1
:10D3A8003A1892781A4112F0010F4FF001020BD08F
:10D3B800AC420E7803D09A4042EA060602E09A4050
:10D3C80026EA02060E7004E09A400E7826EA020267
:10D3D8000A700133082BE3D10B7803B90C70F0BD48
:10D3E800961E0020312200230178194111F0010F07
:10D3F80002D00449C9180A7501330132082BD2B288
:10D40800F2D17047F401002070B57B4B044631B16E
:10D418001B78532B40F0EF80533B037070BD1A7894
:10D42800302A34D1754A53785BB1754B75491B78EE
:10D43800182000FB03135B7913F0100F01D00123B0
:10D448005370714B20781978014012D09278002AD5
:10D4580040F0D1801978114111F0010F05D0012158
:10D468009140207820EA010121700132082AF1D187
:10D4780041E01A780A4112F0010F04D001228A40D3
:10D4880020780243227001310829F2D133E0A2F159
:10D498003101C9B2072938D858494A785AB1584A87
:10D4A80058481278182505FB0202527912F0100F1D
:10D4B80001D001224A701B78534A313B1278DBB203
:10D4C8001A4112F0010F00F09680227852FA03F008
:10D4D80010F0010F09D08978002940F08C800131C3
:10D4E80011FA03F322EA030204E0012111FA03F31B
:10D4F80043EA02022270002112224448F2F74AFF4E
:10D508002046BDE87040FFF7F3BE132A0CD0552A19
:10D5180017D13B4B3B4A1B78182101FB03235B794E
:10D5280013F0200F03D170BD344B01225A70002034
:10D538002146FFF72DFF344B9B78002B5BD0002052
:10D5480051E0142A0CD02A2A17D12D4B2D4A1B78CA
:10D55800182101FB03235B7913F0200F03D170BD61
:10D56800264B01225A7001202146FFF711FF264B56
:10D57800DB78002B3FD0012035E0152A0CD0232A78
:10D5880017D11F4B1F4A1B78182101FB03235B7916
:10D5980013F0200F03D170BD184B01225A700220DE
:10D5A8002146FFF7F5FE184B1B79002B23D00220EC
:10D5B80019E0162A0CD0442A1DD1114B114A1B78A8
:10D5C800182101FB03235B7913F0200F03D170BDF1
:10D5D8000A4B01225A7003202146FFF7D9FE0A4B55
:10D5E8005B7943B103200949102246F6F953BDE897
:10D5F8007040FBF79BB970BDC01D00202F130020A1
:10D608008A1E0020843C0020961E0020C21D002097
:10D618002DE9F04F87B09DF840408146072C0D4614
:10D6280005929A4637D1073C27462B78234113F0B9
:10D63800010F2CD0012623B24FF00008029351208D
:10D648003146324633460096CDF8048004F0E2FABB
:10D658001B204146A2194346CDF80080F5F74EF845
:10D6680037B9112039463A4633460097F5F746F858
:10D67800534B204613F8242001276FF3000203F8C8
:10D6880024201199F5F7C4FE2046F6F7CBF80134AB
:10D69800082CCAD10DE2012C03780CD10BB90B78F8
:10D6A80023B3FF2300930021464B01911B780C20E4
:10D6B8000133029316E0022C09D10BB90B78ABB1F8
:10D6C8000021FF2300930191029134200AE0062CE7
:10D6D8000CD10BB90B784BB10021FF2300930191BA
:10D6E8000291652004220B4604F094FABAF1010F66
:10D6F80099F800302BD13BB1334B0020D979024641
:10D7080053460090F4F7FAFF2B783BB12E4B0120DB
:10D71800D979002203460092F4F7F0FF0020F5F7CC
:10D7280069FE99F80030002B5BD0284B1978002946
:10D7380057D1274BDB78002B53D0FF2300933A2097
:10D7480001220B460191029104F064FA49E063B1A9
:10D75800052C4FF0000102D100910F2001E000914B
:10D768000B200A460123F4F7C9FF2B7883B1052C57
:10D778004FF0000106D110200A4601230091F4F76A
:10D78800BDFF12E00C200A4601230091F4F7B6FF12
:10D79800022C25D0032C01D10E4B02E0042C02D11F
:10D7A8000D4B1F781DE0052C01D10C4BF9E7012C1E
:10D7B80001D1044BF5E7062C0CBFFF27002710E02A
:10D7C800361A0020171B0020961E0020241A00205D
:10D7D8002F130020B020002087590020033F00208D
:10D7E800FF2799F80030002B00F0B580934B944E3A
:10D7F8001A78984602F02002D2B262B1317811F05C
:10D80800010108D1FF230093282001220B46019132
:10D81800029104F0FFF998F8003003F01003DBB22E
:10D828006BB1317801F00201C9B241B9FF2300930D
:10D83800292001220B460191029104F0EBF998F896
:10D84800033013F0010F0DD0317801F00401C9B293
:10D8580041B9FF2300932A2001220B46019102912E
:10D8680004F0D8F998F8033003F00203DBB26BB187
:10D87800317801F00801C9B241B9FF2300932B2088
:10D8880001220B460191029104F0C4F998F8033083
:10D8980003F00403DBB26BB1317801F01001C9B2B7
:10D8A80041B9FF2300932C2001220B4601910291DC
:10D8B80004F0B0F998F8033003F00803DBB26BB159
:10D8C800317801F02001C9B241B9FF2300932D201E
:10D8D80001220B460191029104F09CF911F0C4F861
:10D8E80068B1317801F04001C9B241B9FF23009312
:10D8F800492001220B460191029104F08BF998F816
:10D90800033003F04003DBB26BB1317801F08001E2
:10D91800C9B241B9FF2300934E2001220B46019161
:10D92800029104F077F9767816F0010613D145488C
:10D93800314617F00EF858B1FF230093731C0021ED
:10D948001BB20293752001220B46019104F062F983
:10D958000136702EEBD1119B3B4A19783B4B51B1E4
:10D9680099F8001011702A781A702B780BB154208E
:10D9780005E0522003E011702A7853201A7004F051
:10D9880017FD119B00261A78314B1A7099F8003050
:10D99800334113F0010F2DD03146059816F0D9FF09
:10D9A8000122014628B933B2019000920293104631
:10D9B80005E0002133B200920191029324200B4626
:10D9C80004F028F9BAF1010F05D1224B8020DA7949
:10D9D8000521013208E0022C07F1010202D1802062
:10D9E800072101E0802006213346F6F757FA304632
:10D9F800F5F7ECFE2B78334113F0010F55D00021D9
:10DA08004FF0010B33B2029302205A460B46CDF871
:10DA180000B0019104F0FEF8DA45DFF83C801DD132
:10DA280018F8263013EA0B0332D10A4A0520D179B7
:10DA38000093594406EB0B0228E000BFF83A002097
:10DA4800091C0020141A0020821A0020831A0020C2
:10DA5800271C0020961E0020361A002018F82630B1
:10DA680013F0010314D1022C0CD1134B1B7803F0D3
:10DA78002403042B04BF114B83F800B00023009348
:10DA8800072001E000930620791C721CF4F736FE8B
:10DA980011993046F5F7BCFC3046F5F7C3FE18F887
:10DAA80026306FF3000308F826300136082E7FF47D
:10DAB8006DAF07B0BDE8F08F301C002028130020A0
:10DAC8002DE9F04180460E46174646F2BF75002400
:10DAD8003846214616F03DFF88B1294608220B48F2
:10DAE80004F02BF80948414616F0E0FE074816F006
:10DAF80003FF20B90123A340327813433370013464
:10DB08000835082CE4D1BDE8F08100BF1F1C0020B7
:10DB18002DE9F04387B08046894604A847F2E91109
:10DB2800082204F00AF8002440462146E7B216F01D
:10DB380010FF002843D03846F4F71AFB0025661C6E
:10DB48000246314611202B460095F4F7D7FD0123F4
:10DB580021462A460420FF080095F4F7CFFD4BF232
:10DB6800DF50381803F0D8FF04F00703C1B2194199
:10DB780011F001014FF002024FF001030AD00092A8
:10DB8800019336B27720294692182B46029604F064
:10DB980041F814E00092019336B2232004220B4688
:10DBA800029604F037F8B9F1000F08D004A821460E
:10DBB80016F0CFFE18B10548214616F0B4FE013420
:10DBC800402CB1D107B0BDE8F08300BF5F1A002038
:10DBD8002DE9F74F174698463B7805460C469DF8C1
:10DBE80030909DF834B09DF83820DFF8B8A043B1E4
:10DBF80002EA03033B7009789AF800208A18D31ABE
:10DC08000370237883B122482146F5F7B7FD2149EF
:10DC18001F4816F04BFE1E480121FFF779FF1C48EC
:10DC280041462246FFF74CFF1B4B00261E70297801
:10DC380043F6FB2003F066FF494646F2CD6003F049
:10DC480061FF204639464A46F5F78AFB134B4246A0
:10DC58001E7139464B462046CDF800B00195FFF7B6
:10DC6800D7FC2846F8F744FB2B780D480D498AF86D
:10DC78000030F5F783FD11F037FF88F800603E703B
:10DC880026702E7003B0BDE8F04F04F09BBA00BFB9
:10DC9800281C00207A1A0020D41E00202F130020F0
:10DCA8000B1C0020241A002010B50B4B0B4C02460D
:10DCB80003CB206061600A48114616F018FE214621
:10DCC800074816F0F3FD064816F016FED0F10100DD
:10DCD80038BF002010BD00BFB02E0020151C00204A
:10DCE8001F1C002010B50A4C637C4BB10020094969
:10DCF800FAF7D0FE084B1B78432B01D1433B6374E2
:10DD0800607C20B90549BDE81040FAF7C3BE10BDD4
:10DD1800C21D00202DF90208C01D00200CF90208C0
:10DD2800034B1A7801321A7001230370704700BF41
:10DD3800D41E002010B50C48FAF752FE0B4A0024F6
:10DD480014700B4A0B4B14700B4A5C7114700B4A1D
:10DD58001C7114700A4A5C7014700A4A1470FAF73D
:10DD68005DFF094B1C6010BDE81E0020961E0020B8
:10DD7800C11D00202F130020D81E0020E51E002002
:10DD8800FC1D0020D41E0020F81D00202DE9F04FB6
:10DD9800974B984E93F800903368DFF8A8829C7CE4
:10DDA800954BF0221A7098F800308BB00D2B354641
:10DDB80047463DD1914B93F805C0BCF1010F02D9FC
:10DDC80000208F492FE01AD100245C718D4A8E4BB8
:10DDD8008E498F488F4D04701C7014700C70CDF8EC
:10DDE80000C001942D780295FFF7F2FEFAF716FFAE
:10DDF800894834600BB0BDE8F04FFAF7F1BD8748A9
:10DE08008249F5F7BBFC864B864A03CB864B1060EC
:10DE18001B785160532B5FD198F800308349013348
:10DE280088F8003000200BB0BDE8F04FFAF732BE9A
:10DE3800092B0FD17C4B1B78532B3DD17C4B0022F7
:10DE48001A700D2388F800307A4B1A7842F00602CF
:10DE58001A7089E20E2B37D1734B1B78532B2BD1B9
:10DE680075496E4816F022FD6C48FFF71DFF044601
:10DE780040B198F800300522013B88F800305F4B2C
:10DE88005A7171E2082246F2CE61664803F055FEE7
:10DE980064496A4816F02BFD012300935D4B0194F9
:10DEA8001B785B4802935949564A574BFFF790FE37
:10DEB800FAF7B4FE346057E2232B40F055820BB0DA
:10DEC800BDE8F04FFFF736BF33B95D4B1A781AB982
:10DED80001321A7011F008FE631E48BFA31DDB1043
:10DEE800013303FB09F91FFA89F909F5CC46A9F5AD
:10DEF8009449A9F121094F4BCDF81C901A78CE36D8
:10DF080012F0010F4A4C00F02081474B1A789946CD
:10DF1800432A40F0C9803B780D2B40F0C5803F482C
:10DF2800217816F016FD002800F0BE803D482178C3
:10DF380016F00FFD002840F0B780079920780FFAF7
:10DF480081FB0BEBD00003F0E7FD23784FF0010ACB
:10DF580003F007020AFA02FADFF8EC805FFA8AFA9D
:10DF680010EA0A0FC8F8000027D0244BDB78002BF2
:10DF780040F09A80274BD879F8F718F9002800F074
:10DF88009380D8F80010CAF1FF0A20780AEA010144
:10DF9800C8F800100BEBD00003F0B4FD20780FFA9E
:10DFA80086FB0BEBD00003F0B7FD00EA0A012078EE
:10DFB800C8F800100BEBD00061E032B202EBD300DE
:10DFC800059203F0A9FD10EA0A0FC8F800003DD138
:10DFD80040EA0A01059B2078C8F8001003EBD0003E
:10DFE80003F090FD2178154816F09DFC5CE000BF19
:10DFF800871E0020F81D0020E31E00202F1300209C
:10E00800D2F90208D81E0020C11D0020E51E0020FC
:10E01800FC1D0020961E0020E81E0020281C002061
:10E02800B02E00200C1A0020C01D002098FA02080B
:10E03800921E0020D71E00206F1A00207A1A002096
:10E0480070140020D41E0020A01E0020924BDB7804
:10E0580023B9924BD879F8F7A9F8B8B92078DDF840
:10E0680014C0CAF1FF0A0CEBD00003F055FD8C4A2E
:10E0780000EA0A01059B2078116003EBD00003F049
:10E0880041FD2178874816F059FC0DE020780BEB0C
:10E09800D00003F041FD40EA0A012078C8F80010DA
:10E0A8000BEBD00003F02EFD99F80030232B10D194
:10E0B8002A682378927C013A93420ADA7A4A013331
:10E0C80013707A4B9B7803F00203DBB20BB1FAF7BB
:10E0D800DDFB99F800302A2B0CD1237853B1724A12
:10E0E800013B1370714B9B7803F00203DBB20BB159
:10E0F800FAF7CCFB99F80030552B12D12968227811
:10E10800897C694B08398A4201DA083200E000222A
:10E118001A70664B9B7803F00203DBB20BB1FAF777
:10E12800B5FB99F80030442B0FD122785E4B072AB3
:10E138009CBF2A68927C083A1A705C4B9B7803F063
:10E148000203DBB20BB1FAF7A1FBFBF76DFD584AEE
:10E15800237811789246994288BF137012780F324B
:10E16800934202DD524A0F3B13702B684FF0000BAD
:10E1780093F81280CDF818B0B8F10F0F9ABFC8F114
:10E1880020085FFA88F84FF0100839784FFA8BF3B7
:10E198000D2905D19AF800209B18DB10454A04E0A8
:10E1A8009AF800209B18444ADB10D35C9AF80020A8
:10E1B80005934FFA8BF39A180D2902F007094FEAD5
:10E1C800E20202D13D49895C0691DDF81CC0049346
:10E1D8000FFA8CF0101803F09FFCC0B2049B089053
:10E1E8009AF8000032B2181802EBE00003F094FC31
:10E1F80039789AF80020049BC0B209919A1846E031
:10E20800059BDDF824C043FA09F12D4B01F001010B
:10E2180000290CBFA521DB21BCF10D0F03F8081064
:10E2280014D128494FEAE20C11F80C1041FA09F10F
:10E2380011F0010F08D0DDF818C04CFA09F111F0FF
:10E24800010F03D0582110E02D210EE0DDF820C089
:10E258004CFA09F111F0010F01D0502105E040FA04
:10E2680009F111F0010F02D0542103F8081009F147
:10E2780001095FFA89F90BF1010B08F10108013274
:10E28800B9F1080F5FFA8BFB5FFA88F81CD0B8F178
:10E29800200FB5D125E000BF2F130020961E0020C7
:10E2A800A01E00207A1A0020921E0020E81E0020DE
:10E2B800891E00206F1A0020CF1A00200C1A002097
:10E2C800F4010020281C0020B8F1200F09D09AF88A
:10E2D80000304FFA8BF2D2182B689B7C9A42FFF6DB
:10E2E80054AF23490B7813F0010F17D02B68214A3C
:10E2F8009B7C12780F2B02F0800298BFC3F11003A9
:10E30800D2B294BFDBB2002342B122789AF800104F
:10E318001032521A1849CB185F219954174EB37806
:10E3280003F00203DBB293B1F11D652246F6954373
:10E338002078FAF7FBFA2B689B7C102B02D9052072
:10E348000B2101E0002007213246FAF75BFB2B681E
:10E358009B7C102B08D921780948013102220BB087
:10E36800BDE8F04FFAF7BCBB0BB0BDE8F08F00BFBB
:10E37800D71E0020F83A0020F4010020E81E0020F3
:10E38800F50100202DE9F043002387B08DF8173000
:10E398007C4B1B78012B00F070827B4B1A789846D7
:10E3A80072B17A4BDB78002B40F06782784C237887
:10E3B800002B40F0B580FAF731FC09232370AFE059
:10E3C800734B19781C46082900F2AA80714909780C
:10E3D800232913D11A70FAF721FC6F496F4A0B7879
:10E3E80053B16F48013B0478DBB244F00604047073
:10E3F8000B706C4951F823301360AFE2684B1A7800
:10E4080012F0010F04D101210A438DF817101A7078
:10E41800F4F7A8FD28B923781BB90DF11700FFF709
:10E428007FFCF4F7ADFD30B92378012B03D10DF152
:10E438001700FFF775FCF4F7B1FD30B92378022B0C
:10E4480003D10DF11700FFF76BFCF4F7B3FD30B9FA
:10E458002378032B03D10DF11700FFF761FCF4F7C4
:10E46800B7FD48B9F4F7E0FD30B92378042B03D1A0
:10E478000DF11700FFF754FCF4F70AFE30B92378C2
:10E48800052B03D10DF11700FFF74AFCF4F7F4FD53
:10E4980030B92378062B03D10DF11700FFF740FCA4
:10E4A800F4F7A4FD30B92378072B03D10DF1170039
:10E4B800FFF736FCF4F7A8FD30B92378082B03D111
:10E4C8000DF11700FFF72CFC9DF8173043B32378A4
:10E4D800082B23D8DFE803F005080D101316191CC4
:10E4E8001F000020304901E030490020FAF7D2FA35
:10E4F80016E000202E49F9E700202E49F6E7002013
:10E508002D49F3E700202D49F0E700202C49EDE7DD
:10E5180000202C49EAE700202B49E7E7FAF77EFBC1
:10E528001B4F3B783D46092B40F0B2801C4E194FDB
:10E53800317811F0010153D1244C12222046F1F711
:10E5480029FF01236374224A98F80030137003B935
:10E558006374637C13B11F4B00221A70FFF7C2FB70
:10E568001B48617CFEF750FF337803F0FD0343F04E
:10E5780001033370184B1A7882B33A7000221A706C
:10E588002EE000BFE31E0020241A00202F130020D5
:10E59800D41E0020C01D0020B71E0020F81D00203A
:10E5A800D71E0020C41E00207EFF02085DFF02085F
:10E5B8009FFF0208C0FF0208E1FF020802000308EB
:10E5C800230003084400030865000308C21D002057
:10E5D800FC1D0020281300208C1E002030233B70D7
:10E5E8003B78884E13B97378102B4DD1DFF86492BD
:10E5F800854CFFF777FB844899F81110FEF704FF64
:10E60800237823B1002010214A46FEF79BFE98F894
:10E61800003024787D4A24EA030111707C4A23EAF9
:10E62800040111703A78A2F15200C0B2012803D94E
:10E638007078744F10280CD1002373701CB911B175
:10E648000133009311E1042373712B7801332B708C
:10E658001AE0432A18D1BBB9FC78ACB96D4BD8790C
:10E66800F7F7A4FD38B96C49FAF714FA05237B715A
:10E6780008332B7004E020466849FAF70BFA7C71DE
:10E68800674A684B1A6069E15F48FEF7ABFE65E1CF
:10E698000A2B31D15D4809F07DFCC6B2594C36B31E
:10E6A8006379042B02D100205F4903E0022B04D1D7
:10E6B8005E490020FAF7EEF902E00BB90433637102
:10E6C800314602225A48FAF70BFA5A4B1E78232E83
:10E6D80000F0D3803046FAF799FA002800F03E811E
:10E6E800312E40F03B812B7801332B7002E03B78D0
:10E6F80001333B70042332E00B2B32D1434809F03D
:10E708002FFCC6B23F4C36B36379042B02D10020EC
:10E71800494903E0022B04D148490020FAF7BAF925
:10E7280002E00BB904336371314602224048FAF71C
:10E73800D7F9404B1E78232E00F09F803046FAF719
:10E7480065FA002800F00A81312E40F007812B7805
:10E7580001332B7002E03B7801333B70082363716F
:10E76800FCE00C2B40F0FA80284809F0DFFB002180
:10E77800C4B2264809F0B0FB002C6DD0214E337985
:10E788002BB9BE2016F0D2FE337901333371737979
:10E798001C4A092B02D900201F4915E010D11D4B36
:10E7A80000241C705471264B194A18491648012533
:10E7B8001C7014700C7004700095019402949EE013
:10E7C800082B04D11F490020FAF764F911E0062B41
:10E7D80002D100201C49F7E7042B02D100201B4975
:10E7E800F2E7022B02D100201949EDE70BB90833F3
:10E7F80053717379082B3CD80D4821460222FAF749
:10E808006FF936E02F130020FC1D0020E51E0020C4
:10E81800D81E0020961E0020D2F902084EF90208E0
:10E8280078700208F81D002056FA020877FA0208E4
:10E83800F4010020C01D002014FA020835FA02086D
:10E84800C11D00206FF9020890F90208B1F9020809
:10E85800F3F90208C21D0020012542484249434AF3
:10E868002B460095F5F73CF90095414B01941B7830
:10E8780040E0404F3C78232C02D1FFF75BFA6DE073
:10E888002046FAF7C3F9002868D0303CE4B2631E8A
:10E89800DBB2012B3C7039D8022C354D1ED1E879FA
:10E8A800F7F784FC002838D02E48FFF7FDF9002838
:10E8B80033D1082246F2CE612F4803F03EF92949A8
:10E8C8002D4815F0FEFF2C49082246F2CE6003F0D1
:10E8D8002EF92949294816F00AF806E001232148AB
:10E8E8002149224A0093F5F7FBF8012300240093FD
:10E8F80001942B78029322481C49224A1A4BFFF7AD
:10E9080067F9FAF78BF9204B1C6027E0032C25D117
:10E91800174BD879F7F74AFC10B90C2373711DE02F
:10E9280000241048214616F014F828B1E02016F00B
:10E93800FDFD204616F036FE0134402CF1D1134A75
:10E948000023137073712B78114A01332B700E4B0F
:10E958001A60104B1A7842F006021A7007B0BDE828
:10E96800F08300BF281C0020C11D0020E51E0020E8
:10E97800961E0020C01D00200C1A00207A1A0020C4
:10E98800FC1D0020D81E0020F81D0020921E00202B
:10E9980078700208D71E002088234B43054A03EBF2
:10E9A800D003D35C00F0070053FA00F000F0010038
:10E9B800704700BF4C0D002070B504461646157808
:10E9C80039B912E00135EDB228462146FFF7E4FFD8
:10E9D80048B9202DF6D970BD013DEDB22846214633
:10E9E800FFF7DAFF08B1356070BD002DF4D170BDB6
:10E9F800064B38211B78032201FB003104484423CD
:10EA08000370C9B2173BC370FAF76AB8921E0020A8
:10EA1800F4010020012802D0022806D102E01D20BE
:10EA2800044904E01D20044901E004491D20FAF7C7
:10EA380031B800BF79F2020858F202089AF20208C7
:10EA4800037809680F4A03EB0310401802EBC00073
:10EA580050F8240C0C4988420FD1882101FB03236C
:10EA68009A68A0F59C63063B9A4208D0A0F5986086
:10EA78000538101A18BF0120704700207047002081
:10EA8800704700BF4C0D002037F2020803780A686F
:10EA980003EB0313D318084A053B02EBC303596879
:10EAA800064A914205D1187A09288CBF0020012016
:10EAB80070470020704700BF4C0D002037F2020855
:10EAC8002DE9F04F984B994FF0221A703B6889B0A6
:10EAD8009C6847F2F373E11A4C4244EB0104DD3AB7
:10EAE8006243934B9D5C03EB0208C5F30005EEB24D
:10EAF8003A46002E2CD130468E49F9F7CBFF8E4B83
:10EB08001B78232B41F0388298F8013066F3041300
:10EB180088F80130FAF782F8884B1A7842F0060232
:10EB28001A70874A1378013BDBB21370854A52F892
:10EB380023303B60844B1D70844B1D70844B1D70CB
:10EB4800844B1E60844B1D70844B1D7001F014BAF9
:10EB5800814D95F80090B9F1000F0CD04FF4366153
:10EB6800614309F1FF30342303FB00137C49CB18C0
:10EB78001B798DF81F307B4B1E787EB17A4E20466C
:10EB8800317810F055FE002840F05C8475493070EB
:10EB9800087007460646804600F05BBC6D490B6866
:10EBA8008B46A3F11200032809D9A3F11601032902
:10EBB80009D9A3F11A01032909D9374605E03746CF
:10EBC8004FF0010805E037460126B84601E0012765
:10EBD800B04659490978532940F0D581B9F1000F59
:10EBE8003AD1722262436149885C10F0020F0AD060
:10EBF800002B41F0C181013363F383008854CBF8C3
:10EC0800003001F0B9B95A4B997989B120464A4682
:10EC180010F0F6FDFF2801F0AF8101302870CBF825
:10EC28000090F9F7FBFF2046FFF7E2FE01F0A4B9D8
:10EC3800DFF8FCC0132202FB04C25178204669F3B6
:10EC4800041151704B4A022182F80090039310F08E
:10EC58007DFD0122039BCDE209F1FF312046C9B2B7
:10EC680010F0E6FD002840F08B80DFF810B1DFF8E7
:10EC7800EC909BF80020012332B98BF80030324B1E
:10EC880089F800201A70E4E305900393F9F7C6FFAA
:10EC980005988BF80000039B89F80030364A835C9E
:10ECA8009246A3F13001C9B2092904D9413BDBB22C
:10ECB800052B01F2618101300A28EFD14FF00008DD
:10ECC80047460AEB480015F079FE7B080237FFB289
:10ECD8000A2F294E0AF8030008F10108F1D130463D
:10ECE80011F092FA002801F04781304610F0FAFF3F
:10ECF8000746002841F040811D4B3046997911F0B4
:10ED080092FA002801F038812978337901392046B0
:10ED1800C9B202220097019611F0D8FA022389F8A5
:10ED2800003001F029B900BFE31E0020F81D0020C3
:10ED38000C3B0020C7E30208C01D0020D71E00209E
:10ED4800B71E0020C41E0020DD1D0020061E002066
:10ED5800871E0020A01E0020921E0020891E002071
:10ED680070400020D41D0020881E0020305700204D
:10ED78002F130020D61E0020B81E0020931E00204E
:10ED8800DBF80030DFF80893202B27D0212B23D184
:10ED98004FF43662624329783420013900FB01229E
:10EDA800AC489DF81F3012184FF0000B2046019216
:10EDB800C9B20322CDF800B011F088FAF9F72EFF96
:10EDC8002A78A54B013AA5481A701423C9F800B04F
:10EDD80085F800B003703CE31E2B03D10133C9F85A
:10EDE800003019E31F2B18D14FF43662624329789B
:10EDF8003420013900FB012296484FF0000B12180D
:10EE080001929DF81F302046C9B20622CDF800B005
:10EE180011F05CFAC9F800B0FEE29A1F062A0ED873
:10EE28008F4B1A7819462AB901321A708D4B1A7805
:10EE38008D4B00E3012A40F00C830223A1E1A3F1EA
:10EE48000D02042A3AD88949D3B291F800C095F83E
:10EE580000E08048864ABCF1000F1ED04FF0000C3D
:10EE680081F800C011784FF4366262430EF1FF3E1C
:10EE78000CF1340C0CFB0E228018C0184174382099
:10EE880000FB04EE5FFA8EF000EB800000F5F8401E
:10EE98001B30C01802F036FEDBE24FF0010C81F89F
:10EEA80000C04FF4366161430EF1FF3E0CF1330CA4
:10EEB8000CFB0E1E7044C3185B7C59E0A3F11202D0
:10EEC8000B2A4CD86B4A29781078002845D00020A6
:10EED8001070A3F1120938224B1E02FB0433203AAA
:10EEE800DBB2534303F5FC435FFA89F9DFF894B1C9
:10EEF8004B3303EB49039BF800101846039302F0C9
:10EF080001FE5D4A4FF4B66C0CFB04FC11781A2222
:10EF1800013902FB01C14F48494400EB41019BF80C
:10EF28000000DFF870B18875039B9BF80010581C2F
:10EF38000492CDF814C002F0E5FD4F49049A0B780D
:10EF4800DDF814C0013B02FB03C2424B4A4403EB09
:10EF580042029BF80030D3757BE2012308E0DFF81A
:10EF6800209199F800302BB9012289F80020434AF2
:10EF780013706EE2F9F752FE002389F8003020463C
:10EF8800FFF736FD65E243294BD1354A1278002A4E
:10EF980040F05F82354A1278002A40F05A82B9F16F
:10EFA800000F00F05682364A1278002A40F051824B
:10EFB800212B30D01F2B30D02E4B1978012919D98D
:10EFC800B8F1000F02D1002F00F043822D4B023917
:10EFD8001A7852FA01F010F0010F4FF0010004D036
:10EFE80010FA01F122EA010225E210FA01F141EAE0
:10EFF800020220E200F02D8209F1FF312046C9B259
:10F0080010F016FC20B9204B1B78002B40F0218211
:10F0180000232B7000E2202300E01E23CBF80030F1
:10F02800FAE1232940F096800D4B1B78002B40F025
:10F0380010820E4B1978002940F00B82104BB9F161
:10F04800000F50D01A783AB30C480F2A01700F48B5
:10F05800017042E170400020881E0020D41D00206D
:10F06800D61E0020861E0020E41E00209F1E0020C1
:10F07800541F00208B1E0020921E0020DD1D002042
:10F08800871E0020851E0020931E0020061E0020DB
:10F09800A01E0020D51E002009F1FF312046C9B26C
:10F0A80010F0C6FBB0B19A4A13787BB1B8F1000FE3
:10F0B80001D0082B08D90EB1012B05D9002F00F07B
:10F0C800C881042B00F2C281013351E79DF81F006B
:10F0D8000121F6E08F4B1A78511EC9B208296FD862
:10F0E80001321A706CE0DFF86CC2132101FB04C115
:10F0F800487869F30410487002212046049203936B
:10F1080010F024FB08F0F4FDF9F788FD824908782F
:10F1180040F006000870814801780139C9B20170D1
:10F128007F48049A50F8211011607E4A82F80090B6
:10F138007D4A82F80090039BCBF8009083F80090FA
:10F148007A4B85F8009083F80690794B83F8009005
:10F1580000F012BF2A2936D1764B1B78002B40F0DD
:10F168007881754B1A78002A40F0738173490B78BF
:10F178004BB16C48012B02706B48027040F26981F8
:10F18800013B0B7065E1B9F1000F00F0628109F1F4
:10F19800FF312046C9B210F04BFB58B15C4A1378D6
:10F1A80023B1012B40F25581013BE1E69DF81F0098
:10F1B800002186E0574A1378012B01D9013B1370CF
:10F1C8000022584B37E1442940F08D80594A127883
:10F1D800002A40F03E81B9F1000F0DD1534B9A79C6
:10F1E800511EC9B2012901D8013203E0032A40F0B7
:10F1F8003081023A9A712CE1504A1278002A40F084
:10F208002881444A1278002A40F023814A4A127819
:10F21800002A58D13E4B1B78012B09D9002E00F04B
:10F228001881474B1A78102A00F212810132AAE09D
:10F2380019D1B8F1000F0BD0424A03201178984633
:10F24800013191FBF0F000EB4000091A117000E168
:10F25800002E00F0FE803B4A1E461178013101F075
:10F2680003011170F5E0314B204699794A4610F0B8
:10F27800C7FAFF2800F0ED80DBF80030212B00F002
:10F28800E8801F2B00F0E580013028702046FFF74A
:10F29800AFFB4FF43662624329783423013903FB0C
:10F2A8000123294A9BF80000D31893F80490494693
:10F2B8008DF81F90FFF770FB0146002840F0AC80E6
:10F2C8004846224AA6E00D2B0BD19DF81F0010F0EE
:10F2D80061F930B11E4B1A783F2A00F2BA80013228
:10F2E800A9E00120AAE0552940F0B380114A12781C
:10F2F800002A40F0AE80B9F1000F2DD10B4B9A795E
:10F30800012A01D9013A75E740F0A380032271E789
:10F318008B1E0020931E0020D71E0020B71E002041
:10F32800C41E0020DD1D0020061E00202F13002013
:10F33800891E0020D61E00209F1E0020871E002048
:10F34800851E0020D51E002070400020A01E002031
:10F35800541F00200C3B0020894A1278002A78D1DB
:10F36800884A1278002A74D1874A1278002A56D11E
:10F37800864B1A78012A08D9002E6AD0844B1A784D
:10F38800012A65D9013A1A7062E012D1814B1978C5
:10F3980011B1013919705CE0B8F1000F03D00221F6
:10F3A8001970904655E0002E53D003211970164667
:10F3B8004FE0B9F1010F4CD9774BA9F10202204671
:10F3C8009979D2B210F02AFAFF2842D0DBF800303F
:10F3D800DFF8D091212B3CD01F2B3AD00130287078
:10F3E8002046FFF705FB4FF4366262432978342341
:10F3F800013903FB0123694A99F80000D31893F8EF
:10F4080004B059468DF81FB0FFF7C6FA014618B97F
:10F4180058464A46FFF7D0FAF9F700FC19E00D2BD9
:10F428000BD19DF81F0010F0B5F830B15C4B1A787D
:10F43800012A0ED9013A1A700BE0FF2058490FF043
:10F44800C7FF06E000273E46B84602E0012700E075
:10F4580001262978DFF89891002940F0CB8099F8A7
:10F46800003013F0010205D143F0010389F80030A0
:10F478004C4B1A6000252046294610F059FC30B143
:10F4880072236343484AD15C41F00201D1540135EB
:10F49800382DF0D13A356543434E735D13F0020FB2
:10F4A80043F3400015D03F4C206810B93F4900F0A5
:10F4B800CFBC00203E49F9F7EDFA735D13F00C0F4D
:10F4C80043F3810540F05885F9F7A8FB256000F063
:10F4D80053BD314DAB79A3B1012B01D1354906E0BC
:10F4E800022B01D1344902E0032B02D13349F9F749
:10F4F800D1FAA979204610F0CDF902220146304808
:10F50800EDE114B920462F4901E02F491846F9F7D3
:10F51800C1FA2E4803786BB92D490A222D48F1F714
:10F528000FFA2D49132303FB04135A7842F01002F3
:10F538005A7004E0274829490A22F1F701FA284DB0
:10F548003821022205F11E00F9F7CAFA204610F008
:10F55800C5F90222014605F11900F9F7C1FA214B54
:10F5680000221A70204B1B7803F08003DBB2002BBB
:10F5780000F002851D4B1B88EB8100F0FDBC00BF2D
:10F58800871E0020931E00209F1E00208B1E002037
:10F59800851E0020D51E00202F130020704000205B
:10F5A800541F0020A01E00203057002009E4020844
:10F5B8002AE4020832E5020853E5020874E5020865
:10F5C800120200206CE40208F0E40208D41D0020B6
:10F5D80095E50208FA0100200C3B0020B6E5020878
:10F5E800F4010020891E0020F83A0020695703081A
:10F5F800D71E002001392046C9B210F019F9002899
:10F6080000F00284954B93F800B038230BF1FF3BD0
:10F6180003FB04BB99F800305FFA8BFB13F0010F72
:10F6280003D08F4A1378002B41D08E48F9F7D8F9C8
:10F638000BEB0B1101F5E84110228B483B3102F02E
:10F648007CFA884B11229A71884B1B6813B91020D9
:10F65800874921E0012B02D1102086491CE0022BAA
:10F6680002D11020844917E0052B02D110208349CC
:10F6780012E01E2B02D1102081490DE01F2B02D170
:10F688001020804908E0202B02D110207E4903E099
:10F69800212B03D17D491020F9F7FCF999F80030A6
:10F6A8006F4843F0010389F8003000230370784B5A
:10F6B8001A78002A00F0AB800BEB0B1B0BF5E8491E
:10F6C80009F13B0910227348494602F036FA002234
:10F6D8009346704B995C41B10BF1010B5FFA8BFBC0
:10F6E8000132BBF1100FF4D107E06A49C2F11002F0
:10F6F80001EB0B002021F0F74DFE654A10785845C4
:10F708000BD90138484402F007FA30B9604B202180
:10F7180018780138484402F0F5F9DFF894B19BF8FD
:10F72800003018460393F9F771FADC46039BDFF8BB
:10F7380078B110B9432B44D101E0432B05D1002304
:10F748008BF800304FF0200A30E05348534A90F8C5
:10F7580000E053499E450ED1AEF1300E0A201378D1
:10F7680000FB0E1E0133DBB21370734493F8AD3007
:10F778007BB913700DE003709BF800304FF0000E5A
:10F7880082F800E02BB1424803780F2B01D80133EF
:10F79800037040238BF8003013789CF800200A206F
:10F7A800303A00FB0211C91891F8ADA03849394A1E
:10F7B80008785146013802F800A0484402F0A2F93E
:10F7C8000FE0384B1B7803F08003DBB24BB19BF89A
:10F7D800003033B92E482F490378FF22CB1803F89D
:10F7E800012C9BF8003013B12F4A013B13709BF892
:10F7F8000030012B10D1264A13780F2B01D8013382
:10F808001370264A00238BF80030137004E004209C
:10F818000C21144AF9F7F6F8144A13689346002B9A
:10F8280048D14FF43662624329783424013904FB05
:10F8380001241E4AA4186178164AC1F3C30109B904
:10F848003F2004E0994201D9DB2000E0A5200133E4
:10F85800DBB2907501320A2BF1D18DE3921E0020A4
:10F86800891E0020E81E0020EF1E0020A01E002098
:10F87800B3F102089DE60208DFE60208A5E70208E0
:10F888004AE802086BE802088CE80208ADE80208BA
:10F89800871E0020F4010020DA1D0020061E00202B
:10F8A800D46E0208F83A0020DD1D002078400020C0
:10F8B800C01D0020012B15D14FF4366363432A780D
:10F8C8003424013A04FB0234AB4BE418637813F098
:10F8D800070300F0518314215943A8488322F9F7FC
:10F8E800FFF849E3022B26D1A54A9DF81F3088214D
:10F8F80001FB03232978A34AD87901390623202557
:10F9080002F8015950FA03F515F0010F10D04FF421
:10F9180036656543342606FB01559B4E7519ED790E
:10F928001D4115F0010F01D0DB2500E0A52555701C
:10F93800013BE4D220E3032B13D14FF43663634336
:10F948002A783424013A04FB02348F4B1C19237A99
:10F9580013F0010F02D010208C4979E210208C4955
:10F9680076E2042B13D14FF4366363432A783424A8
:10F97800013A04FB0234844B1C19237A13F0020F5A
:10F9880002D01020834963E21020834960E2052BEE
:10F9980015D1162700262B783422013B53434FF408
:10F9A800366202FB0433784A7C49D318985DC9193A
:10F9B800013614F0E9FF0237052EECD1DCE2991F7D
:10F9C800062900F2FF809DF81F206D4F02EB021000
:10F9D800411807EBC101C968714801F1100651F8D7
:10F9E80004CBB14240F804CBF9D19E1FF6B202EB2A
:10F9F80002129219013207EBC202507A92F80AC039
:10FA0800684A29781378904673B94FF4366363438C
:10FA18003422013902FB0131634BCA5E634B024158
:10FA280002EA0C021A7011E0022B0FD1604B013967
:10FA38001B784FF0000900932046C9B204223346D0
:10FA4800CDF8049010F042FC88F8009098F8003047
:10FA5800012B29D1574BDFF8589193F800A0504655
:10FA6800F9F7D4F810B9BAF1430F1AD10DF11F0004
:10FA78005149FFF70BF810B1002389F800309DF8C1
:10FA88001F30DBF8002003EB03139B1807EBC303BD
:10FA9800504699F8001013F8202CFAF7E5F889F881
:10FAA800000099F800A003E013B9404B93F800A0B8
:10FAB800BAF1090F07D9BAF1630F8CBF4FF00309E8
:10FAC8004FF0020901E04FF001099DF81F3003EBE8
:10FAD80003139E1907EBC607FB685A7BE02A02D17D
:10FAE8002E4A202151779A7BE02A02D12B4A2021E5
:10FAF8009177DA7BE02A02D1284A2021D17798F839
:10FB080000200ABB4FF43662624329783424013955
:10FB180004FB0124184AA418A27812F0080F1BD07D
:10FB28005A7BE02A02D11D4A3F2151779A7BE02A6D
:10FB380002D11A4A3F219177DB7BE02B40F01C82EF
:10FB4800164B3F22DA7717E21C4B1B7803F0800331
:10FB5800DBB2002B40F010820DF11F001649FEF7B2
:10FB68006FFF18B15046FEF755FF05E2144851469D
:10FB7800C9EB00004A46B2E6784000200F02002098
:10FB88004C0D0020130200207040002042E70208BC
:10FB980063E7020808E80208E7E70208F401002022
:10FBA80004020020D61E002075400020861E00207A
:10FBB800E41E0020C01D0020A01E0020F83A0020EE
:10FBC80014020020A3F10D02042A31D89DF81F3039
:10FBD800D6B2222202FB03639F4A02EB83035F6CC7
:10FBE8003846F0F727FE394602469C48F0F7A8FE4B
:10FBF8009B4B1B786BB19B4B1B7803F08003DBB2EC
:10FC08001BB1994820210222FBE0984B96481978AD
:10FC18000CE04FF4366363432A783424013A04FB3A
:10FC28000234934B90481C19A619717C822256E61F
:10FC3800123B0B2B00F2A0819DF81F20DBB2222182
:10FC480001FB0231844A163152F82120834902F11E
:10FC580010008A4652F804CB824241F804CBF9D10D
:10FC6800DFF84C92DFF84CB22FB199F80020012A46
:10FC780015D1013209E096B199F80020012A07D977
:10FC88007C49097803290AD1013A89F8002006E05D
:10FC980005D178490978032908BF8BF8002099F81D
:10FCA80000209AB94FF4B6614C432A781A21013AD8
:10FCB80001FB02446E4AE318083302EB43039A79C6
:10FCC8008BF80020DA796B4B1A7055E16A4C2021C9
:10FCD80004F118000822F0F75DFBB8F1000F00D11D
:10FCE800AEB1644D2B78012B01D1644A01E04BB9C8
:10FCF800634A136823615368CAF80430B8F1000FE7
:10FD08002FD00BE0022B0CBF5E4A5F4AF1E75F4A37
:10FD1800136823615368CAF8043027E19BF8000090
:10FD2800554A3121002350FA03F515F0010F01D08F
:10FD3800117601E02D251576013301310132082BAA
:10FD4800C9B2F0D1474B1B7803F08003DBB2002B1C
:10FD580044D099F80030012B40D9E4182023A3752A
:10FD68003CE0002E00F00281202108224848F0F7EC
:10FD780011FB3D489BF800108222F8F7B1FE394B81
:10FD88001B7803F08003DBB21BB199F80030012B1C
:10FD980002D82B78032B21D1202102223248F0F7F8
:10FDA800F9FA1BE050FA03F515F0010F01D01177AD
:10FDB80001E02D251577013301310132042BC9B239
:10FDC800F0D1284B1B7803F08003DBB233B199F8EC
:10FDD8000030012B02D9E4182023A376214B1B788D
:10FDE80003F08003DBB2002B00F0C68099F80030E6
:10FDF800012B40F0C180002F40F0BE801748202121
:10FE08000822F0F7C7FAB7E099F80030214D13F04F
:10FE1800010F04BF43F0010389F800302E78002E4B
:10FE28004AD12D210A221C48F0F7B4FA04201B49B4
:10FE3800F8F730FE1A4B1B78012B02D11020194914
:10FE480006E0022B02D11020174901E017491020C3
:10FE5800F8F720FE90E000BF4C0D002004020020BF
:10FE68009F1E0020F83A002012020020541F002094
:10FE780070400020D51E0020F4010020EDF002089B
:10FE88000EF102082FF1020850F1020869F0020889
:10FE98000C020020931E0020B81E0020DCF202088D
:10FEA800891E0020C6E7020884E70208A5E70208C1
:10FEB8008B1E0020851E0020314B1C782046F8F749
:10FEC800A5FE304B304A00282AD0304F30493878C8
:10FED800A04216D130380C782E4E00EB80073C1922
:10FEE800345D04B90C700F7800EB8000C419013739
:10FEF800FFB2C0190F70315C345D59B924480170E4
:10FF080008E00120087019783C7019B1092E9CBFCF
:10FF180036182E702978511801F8014C40211970B3
:10FF2800197811B11748013901701978012909D1D7
:10FF38002978092902D8184801310170002119705F
:10FF4800134B19701168154BC3F816105168C3F894
:10FF58001A101289DA83124A127802F08002D2B299
:10FF680052B12A789B1820225A7505E09BF80000A8
:10FF78000A4A3121002315E709B0BDE8F08F00BF18
:10FF8800C01D0020DD1D0020B81E0020DA1D002045
:10FF9800061E0020D46E0208931E0020F4010020E3
:10FFA800F83A00201FB5044611B100200B4901E0C2
:10FFB80008460B49F8F76EFD217810220139C9B2BD
:10FFC80001EB011101F5C2414831684601F0B5FD68
:10FFD800102001466A46FDF7B5F91FBDD4D00208C6
:10FFE80016D102080B4B1B78442B06D0552B0378EF
:08FFF80001D013B17047013B79
:020000040801F1
:1000000001E003780133037003780BB9403302E059
:10001000412B01D1403B0370FFF7C8BFC01D00203A
:100020002DE9F74FDFF8C881DFF8D4A198F8003048
:10003000554643F0010388F800309AF80130624CCD
:1000400023F07F039B46D3B100206049F8F726FDDB
:100050005F482A21F0F720FA18B121788222F8F7B8
:1000600043FD2278002A40F0AB802B6862F3CF3347
:100070002B60584B1A7842F003021A70A0E0DFF8A8
:100080005491237099F800304E4603F00202D2B228
:100090000192514F002A40D013F0010813D0584666
:1000A0004E49F8F7FBFC3B78232B20D14C4B4D4AB3
:1000B0004D481A600121FFF779FF337803F0FE0302
:1000C0006BF3410312E040464849F8F7E7FC3B7800
:1000D000232B0CD1424B434A43481A600121FFF7BE
:1000E00065FF337868F3000368F3410333703B78AE
:1000F0002A2B65D1337803F0FE036FF3410333708D
:100100002B6843F400432B600F232370364B187881
:1001100003B0BDE8F04F0DF039BF0DF081FE05468C
:1001200000282DD001213048FFF760FF3B78532B8A
:1001300012D13378019A03F0FD0362F300033370A8
:10014000DAF8003043F40043CAF800300F2323707C
:10015000254B18780DF01AFF3B78232B30D13378DC
:10016000002203F0FD036FF3000333701E4B1A707F
:10017000F8F758FD1E4A137843F00603137015E094
:100180001C49F8F78BFC3B78232B19D199F80030E8
:1001900065F3410365F3000389F80030F8F742FD89
:1001A00098F8003043F0060388F80030124A1378BC
:1001B000013BDBB21370114A52F82320084B1A603E
:1001C00003B0BDE8F08F00BF925A002058D102085A
:1001D000F4010020073E0020C01D002079D1020854
:1001E000F81D002094700208921E00209AD1020887
:1001F000D71E0020BBD10208B71E0020C41E00205D
:10020000F83A00202DE9FF412C4D2D4C2B7843F07E
:1002100001032B70217801F00401C9B211B92948FA
:10022000FFF7E4FE284E3378232B21D12378274F84
:1002300013F004080AD0224A6FF382031370244B90
:1002400020483B600021FFF7B1FE11E0F8F7EAFC1F
:100250002B78204A43F006032B701378013BDBB266
:1002600013701D4A52F823303B60164B83F8008010
:100270003378532B1FD12378052243F004032370D6
:10028000104B16491C78013CE4B204EB840000F5E5
:10029000CA40883001F04FFC00201149F8F7FEFBFE
:1002A000FF23002100930134162004220B46019104
:1002B000029401F0B3FCBDE8FF8100BFD71E00200F
:1002C000073E0020921E0020C01D0020F81D0020C7
:1002D000B0700208B71E0020C41E0020CC700208B7
:1002E00037D102082DE9F041984B04469A7812F074
:1002F000010F00F017811B88002B40F01381944DF3
:1003000095F820303F2B40F2D780012C14D1914B2F
:100310001B7803F00203DBB2002B00F0C48095F8D9
:1003200020208B4B402A03D1013283F82020FBE0B0
:10033000482283F82020B6E0022C03D1482385F818
:100340002030B0E0844E337803F02002D2B28AB17C
:1003500095F82020402A0DD1032C0BD07F4B804AEA
:1003600003F1100153F8040B8B4242F8040BF9D14E
:10037000412395E003F01003DBB28BB195F82030F8
:10038000412B0DD1032C0BD0764B754A03F1100194
:1003900053F8040B8B4242F8040BF9D142237FE05F
:1003A000F37813F0010F0FD095F82020422A0BD1DB
:1003B0006D4B6B4A03F1100153F8040B8B4242F86A
:1003C000040BF9D143236BE003F00202D2B27AB1FD
:1003D00095F82020432A0BD1644B614A03F11001A8
:1003E00053F8040B8B4242F8040BF9D1442357E035
:1003F00003F00402D2B27AB195F82020442A0BD13E
:100400005B4B574A03F1100153F8040B8B4242F83F
:10041000040BF9D1452343E003F00803DBB28BB1B1
:1004200095F82030452B0DD1032C0BD0514B4C4A65
:1004300003F1100153F8040B8B4242F8040BF9D17D
:1004400046232DE00EF014FBA0B14B4B1B788BB173
:1004500095F82030462B0DD1032C0BD0474B404A4A
:1004600003F1100153F8040B8B4242F8040BF9D14D
:10047000472315E0F37803F04003DBB29BB195F816
:100480002030472B0FD1032C0DD03D4B344A03F1C4
:10049000100153F8040B8B4242F8040BF9D14823A6
:1004A00085F8203078E095F820300133DBB2472B17
:1004B00085F820307FF629AF95F82060472E04D9C3
:1004C000234B002683F8206001E00136F6B206F1E6
:1004D0004007FFB212E02B48314614F03EFA08B153
:1004E000032C04D1284B9B5D23B1032C02D185F84A
:1004F00020600FE00136F6B2BE4203D03F2EEAD9AB
:10050000402E07D1214B1E221A70402385F820303F
:10051000BDE8F08195F820001149652246F6954323
:10052000F8F708FA012C37D1194B0D4A03F11001E5
:1005300053F8040B8B4242F8040BF9D1044B93F8A7
:1005400020303F2B3CD9002012493EE0E81E00201D
:10055000F4010020251A0020F83A00200CD80208E7
:10056000EF1E00202DD802084ED802086FD80208CE
:1005700090D80208B1D8020864400020D2D80208FE
:1005800014D90208CF1A0020851A0020941E0020DA
:100590000C3B0308CAD70208104BD87800F02000A3
:1005A000C0B220B1022C06D000200D490DE0032C72
:1005B00001D10C4909E00C4B93F820303F2B02D8B5
:1005C00000200A4901E00A490020F8F767FA1020E4
:1005D000084A0146BDE8F041F8F718BAF83A002099
:1005E000E5CE0208EBD70208F401002088D7020804
:1005F000F3D80208E81E002010B5F8F713FB084BEB
:100600001B7803F00403DBB22BB106490020BDE8E0
:100610001040F8F743BA0220BDE81040FFF762BE71
:10062000251A0020BAD5020870B5224B06461B7861
:10063000214CF3B9257819E02048294614F08DF9AA
:1006400078B123689D4202D9FF2E02D007E0FF2E29
:1006500002D19D4208D202E036B91DB913B9256016
:1006600012E00EB9013500E0AD19EDB23F2DE3D92E
:100670000AE0013B2021124810222360EFF78EFE92
:1006800000201049F8F70AFA0F48F8F7ADF946F6D6
:10069000954320780D496522F8F74CF9084D2168FB
:1006A00005F1100001310222F8F71EFA2D23AB7478
:1006B00070BD00BF871E0020A01E0020FE1D002070
:1006C000F401002088190308E81E0020EF1E002016
:1006D000F8B5594BF02259481A700378044613F0C4
:1006E0000E051DD1564A43F00203156000F8013B88
:1006F00014F0D8F82C46534BE35C1BB1524821460A
:1007000014F015F90134402CF5D1504B01221A7028
:100710000FF0EEF94E4B1A7842F001021A70F8BD54
:1007200013F00C0543D12E464748294614F015F91D
:1007300008B10136F6B20135402DF5D11EB9237846
:1007400043F0040331E0002542482946EFB214F09B
:1007500004F968B13B4BEB5C53B13F4B01371F7061
:100760000020FFF761FF237843F00803237002E0C5
:100770000135402DE8D1394D3A212846EFF78CFE5E
:1007800038B1401BC0B20130281831460222F8F7B8
:10079000ABF9334B1B78532B4CD12F4B00201870E7
:1007A000FFF742FF237843F008032370F8BD6FF38F
:1007B0004103037003F00403DBB2294D23B1002091
:1007C0002849F8F76BF90EE02B78552B01D1FF2063
:1007D00002E0442B02D10120FFF726FF13200D2158
:1007E000214AF8F713F92B78232B23D12478134EC1
:1007F00004F00204F4B9154B1C700FF079F933784A
:1008000003F0FB0364F3C30333700D4B1C60F8F774
:1008100009FA0F4B1A7842F006021A70134A13783D
:10082000013BDBB21370124A52F82320114B1A60BD
:10083000094B1C70F8BD00BFE31E0020FD1D002009
:10084000A01E0020202D0020FE1D0020701400207E
:10085000D71E0020261A0020871E0020F401002049
:10086000C01D0020CE2A0308E81E0020B71E00206D
:10087000C41E0020F81D002070B505460C46164623
:100880003BB143004BF2B94018184018114601F033
:100890003DF9054B182202FB0535F3092C1906F02A
:1008A0007F066370E67070BD843C002038B510B3DD
:1008B000A0F14103DBB2432B1FD9C50900F07F042F
:1008C0000BD0052C19D90021601E0A460AF0F2FB54
:1008D000D0F1010038BF002038BD082C0FD9601EB0
:1008E000C0B229462A460AF05FF850B9402C8CBFA6
:1008F0000020012038BD012038BD002038BD284629
:1009000038BD284638BD0000F7B5604C312323744C
:100910005F4F01332376053B637463763B784BF27C
:10092000B9405B00181801F0FBF8C0B220F07F025C
:1009300000F07F01D2B28DF804108DF8002004F190
:10094000120359B9534A04F1150011889278618253
:100950009A7020210222EFF721FD0CE0D20904EB6E
:100960008202526A10886082927804F115009A70AF
:100970000222F8F7B9F83878400000F53440BA3070
:1009800001F0CEF8C0B220F07F0300F07F01DBB2AF
:100990008DF805108DF801303F4851B93D4B20319D
:1009A0001A889B786283837002220330EFF7F6FC8B
:1009B0000BE0DB0904EB83035B6A1A8862839B7894
:1009C000022283700330F8F78FF8344B1B7813F052
:1009D000010F5AD0324D02A92A788B1813F8041C43
:1009E00013F8086C2F4B1B78232B04D1002A41D11C
:1009F000223B2B703EE02A2B04D1002A3AD0013A48
:100A00002A7037E0552B46EA010611D10DE02B780C
:100A100002AAD318013E13F8081CF6B23046C909E1
:100A200013F8042CFFF742FF98B9002EEFD121E014
:100A3000442B19D115E02B7802A9CB18013613F8F5
:100A4000081CF6B23046C90913F8042CFFF72EFF34
:100A500038B1134B3878197832460123FFF70CFF71
:100A600008E0902EE7D905E0532B03D1533B2B70C0
:100A7000F9F7DEF80C4B1B7803F08003DBB223B1EF
:100A80002B782022023304F83320FEBDF40100202D
:100A9000871E0020CB3603080E020020D71E002040
:100AA000921E0020C01D0020F83A002002480021BC
:100AB0000922EFF773BC00BFA51E002070B50A46DF
:100AC000002405E01B19811A2A2501345D54E4B283
:100AD0000E4D0F4B295D09B19442F3D1801A0019D4
:100AE00018182021121BEFF759FC0A4B1E785EB133
:100AF000432E04D10CB1013CE4B200232B55304607
:100B0000F8F788F800B12E5570BD00BFA51E002073
:100B1000F4010020C01D002038B5184C184DA078F5
:100B200000F01000C0B250B91649F7F7B7FFFFF751
:100B3000BDFF236843F4801323600F232B702A78B2
:100B40002AB92368FF2062F31453236038BD0E488E
:100B5000C5792DB91C200821FFF7B0FF284638BD04
:100B600023680A496FF3145308222360EFF796FEB7
:100B700000280CBF0120FF2038BD00BFF83A00203C
:100B8000E61E00201DD60208A51E00202C560308D4
:100B9000F0B55C4C85B0667806F01006F6B2002E13
:100BA0003ED1594B1A78594B013A53F82230584AE2
:100BB000934204D1574B1A7842F0020207E002F147
:100BC0001C018B4208D1534B1A7842F004020221D7
:100BD00061F3C7021A7019E03832934216D1FFF759
:100BE0009BFF002800F08C8001284A4D06D12B780D
:100BF000022243F0010362F3C70306E03046464990
:100C0000F7F74CFF2B7866F3C7032B70434B1A782A
:100C100042F001021A70236843F4805323606FE0AE
:100C20003C4D2B7813F0F80606D03D49002005B066
:100C3000BDE8F040F7F732BF13F0070F41D003F0E3
:100C40000202D7B24FB11220314610F0BBF8FF2399
:100C500000930196029643202AE003F00406F6B2C0
:100C6000A6B13946384610F0ADF8382102200EF012
:100C700053FC09F0ABFC0DF0FBF8FF230093019748
:100C800002974420394604223B4614E013F0010F3A
:100C900013D0012143F6206010F094F83046F5F7A8
:100CA000F3FA204B45201E80FF2300930196029605
:100CB00031460422334600F0B1FF00201A49F7F70D
:100CC000EDFE2B7803F0FA036FF341032B70174B03
:100CD0001B78232B14D123686FF30C332360F7F7B1
:100CE000A1FF0E4B1A7842F006021A70064A1378DA
:100CF000013BDBB21370054A52F823200C4B1A60FB
:100D000005B0F0BDF83A0020B71E0020C41E002038
:100D1000D4700208145800203ED60208D71E0020C6
:100D20006A2E0308D61D0020492E0308C01D00208E
:100D3000F81D00201FB50446F5F792FBA8B14B2023
:100D400001F03AFBFF2300930121FF3B019339207F
:100D500004220B460134029400F060FF064B012090
:100D60005A7842F004025A7004E0044B18880038A4
:100D700018BF012004B010BDF43D0020A85A002087
:100D8000F0B5204E0024337A0546013385B00F4676
:100D9000337210202146012223460094F1F7B2FC61
:100DA00055B9FF2300934F20294604222B46019575
:100DB000029700F033FF0EE0012D0CD1FF230093CA
:100DC00050202346214604220194029700F026FF7A
:100DD000337A013B3372337A052B11D1FA33012177
:100DE0000024009327200B4604220194029400F073
:100DF00015FF044B1C7205B0BDE8F04001F0AEBA1F
:100E000005B0F0BD961E0020074B182202FB0033F0
:100E10005B7913F0100F05D0044B173ADA715A7052
:100E200009329A70704700BF843C00202F130020C5
:100E30002DE9F04F9A4B87B01A78074699461AB1B8
:100E4000012A40F0E68130E0964B1A68964B9A42B0
:100E500000F0E181F4F782FF944B5B7803F002032A
:100E6000DBB253B9924B5B7803F08003DBB223B95A
:100E700001F09AFA08B909F0A9FB8E4B1A686FF3D2
:100E800010421A608C4B1878F7F7C4FE002800F067
:100E9000C281FFF70BFE894B3C221A70F7F706FD63
:100EA00099F80030013389F80030844B1C7874B90C
:100EB000834B791C1A78204664F3C30264F304124E
:100EC0001A70C9B2FFF75CFF89F80040A3E17D4DBD
:100ED000384609F0B3FBF7F7DDFC00207A49F7F755
:100EE000DDFDDFF8F4812B78AA46434413F8313C4A
:100EF00023B91B200621FFF7E1FD8CE1704A0B218D
:100F0000137804A8C3F3C004C3F3001603F0F70377
:100F10006FF304131370002389F80030062200F0E9
:100F200010FE2A78414604A8303AEFF75DF9804672
:100F300028B14FF000084FF0120945462AE04AF266
:100F40006B7000F0EDFD0028F3D0604D85F808804F
:100F5000F5F76CF80446002840F05D815C4A514B7F
:100F600021461A60FF23009301900290042208207A
:100F7000234600F053FE012223460E202146009412
:100F8000F1F7C0FB534B1A7842F004021A700123A8
:100F9000AB7140E14946062204A800F0D2FD9AF860
:100FA000002004A84C49303AEFF71EF9002840F021
:100FB00021812846FFF7BEFE002840F02C81DFF893
:100FC0000CB101218BF808002846F5F73DF8814661
:100FD000F5F72CF8DA46002840F0B58048463F493E
:100FE000EFF7E0FAB0B901F0F1F82E4B14B916B9E9
:100FF0003B4A23E036B13B4A1A603B4B1A786FF309
:10100000410205E0394A1A60374B1A7866F341020B
:101010001A70D7E048463649EFF7C4FA20B148467F
:101020003449EFF7BFFA70B9002C40F0F480002E7D
:1010300040F0F18001F0CAF82F4A1A4B1A60384686
:10104000FFF7E2FEBEE048462C49EFF7ABFA50B995
:101050004AF26970012100F059FD164A136843F401
:1010600000531360E0E748462549EFF79BFA38B98B
:10107000002C40F0D080002E40F0CD80214A0CE0C2
:1010800048462149EFF78EFA002841D1002C40F064
:10109000C280002E40F0BF801C4A024B1A6091E0D3
:1010A000F41D0020F81D002028710208E234002001
:1010B000033E0020F83A0020C01D0020E61E00205C
:1010C000A41E0020DC1D0020C4CE0208961E0020B5
:1010D00044710208F1260020A51E0020B557030820
:1010E0009073020818750208D71E00203475020894
:1010F00031570308C1590308507502086C5703089B
:101100006E570308887502087E590308DC750208CB
:1011100048464249EFF746FA002853D101F056F805
:101120003CB13F4A3F4B1A603F4B1A786FF3410284
:1011300070E0002E6FD03D4A3A4B1A603A4B1A7855
:1011400064F3410266E048463449EFF72BFA06465D
:1011500020B901F03BF8002C5DD01BE04846344933
:10116000EFF720FA002856D048463249EFF71AFA2E
:1011700038B9002C4FD1304A2A4B8BF807501A60EF
:1011800049E048462D49EFF70DFA064650B9A4B19B
:1011900001F01CF8224A234B1A60234B1A7866F39D
:1011A000410237E048462649EFF7FCF920B14846AE
:1011B0002449EFF7F7F900B96CBB234A194B1A60C1
:1011C00001F004F808F56A507C308AF8075000F006
:1011D000A7FC8AF800009AF8070000F5D6406930AD
:1011E00000F09EFC8AF801001848F5F765F8402DDC
:1011F00011D108E00135EDB2402D08F1010809F1E7
:1012000007097FF4C7AE791C0020C9B2FFF7B8FD0B
:1012100001E000221A7007B0BDE8F08F7057030894
:1012200034750208F81D0020D71E0020187502082A
:101230006E5703087E590308DC750208B55703088A
:10124000315703086C570308F8750208961E0020F2
:1012500010B52148214903680A789C7B944203D940
:101260009C8914F0200F18D09A8912F0800F01D1B8
:1012700005E01C3B9A8912F0400FFAD000E01C33C5
:10128000036000230B7003689B8913F0200F16D0B6
:10129000134BDA79114B1A7011E00132D2B20A7095
:1012A000986843F60953984209D101E00132D2B25D
:1012B000162A03D80B4853B29840F7D40A700A4A4A
:1012C000136843F480731360F7F7F0FA074B1A784A
:1012D00042F006021A7010BDF81D0020871E002083
:1012E000961E002000060088F83A0020D71E002035
:1012F00010B52349234A0B78D3B11068848914F0C0
:10130000200F15D1013BDBB20B70846843F6095204
:10131000944228D104E013B1013BDBB200E0837BAF
:10132000162B03D8184C5AB29440F4D40B701AE020
:101330001368988910F0400F01D106E01C3398899A
:1013400010F0800FFAD0136002E00E481C3B0360DF
:1013500013689A7B0A709B8913F0200F03D00B4B04
:10136000DA79074B1A700A4A136843F480731360E2
:10137000F7F79CFA074B1A7842F006021A7010BD74
:10138000871E0020F81D002000060088961E002001
:10139000F83A0020D71E0020084B1A68084B9A42E2
:1013A00004D003F580630C339A4205D1054B1878BD
:1013B000003818BF0120704700207047F81D00203A
:1013C00028710208241A0020074B084A1B68934220
:1013D00002D03832934205D1054B1878003818BF37
:1013E0000120704700207047F81D0020DC750208BE
:1013F000241A00202DE9F04F814B824D1970A0F185
:101400001103DBB2012B87B00E46287006D81228D4
:1014100001D1113800E00020F4F794FF2B78522B13
:101420000DD1F1F789FE28B9F1F77AFE10B9F1F77D
:101430009BFE20B1744B1A7842F008021A70734B6D
:10144000734C1B78002B2FD12168724A91422BD00C
:10145000714A23601370714A71481178037063F305
:10146000C30163F3000163F3071111706D4A117832
:1014700063F3010111706C4A117863F3C5011170B7
:101480006A4A13706A4A117863F3410163F30001F9
:1014900063F382011170674A116863F30C311160C4
:1014A000654A1370654A93712368002B40F05F8191
:1014B000604F7B7803F02003DBB273B1604B93F88D
:1014C0000080B8F1000F08D14AF26970414600F07F
:1014D0001DFB3B6868F34D333B605A4B187810F0A6
:1014E0001E0002D00020584907E0544B93F80890A2
:1014F0009846B9F1000F05D0544907B0BDE8F04F48
:10150000F7F7CCBA524F97F801B0BA46BBF1000FCB
:101510002DD0BBF1070F15D94E48F7F765FA4E49A4
:10152000B878652246F69553F7F704FA387807231A
:1015300010F003007B700EBF484948464849F7F752
:10154000ADFA0CE0BBF1020F09D84248437823B151
:10155000F7F74AFA87F80190B4E202237B70102073
:101560003C4A014607B0BDE8F04FF7F74FBA3D4F90
:10157000BB795BB187F806B000F036FC8E20594687
:1015800001225B46CDF800B0F1F7BCF80020F1F77E
:1015900035FF224A20491378334843F0060313707D
:1015A00000230B70314923600B7088F8033088F8F2
:1015B00001300370183303FB06FC2D49934611F8E4
:1015C0000CC089461CF0080F04D130460593FFF784
:1015D0002FFC059B03FB06935B7913F0100F04D0DF
:1015E0002A78133AD2B2032A46D913F0200F79D0C1
:1015F0002B78442B40D03DD8232B3DD02A2B3AE0EA
:101600008A1E0020C01D0020771A0020E31E002043
:10161000F81D002078700208B71E0020D71E002099
:10162000921E0020D91D00208D1E0020951E002036
:10163000A41E0020F83A0020E21E00202F130020F4
:10164000241A0020915A002027CF020886000308A0
:101650008F1E0020E81E0020EF1E00202FD0020861
:101660000ED00208961E00208C1E0020871E00202F
:10167000843C0020552B35D18C4B1B78002B31D16D
:101680008B4B93F80090B9F1000F2BD143F6DB2080
:1016900000F046FA012825D13F23FB7188F80300AA
:1016A00043F63B3000F03CFA3870F87900F5D6404C
:1016B000693000F035FA78707E48F4F7FDFD9BF84C
:1016C0000030304669F341038BF8003008F0B6FF74
:1016D000F7F7A8FA784B79482360794BC3F8009064
:1016E0002B7803702B78432B0AD1714B1B783BB9B5
:1016F000013388F80330734B3046236008F09EFFB7
:1017000028781738C3B2072B27D86F49FF220AF071
:1017100075FD9AF800106D4B60F301018AF8001016
:1017200001F00301022918D00122032041B10090E9
:1017300001929B7868309B1802930021033206E0E7
:10174000009001929B786C200133029304220B4697
:1017500000F064FAFF238AF8013098F80730002B74
:1017600000F0B08152232B70594B0022DA712268AD
:10177000544B9A4250D12878A0F14303DAB2122A8E
:1017800022D8544A5BB29A401ED5432840F09A8131
:10179000464B1B78002B40F0958100F021FD4E4B0D
:1017A00048B11A7803201109013191FBF0F000EBE8
:1017B0004000091A04E01A781109013101F007010B
:1017C00061F307121A707DE1F7F724FA002823D09D
:1017D000414F3A7812F0F00308D163F307123A70E0
:1017E00023603E4B1A7842F008020EE0102B13D112
:1017F00000F0F6FC80B13B786FF307133B700023D9
:101800002360364B1A7842F0100230461A7007B047
:10181000BDE8F04FFFF70CBB314B1E211A78264F65
:1018200061F346021A702B78232B1CD12368BB422C
:1018300019D12C4B182202FB0636737913F0100FC6
:1018400011D0294B1B7873B11A4EF7F7EBF9FCF75F
:1018500075FAF07900F56A507C3000F061F930706B
:10186000AA20F1F7CBFD1C4E337813F0010F43D0C3
:101870002368BB420BD01D4A934208D0FFF78CFD72
:1018800028B9FFF7A1FD10B9AA30F1F7B7FD22681A
:10189000174B9A4202D10020F1F7B0FD2B78522B62
:1018A00040F0D5805322134BC9E000BF241A00201A
:1018B000F41D0020961E0020F87502088C1E0020E2
:1018C000C41E002028710208911E00208F1E0020D7
:1018D0002F130020002000C0D71E0020A41E0020CF
:1018E000551F0020843C0020B71E0020787002089D
:1018F00030760208C01D00202368BB420BD0734A1B
:10190000934208D0FFF748FD28B9FFF75DFD10B9F5
:10191000AA30F1F773FD2B78552B1ED1FFF7E8FCA9
:1019200033786B4843F0060333708378694F03F0D4
:101930000203DBB24BB1F7F757F823681868FAF7E0
:10194000C9F93B786FF341033B706348837803F038
:101950000203DBB20BB1F7F747F82B78442B1ED10B
:10196000FFF776FC33785A4843F0060333708378E8
:10197000584F03F00203DBB24BB1F7F735F8236899
:101980001868FAF7A7F93B786FF341033B705248A8
:10199000837803F00203DBB20BB1F7F725F82B785D
:1019A000522B09D13378002243F0010333704B4BA3
:1019B0001A704B4B45321A704A4B00271F702B7818
:1019C000232B44D1484B42481F70484B1F70F7F7F8
:1019D0000BF84148F7F708F83378454943F0060318
:1019E00033700B783B4A002B2BD0424A013B1770D7
:1019F000414ADBB20B7052F8233023603F4B1A7818
:101A000012B11F700EF074F823683D4A9B68934230
:101A100002D109F089FE1AE002F5D2718B4203D09F
:101A200002F50C718B4204D10120014606F06CFFD7
:101A30000DE002F51372934209D1324B00221A7065
:101A400005E0117863F30711117023603AE02E4B23
:101A5000DB7813B10020F1F7D1FC23681F7B17F06E
:101A60000F0702D1FBF71AFB1BE0012F02D1F8F799
:101A70008DFA16E0022F02D1F9F7F6F911E0082FDE
:101A800005D84FF09C53BB4001D5F9F79FFC042FBC
:101A900003D123689B69984703E0052F01D1F8F72C
:101AA00063FF337803F00203DBB21BB123681868CD
:101AB000FAF710F933786FF3410333702B780BB1D9
:101AC000084A137007B0BDE8F08F00BF78700208B5
:101AD000E81E0020D71E0020081E0020921E0020B5
:101AE000C01D0020DA1D0020951E0020E21E0020EF
:101AF000B71E0020871E0020C41E00207014002086
:101B00004C760208071E00202F13002007B502ABF9
:101B100003F8011D19460122002305F0A1FB0EBDAB
:101B200007B5002302A901F8013D012205F000FCE0
:101B30009DF807000EBD08B5002305F091FB0020BD
:101B400008BD034610B508461446194605F0F0FBDB
:101B5000E0B210BD10B5034600248454084619466F
:101B600005F0E6FB204610BD37B50546002400E031
:101B70001446012260190DF1070105F0D9FB9DF80B
:101B80000730621C203BDBB25A2BF1D920463EBD08
:101B9000F8B500252C461E4B1C21585D01FB043175
:101BA000400000F574506630043102220134FFF722
:101BB000C2FF1C355C2CEED143F6C43420B20422A3
:101BC00005341449FFF7B7FFA4B243F6EC339C4247
:101BD000F4D1002549F668572C4615E007EB46007E
:101BE00004EB440100B259180222FFF7A4FF0136AA
:101BF000F6B2094B5A199278B242EFD801348037C5
